:020000040800F2
:1000000000200010013B0308D1E40108E963000867
:10001000CFE40108CDE40108CBE4010800000000B2
:10002000000000000000000000000000C9E401081A
:10003000C7E4010800000000C5E401087558000885
:10004000693B0308693B0308693B0308693B0308F4
:10005000693B0308693B0308BD090008AD0A0008B5
:10006000710A0008350A0008F90900080925000886
:10007000F9240008E9240008D9240008C92400084C
:10008000B5240008A1240008693B0308693B030864
:10009000DDE80108693B0308693B030883090008A0
:1000A000AD4F00080D500008693B03081D500008C3
:1000B000FD4F0008ED4F0008DD4F0008693B0308C5
:1000C000693B0308693B0308693B0308693B030874
:1000D000693B0308A159000825590008A9580008E0
:1000E00081640008693B0308B5E40108693B030823
:1000F000BD4F0008693B0308CD4F0008693B03086A
:10010000000000000000000000000000693B030840
:10011000693B0308693B0308F9500108DD500108F9
:100120008D24000879240008652400085124000863
:100130003D240008693B03080000000000000000A7
:10014000693B0308693B0308693B030800000000A2
:10015000000000000000000000000000000000009F
:100160000000000000000000693B0308693B030831
:10017000693B0308000000000000000000000000D0
:0801800000000000693B0308C8
:10018800152303701623C370172383712D2343701F
:100198002E2303712F23C3717047002870B51EDB0F
:1001A8000928044620DD012303EB83035B00B0FB31
:1001B800F3F2092AF8D87BB10D4EB4FBF3F0092805
:1001C800CCBF57223022A6FB03E5024403FB1044B0
:1001D800EB0801F8012BF0D100230B7070BD2D2323
:1001E8000B7040420131DBE7303001F8010BF3E7D7
:1001F800CDCCCCCC884230B44FF001042ED301FBD7
:1002080004F4B0FBF4F58D42F9D284B1AAB901E047
:10021800B0FBF4F5092DCCBF572230222A4404FB49
:10022800150003F8012BB4FBF1F4002CF0D10022E7
:100238001A7030BC7047B0FBF4F5092DCCBF3722DB
:1002480030222A4404FB150003F8012BB4FBF1F417
:10025800002CF0D100221A7030BC70470546002AE5
:10026800EBD1D7E72DE9F04714461D460646002393
:100278004FF47A722046294633F06AFADFF8408153
:100288004B4A4C4F88FB00310144C31782FB002EB8
:10029800C3EB611188FB012887FB00278644464A87
:1002A800C3EBEE2EC1EB011C82FB0E29A0EB8C0CDC
:1002B8000744424A86F806C0C3EB27474FEAEE7C5C
:1002C80008EB010ACCEBA90C82FB07824FEAE17824
:1002D8000CEB4C0CC8EB6A18AEEBCC0EC8EB08184C
:1002E800DFF8E0C086F804E0A1EB880171718CFBAF
:1002F8000010F917C1EBE21240F2B55101FB12727E
:10030800C3EBE050B2F5896F4FEA80073CDA40F260
:10031800DA239A4242DCB2F5B77FB4BF4FF0000C43
:100328004FF0010C4FEA4C09DFF89C8009EB0C03F5
:1003380008EBC3031FFA8CFED88A09EB0C0108EB03
:10034800C10116310B2301E031F8020D824218DA9F
:10035800013BF9D1CC44012338F83C00B37007F2D3
:10036800B2770132121ABE44F270A6F800E02046B5
:1003780029464FF47A72002333F0EAF93281BDE856
:10038800F0870133DBB2E9E74FF0030EF44640F2A1
:100398009650DFF834804FF00609CEE74FF0020E92
:1003A800DFF82480F44640F229404FF00409C4E7FE
:1003B800C5B3A29107452EC2ABAAAA2A73B06D167F
:1003C80089888888792D03110051030803685A1C0D
:1003D8000260197070472DE9F047089C2578002BBA
:1003E800804689460CBF4FF0200A4FF0300A661C41
:1003F80035B3002A29DD334601E0024698B113F8E7
:10040800011B501E0029F8D1971E60B13D46013DE1
:1004180051464046C8476B1C002BF8DC257827EA74
:10042800E770013055B1041B29464046C8473019CA
:1004380016F8015B002DF7D1BDE8F087BDE8F0871D
:10044800002A04DC2846BDE8F0870020EBE7571EA9
:10045800DCE783684268D0ED037A00EB830101335F
:10046800934281ED040A836004BF0023836000EB9C
:10047800830393ED047A036870EE277A9A42C0EDFD
:10048800037A77EEC77AC0ED037A0CDA013307EE08
:10049800103AF8EEC76AB7EE007A87EEA60A03604C
:1004A80030EE070A704707EE102AB8EEC77A87EED3
:1004B800870A704790ED057A90ED004AD0ED066AFC
:1004C800D0ED014AD0ED047A90ED035AD0ED025AEE
:1004D800A4EE007AB0EE406AB0EE470AB0EE667A53
:1004E800A6EE247A67EEC07AA0EE457AE6EE257A83
:1004F80080ED057AC0ED067A7047D0ED057A90ED6B
:10050800013AD0ED003AD0ED064A90ED024A90ED5E
:10051800077A90ED035A90ED086AD0ED045AC0EDC1
:10052800067AF0EE406A27EE830AC0ED056AA3EE6C
:10053800A60A80ED087AA4EE240AA5EE470AA5EEDD
:10054800C60A80ED070A7047D0ED007A90ED017A6F
:1005580030EE670AE7EE007AB0EE670AC0ED007A7F
:10056800704770470A44914214D030B40139551E7F
:1005780041F2210211F8014F082380EA0420040403
:100588004CBF82EA40004000013B80B2F7D18D4267
:10059800F0D130BC70472DE9F74F6A4CDFF8A8E17D
:1005A80023880091DEF80010B4F90480C3EB21120F
:1005B8005B00C3EBE103B4F9021052435943131330
:1005C80008FB03F84FEAA83808EBE12101EB8102A8
:1005D800B1F5FA3802F180024FEAE1794FEA2223B5
:1005E80049F1FF39B4F908200193A8FB08AB08FBCF
:1005F80009F30BEB430BA161D31702FB09F108FBCD
:100608000311A2FB08230B441F03160347EA1257E2
:10061800B4F90A2002FB0BF1D3170AFB03130546B2
:10062800A2FB0A011944020A42EA016292194FEA3E
:100638002123E6887B41003243F50043A2FB0601F3
:1006480006FB03114A10CB1752EA03016FD0B4F925
:100658001060B4F90E00F71706FB0BF10AFB07113F
:10066800A6FB0AAB8B4400FB09F6C11708FB016126
:10067800A0FB08898944DEF804104FEA4846C1F512
:10068800801E4FEA494747EAD8371AEB060AB4F9F9
:100698000C8076464BEB070BF71700264FEACE7017
:1006A800F90716EB0A064FEAC80741EA5E0147EB6D
:1006B8000B0740F6354E861B61EB0707A6FB0E01BC
:1006C8000EFB071133F044F8B4F916204E13470B0C
:1006D80047EAC14702FB06FED31707FB03EEA2FB5E
:1006E80007237344564307FB0366A2FB07233344DF
:1006F800560E46EAC3163218B4F914604FEA636717
:1007080047EB01037143F71700FB0717A6FB00012E
:100718003944C60C46EA413692194FEAE147B4F922
:1007280012607B41100A40EA0360320112180DB1D1
:10073800120A2A60009B13B11A46019B136003B08A
:10074800BDE8F08F98440020C82200207047704709
:100758004FF480538382704707B5F7216A4626F025
:10076800DFFA9DF801309DF800100C4A1B0143EA9E
:1007780001339DF8021043EA111353609DF80430C9
:100788009DF803101B0143EA01339DF8051043EA65
:100798001113136003B05DF804FB00BFC8220020EA
:1007A800012380F84530704770B40468037B2268E1
:1007B800022101FA03F31A4213D042690A495C2064
:1007C80000FB02124FF6FE7650685289C568006831
:1007D800296831402960C168D24392B20A40C26098
:1007E800636070BC704700BF4859002030B40A4BA2
:1007F8001D7875B1094B002003EBC5051A68998867
:100808005062D4682143D160083323F8040CAB420A
:10081800F4D130BC704700BF285C00202C5C00205D
:1008280010B40268047B11680223A340194209D05E
:100838000649406800240C7001684FF6FE74214098
:10084800016053605DF8044B704700BFF44D002011
:100858000023012203604360037083700271837177
:1008680070472DE9F341056906460F467DBBD0F870
:100878000080C8F30A0323B30023D6F8008001934D
:1008880027F05CFA042819D1214C236943F00103AD
:100898002361BBB2A8F8003027F050FA04282ED103
:1008A80008F102030193019B3F0C1F8027F046FAD1
:1008B8002369042823F00103236125D06FF0010583
:1008C80005E027F03BFA042805D04FF0FF3528460D
:1008D80002B0BDE8F0810E4C236943F002032361A6
:1008E800C4F81480236943F04003236127F026FAF3
:1008F8002369042823F002032361BDD0E5E72369B7
:1009080023F001032361D9E7336804333360DEE75A
:1009180000200240F8B504460D468E180027B5425F
:1009280001D12069F8BDE368591CE160234415F83A
:10093800012B1A720429F2D1A1682046FFF791FF12
:10094800E7602061EBE7024B186805F0CBB800BF01
:100958005C23002026F0C8BA10B490E80600047B97
:1009680040690223A3404B6013685DF8044B4FF6BF
:10097800FE710B40136005F04DB82DE9F0410B4EA8
:10098800346873691C400FD0DFF824800127B4FA5B
:1009980084F3C3F11F0307FA03F558F8230003682B
:1009A8009847AC437561F2D1BDE8F081000401407D
:1009B8001C2300202DE9F0410B4E346873691C405C
:1009C8000FD0DFF828800127B4FA84F3C3F11F039E
:1009D80007FA03F558F8230003689847AC43756194
:1009E800F2D1BDE8F08100BF000401401C230020C3
:1009F8002DE9F0410B4E346873691C400FD0DFF8C5
:100A080028800127B4FA84F3C3F11F0307FA03F51A
:100A180058F8230003689847AC437561F2D1BDE8E4
:100A2800F08100BF000401401C2300202DE9F041A3
:100A38000B4E346873691C400FD0DFF828800127FB
:100A4800B4FA84F3C3F11F0307FA03F558F8230037
:100A580003689847AC437561F2D1BDE8F08100BFE7
:100A6800000401401C2300202DE9F0410B4E34689E
:100A780073691C400FD0DFF828800127B4FA84F38B
:100A8800C3F11F0307FA03F558F8230003689847D2
:100A9800AC437561F2D1BDE8F08100BF00040140AC
:100AA8001C2300202DE9F0410B4E346873691C406B
:100AB8000FD0DFF828800127B4FA84F3C3F11F03AD
:100AC80007FA03F558F8230003689847AC437561A3
:100AD800F2D1BDE8F08100BF000401401C230020D2
:100AE800084A094808B5936943F001039361002156
:100AF800402234F092FA054B4FF0FF329A60C3F867
:100B08000B2008BD001002401C230020C822002032
:100B180003681B6A184770B44E1C0568C272867257
:100B2800AC69A44670BC60472DE9F04104461846FC
:100B38000D461646984632F041F92768E672284471
:100B4800A07229467D69434632462046AC46BDE838
:100B5800F0416047036810B504461B68984723684E
:100B680020469B689847A37B0133A37310BD036895
:100B78001B69184710B5036804469B689847FF230C
:100B880001226373227310BD08B5212004F0E4F933
:100B98000C4B186018B1112200238271C3712021F7
:100BA80005F008FA202004F0D7F9074B186018B1AF
:100BB800112200238271C3712021BDE8084005F08D
:100BC800F9B900BF5C2F0020602F002008B504F0A1
:100BD800C3F940B12D2282710022C2712021BDE8E3
:100BE800084005F0E7B908BD0B4B984206D0A3F5BD
:100BF800784398420DD04FF0FF3070470022074BE2
:100C080003EB02135A89013292B25A81588980B291
:100C180070470122F3E700BF003001406444002020
:100C2800F0B5836983B0054613B11A689B881385AC
:100C38006869264F8389C3244FF47A734FF0060EF0
:100C48006E464FF6FF71013703E0013B9BB28B42C2
:100C58001DD002899207F8D504734FF47A7302E025
:100C6800A3B28B4213D00289D20703F1FF34F7D520
:100C7800027BD2B20EB132700136BEF1000F08D03D
:100C88000EF1FF3EFF24002FE3D03C78DBE7FFF7AF
:100C9800ABFFAB6913B11A689B8893619DF8050097
:100CA8009DF801609DF802109DF803409DF804200E
:100CB8009DF8063041EA062143EA002342EA04226D
:100CC800012029876A87AB8703B0F0BD605103080C
:100CD800427A02B9704710B504460368406804F1C7
:100CE8000A0198470023637210BD437A5A1C0344D3
:100CF800D2B242729972037A934200D802B970470D
:100D080010B504460368406804F10A0198470023B7
:100D1800637210BD98B10B4B012210B402FA01F1B5
:100D280003F1750402E00333A34209D01A78824222
:100D3800F9D15A780A42F6D001205DF8044B704781
:100D48000020FAE76851030830B40A4D002305F182
:100D5800680401E0272B0AD003EB43020133A15CAE
:100D68008142F7D12A4430BC92F86A0070470020CB
:100D780030BC70470051030870B5448806460D46DC
:100D8800C4F30B0422460021284634F046F933699F
:100D9800094A934209D3094A934206D22246284671
:100DA8001946BDE8704032F0A5BF23B12146284658
:100DB800BDE87040184770BD34B903081EBA03086F
:100DC800064B07498B4202D30023184670471A88FE
:100DD800C2F30B029042F8D01433F3E798B4030837
:100DE80034B90308024A136823EA00001060704708
:100DF800C0360020F8B5174D2B78A52B28D16B7875
:100E0800BE2B25D1022229464FF6FF70FFF7AAFB19
:100E1800114FAC1C22884AB1A618BE4218D2052A26
:100E280016D92146FFF79EFB3446F3E721460222F6
:100E3800FFF798FB0222A118FFF794FB0634074B33
:100E4800641B1C8041F60F53C31A58425841F8BD21
:100E58000020F8BD00F00308000004082433002037
:100E68002DE9F04FDFF848914C4F8BB00326A7EBE4
:100E780009071822002104A834F0CFF8484BCDF810
:100E8800109005971A69120604D5464A5A6002F16D
:100E980088325A6001228DF824203422DA60424BCD
:100EA800424C1B88ADF800300222694604A8FFF7BF
:100EB80031FD022269464FF6FF70FFF753FBDFF85A
:100EC800F4A080464FF0000B544536D30AAC0025F9
:100ED80024F8245D0222214604A8FFF71BFD022204
:100EE80021464046FFF73EFB40BAC043ADF8080034
:100EF800022202A904A8FFF70DFD079860B106AB0E
:100F0800C0F104022946184434F087F8069904A869
:100F1800FFF7A7FC079508909DF82430089A23B19D
:100F28001F490B6943F080030B61013E2DD0002A55
:100F38009FD1FFF75FFF50B32CE065888DF80DB0A7
:100F4800C5F30B05AB1DADF808302388C3F30B02BE
:100F5800ADF80A201B0B062202A904A88DF80C3054
:100F6800FFF7D8FC062202A94046FFF7FBFA6168A2
:100F780080462A4604A8FFF7CDFC616840462A4609
:100F8800FFF7F0FA143480469EE7002AD1D00520F6
:100F980002F090FE0BB0BDE8F08F00BF000004081F
:100FA8000020024023016745DD51030898B4030877
:100FB80000F0030834B903080378202B024600F137
:100FC8000100F9D0092BF7D02D2B2CD02B2B03BFE8
:100FD8005378B7EE000A0246B7EE000AA3F13001D3
:100FE800C8B209289FED467A10D8F2EE046A07EED7
:100FF800901AF8EEE77A12F8013FE7EE267AA3F1A5
:101008003001C8B20928B0EE677AF0D92E2B4CD03F
:1010180003F0DF03452B0BD0F7EE007A67EE276A63
:1010280020EE260A70475378BFEE000A0246D5E73D
:1010380010B451782D2959D02B290ABF9178501C0A
:10104800901C0024A1F13003092B53D8002303EB93
:10105800830301EB430310F8011FA1F13002092AB1
:10106800A3F13003F3D9B3F59A7F28BF4FF49A73ED
:10107800072B42D9DFED236A1A46F7EE007A083AC1
:10108800072A67EEA67AFAD803F007032BB1F2EE27
:10109800046A013B67EEA67AFBD124B3C7EE276A40
:1010A8005DF8044B20EE260A70475378A3F130010F
:1010B800C8B2092802F10102AAD8F2EE046AF0EED9
:1010C800665A07EE901AF8EEE77A12F8013F87EEB3
:1010D800A66AA3F13001C8B2092866EEA56A37EE00
:1010E800067AEED994E767EE276AD9E7901C9178DB
:1010F8000124A7E7F7EE007ACFE7F7EE007AC5E715
:101108000000000020BCBE4CB5EEC00ADFED317A0D
:10111800F1EE10FACCBF30EE270A30EE670ADFEDA9
:101128002E7A20EE270A30B5FDEEC07A87B017EE8A
:10113800904A054684EAE470002303A9A0EBE47012
:1011480001930093029330F069F8002CACBF202380
:101158002D2303A88DF8003031F030FE012803A9B3
:1011680024D002282DD0032805BF302368466846BE
:101178008DF8013033F059FF684631F01FFE03380F
:10118800C4B222466946284633F086FF00232B5511
:10119800284631F013FE2E22431C2A540DEB04017D
:1011A800E81833F05FFF284607B030BD30236846A3
:1011B8008DF801308DF802308DF8033033F035FFAB
:1011C800DAE7302368468DF801308DF8023033F0C5
:1011D8002CFFD1E76F12033A00007A442DE9F04161
:1011E800064615460846B6FBF2F43CB905FB1464FE
:1011F800124B1B5D00F8013BBDE8F081B4FBF2F730
:1012080067B90E4B05FB174705FB1464DA5D00F858
:10121800012B1B5D00F8013BBDE8F081B7FBF2F83C
:10122800B8F1000F02D04046FFF7D8FF05FB187849
:10123800024B13F8082000F8012BE3E7C47B0308EE
:10124800104B2DE93048D3E9004554EA05020BD18B
:101258000346012200201871587198719A70DA704B
:1012680018801881BDE83088074B1A6814EB020B08
:1012780045F1000C5A466346FEF7F4FF0120BDE82D
:10128800308800BFC8240020B0620020F0B4028873
:101298008578154FC37804794179A2F2B27202F0C9
:1012A800030606EB4606013D05EB8605013B37F8CC
:1012B80015608579008940F2B557920807FB02321C
:1012C800931903EB430304EBC303C3EB031301EBD1
:1012D8008303C3EB031305EB830300214FF47A72F6
:1012E800C2FB0301F0BC704700510308FAB170B4A7
:1012F8008E18044603E0101A14D1B14214D014F821
:10130800012BA2F14103192B11F8013BA3F141056F
:1013180098BF2032192D03F12000ECD9D01A01D141
:10132800002BEAD170BC7047002070BC7047104693
:1013380070474FF0FF32FFF7D9BFA0F16103192BB7
:1013480098BF20387047A0F14103192B98BF20306F
:101358007047202805D0093804288CBF00200120B8
:10136800704701207047613819288CBF0020012080
:101378007047413819288CBF002001207047303849
:1013880009288CBF002001207047A0F13003092BE9
:1013980007D920F02000413819288CBF00200120EF
:1013A80070470120704730B402681146531C03602F
:1013B80011F8024B0160D31C517803609378151D16
:1013C80005601B0443EA0123D078234343EA006005
:1013D80030BC70470368591C1A46016012F8021B9A
:1013E8000260587841EA0020704703685A1C02607E
:1013F8001878704738B504460068154632F07AFC0C
:1014080022682A44226038BD036810B40A0A5C1CAA
:1014180004601A7003685A1C026019705DF8044B66
:10142800704703685A1C026010B4197003680A0AEE
:101438005C1C04601A7003680A0C5C1C04601A7057
:101448000368090E5A1C026019705DF8044B704756
:1014580003685A1C026019700368090A5A1C026062
:10146800197070472DE9F047002488B080460F4670
:101478001E46A14605AD531C0393117839B325299F
:1014880033D1931CCDF810900393507830284ED068
:101498004FF0000AA0F13003DBB2092B42D96C28C7
:1014A80019D0642800F0938024D825281CD063D94B
:1014B800582876D063281BD131784046B847039A1C
:1014C800531C03931178043601340029D7D12046E0
:1014D80008B0BDE8F087039B5A1C03921B78642B65
:1014E8007CD02AD8252B54D1252140460134B84731
:1014F800039AC0E7732833D044D975284FD106F131
:10150800040E30682B4600220A217646FEF772FE4A
:10151800049A0095534639464046FEF75CFF039A05
:101528000444A8E704AA03A926F078FCB7E7D31C6B
:10153800039390784FF0010AACE7732B10D05BD976
:10154800752B3AD0782B96D1A3F15802B2FA82F2D1
:10155800306852092B4610210436FEF74BFED7E7B8
:101568003368049A0093394600234046FEF733FF58
:1015780004360444039A7EE70028B9D1204608B00F
:10158800BDE8F0876E28B3D1039A336804361C602F
:1015980071E72AD9582BD7D0632B8DD06BE77828E1
:1015A800A6D1A0F15802B2FA82F2306852092B464D
:1015B8001021FEF71FFE0436AAE706F1040E306874
:1015C8002B4600220A217646FEF714FEA0E7331DBB
:1015D800306829461E46FEF7E0FD99E7331D30685E
:1015E80029461E46FEF7D9FD92E7002B7FF443AF4C
:1015F800204608B0BDE8F0876E2BC6D03BE70EB496
:1016080000B584B005AB019053F8042B0649039349
:1016180001A8FFF727FF019B00221A7004B05DF8AC
:1016280004EB03B0704700BFD50300082DE9F0476D
:1016380007468CB01E469246002A6AD115461446C3
:101648000A8840F2B1739A423AD98B78581E0B280F
:1016580036D891F803E00EF1FF301E2830D891F803
:1016680004C0BCF1170F2BD891F80590B9F13B0FC6
:1016780026D888793B2823D8B1F80880B8F57A7F2E
:101688001ED24FF00108002E34D109890491002C94
:10169800B4BF2D212B21002CB8BF644203900591C3
:1016A8000795CDF80890CDF804C0CDF800E038468D
:1016B80006942F49FFF7A3FF40460CB0BDE8F0871A
:1016C8000023012118468E46ADF824308DF82830C5
:1016D8008DF829308DF82A30ADF82C3099469C4683
:1016E8001A4698468DF826108DF827100B4609A93A
:1016F800002ECAD00390CDF80890CDF804C0CDF8DC
:1017080000E038461B49FFF77AFF40460CB0BDE8B9
:10171800F087194C84FB0234A318D417C4EB631464
:10172800C4EB0415A2EB85052DB2002D0846B8BF01
:101738006D42FFF7ABFD4FF47A720023804689466D
:1017480032F006F83C230AFB030A4FF47A720023AE
:101758004046494631F0FCFF4FF47A7192B20023BB
:10176800C1FB0A2309A8FEF77DFD24B209A967E792
:101778000C7C0308EC7B0308898888880FB430B593
:1017880083B006AB0B490C4853F8042B0968006872
:101798000193FFF767FE094C0546206803685B69FB
:1017A80098470028F9D0284603B0BDE8304004B077
:1017B800704700BF502F0020542F00205C230020CA
:1017C800DFED2B7AB4EEE70AF1EE10FA4ADDDFED31
:1017D800296A9FED297A01E0B0EE670AB4EEC70ADC
:1017E800F1EE10FA70EE667AF6DC9FED247AF4EEEC
:1017F800C77AF1EE10FA38D5DFED1E6A9FED207A30
:1018080001E0F0EE407AF4EEC77AF1EE10FA37EE26
:10181800A60AF6D4DFED1B7AB4EEE70AF1EE10FA69
:1018280014DDDFED137A37EEC00A60EE006A9FED33
:10183800166A9FED167ADFED167AA6EE867A20EE06
:10184800266AE6EE877AA6EE270A7047DFED117A58
:10185800B4EEE70AF1EE10FA44BFDFED087A37EE8E
:10186800C00AE2E7F0EE407ABFE7B0EE670AD1E7D8
:10187800DB0F4940DB0FC940E4CB1641DB0F49C001
:10188800E4CB16C1DB0FC93F92E741B99730083C5A
:1018980015A82ABEDB0FC9BF09B909E0194690FB94
:1018A800F1F301FB13030846002BF7D108467047F4
:1018B8000146FBE707EE901AF8EE677A9FED837A08
:1018C80027EE800A20EE070AFDEEC07A17EE903A5E
:1018D8002033402B00F28C80DFED7D7AB4EEE70AEE
:1018E800F1EE10FA40F3E880B0EE407A9FED796AA5
:1018F800DFED796A01E0B0EE677AB4EEE67AF1EEF0
:1019080010FA77EE467AF6DC9FED747AF4EEC77A31
:10191800F1EE10FA40F1CD809FED6E6ADFED706A4E
:1019280001E0F0EE477AF4EEE67AF1EE10FA37EEDF
:10193800867AF6D4DFED6B7AB4EEE77AF1EE10FA38
:1019480051DCDFED697AB4EEE77AF1EE10FA44BFC4
:10195800DFED627A37EEC77A27EE076ADFED635A62
:10196800DFED637ADFED636A9FED635AE6EE257A71
:1019780067EE065AE6EE276AF7EE007AA5EEA67A33
:10198800F0EE675AE7EE055AE7EE457A87EEA55A74
:10199800DFED547A30EE277AFDEEC76A16EE903AFC
:1019A8002033402B29D99FED557AF6EE006AB7EE21
:1019B800006AF7EE004AC4EEA57A0023836143610A
:1019C8000362C36180ED045A67EEA66A27EE866A51
:1019D80027EE877AC0ED006AC0ED026A80ED016AE1
:1019E80080ED037A7047DFED3A7A37EEC77AB3E7CE
:1019F800B7EE005AF0EE455ACAE7B4EEE70AF1EE40
:101A080010FA5FDD9FED336ADFED336A01E0B0EE77
:101A1800677AB4EEE67AF1EE10FA77EE467AF6DCFB
:101A28009FED2E7AF4EEC77AF1EE10FA47D59FEDC6
:101A3800296ADFED2B6A01E0F0EE477AF4EEE67AE8
:101A4800F1EE10FA37EE867AF6D4DFED267AB4EEA8
:101A5800E77AF1EE10FA27DCDFED237AB4EEE77AC5
:101A6800F1EE10FA44BFDFED1D7A37EEC77A27EEA4
:101A7800076ADFED1E4ADFED1E6ADFED1E7AE6EE2D
:101A8800246A67EE064AE6EE267AB7EE006AA4EE06
:101A9800A77AF6EE006A36EE476AF8EE007A27EE85
:101AA800277A66EE266A84E7DFED097A37EEC77A89
:101AB800DDE7B0EE677A3DE7F0EE407A24E7B0EE76
:101AC800677AC2E7F0EE477AAAE700BF27D4D23692
:101AD800DB0F4940DB0FC940E4CB1641DB0F49C09F
:101AE800E4CB16C1DB0FC93FDB0FC9BF92E741B991
:101AF8009730083C15A82ABEF304353F0000008043
:101B080010B44C09012250F8243001F01F0102FAE8
:101B180001F10B4340F824305DF8044B70474B0942
:101B280001F01F0150F82320012303FA01F11142AB
:101B380014BF18460020704708B540F2E93300E0AA
:101B48009BB10289013B12F0020F9BB2F8D00173DE
:101B580040F2E93300E043B10289013B12F0010F82
:101B68009BB2F8D0007BC0B208BDFFF73DF8C0B209
:101B780008BDF8B584894FF6FF764FF47A742BB315
:101B880011B30F78013101E0B44217D00589013C47
:101B9800AD07A4B2F8D507734FF47A7402E0BCB26B
:101BA800B4420BD00589ED0704F1FF37F7D5057B63
:101BB800EDB20AB115700132013BE0E7FFF714F806
:101BC800003018BF0120F8BDFF27DFE70120F8BD6E
:101BD800028822F040021204120C0280028822F0CD
:101BE80038031B041B0C59B141F48071002991FA88
:101BF800A1F2B2FA82F108BF4FF0FF310139C900F2
:101C08000B439BB2038003889BB243F040030380DD
:101C180070472DE9F84F334ADFF8D8A03248DFF88B
:101C2800D8B0DFF8D880012304211370FFF7D0FF64
:101C3800DAF8000004F07AFB05212B48FFF77CFF57
:101C480000212948FFF778FF06212748FFF774FF8E
:101C580000212548FFF770FF9BF800402248042127
:101C680044F00104FFF768FF21461F48FFF764FFAF
:101C7800B8F80030B3B11D4D1D4F1B4E002495F828
:101C8800019007213046FFF757FF49463046FFF7D6
:101C980053FFB8F8003015F8012F07F8012F013469
:101CA8009C42ECDB07211048FFF746FFFF210E4856
:101CB800FFF742FF9BF800400B480421FFF73CFF69
:101CC80021460948FFF738FFDAF8000004F034FB32
:101CD80002210548FFF77CFF024A00231370BDE884
:101CE800F88F00BF1D4E002000300140EB4B002054
:101CF800334E0020B86100206C520020680B002091
:101D0800F8B5114D114FC1F1030646EA80060421CA
:101D18002846FFF75DFF386804F008FBF6B2102488
:101D2800E1B22846FFF708FF013431462846FFF79D
:101D380003FF202CF4D1386804F0FEFA022102488F
:101D4800BDE8F84044E700BF00300140B86100201A
:101D5800F8B5444C44480421FFF73AFF206804F0E2
:101D6800E5FA424B1B78012B6DD058D3022B4ED18C
:101D78003F4D08232B704FF4C3733E4E3E4F3380C4
:101D880002210020FFF7BCFF04213748FFF720FF9E
:101D9800206804F0CBFA2D7833480021FFF7CCFEF9
:101DA80029463148FFF7C8FE344B2F481D780221D9
:101DB800FFF7C2FE29462C48FFF7BEFE304B2A48E3
:101DC8001D780321FFF7B8FE29462748FFF7B4FE20
:101DD8002C4B25481D7804210D43FFF7ADFE2946FD
:101DE8002148FFF7A9FE206804F0A6FA02211E4840
:101DF800FFF7EEFE32882448002133F00EF93B78D5
:101E080063B1224B1B7823B300233B70F8BD184DF8
:101E18002B785B06AFD54FF4F073AEE7F8BDA02181
:101E28001148134DFFF788FE00210F48FFF784FE85
:101E380000F00603022B03D000F0050001280DD0A6
:101E480008232B7097E70A4D48232B704FF4F07343
:101E580093E7FFF7DEFE00233B70F8BD48232B70A5
:101E6800D9E700BFB861002000300140BC61002004
:101E78006B0B0020680B002000000020C3610020CD
:101E8800C46100206C520020344E00201D4E0020FA
:101E9800F0B55B4B5B4A97B01968914200AF00F010
:101EA800A3805949594A00234FF47000C1F88800AB
:101EB8003B607B60136843F48033136003E03B6846
:101EC800B3F5A04F09D0136803F400337B603B6877
:101ED80001333B607B68002BF1D04C4B1B6813F43B
:101EE800003318BF01237B607B68012B52D0464C1E
:101EF800464B474AE260474A596A11605A6A42F0BB
:101F080080725A625A6942F4FC025A61002503221F
:101F180007F10801012341F6FF764FF09040FD607C
:101F2800BE603A73BB732CF075FE4FF6FF7307F172
:101F380008013948BB602CF06DFE07F108013748ED
:101F4800374E2CF067FE07F1080136482CF062FE88
:101F580007F1080134482CF05DFE07F10801334809
:101F68002CF058FE07F108002CF0ADFEBB68304994
:101F7800304AA1FB031330499B0CF0204FF0070EA9
:101F88005C370B60566084F823009560C2F800E067
:101F9800BD46F0BD294A1D4B122111605A685A608E
:101FA8005A685A605A6842F480625A605A6822F441
:101FB8007C125A605A6842F4E8125A601A6842F071
:101FC80080721A601A689201FCD559680F4A21F08C
:101FD80003015960596841F002015960536803F0E0
:101FE8000C03082BFAD182E700221A6062B6144B60
:101FF8001B6883F30888134B1B689847FEE700BFEC
:10200800FC9F0020EFBEADDE00ED00E000100240B6
:102018000005FA055C740020000400480008004828
:102028003F190100000C0048001000480014004847
:1020380083DE1B4310E000E0B46200200020024071
:1020480000D8FF1F04D8FF1F70B50F4C0F4DC0EB11
:10205800C00004EB8004686926693043686182B077
:102068009209667BA1600025012101A863618DF8B2
:1020780004608DF805208DF806508DF807102CF0B7
:1020880093FD02B070BD00BF700B0020001002402D
:10209800074BC0EBC00030B403EB8000054C05696A
:1020A80063692B4363610176427630BC704700BF99
:1020B800700B0020001002402DE9F04F5E4C54F8E0
:1020C800204083B0002C71D0A66D984691465B4B9A
:1020D80072682265A160236004F15E014FF4807389
:1020E80004F5AF726161A261E36023610746307E47
:1020F80025F082FFF068A8B1514B00215A68904240
:1021080003F11C0300F0928001310C29F6D1002064
:102118007A1CD2B20C21FFF7BBFF236DF268626311
:102128002433E364B068D8B1454B00215A68904223
:1021380003F11C0378D001310C29F7D100257A1C52
:10214800D2B20B212846FFF7A3FF2346F27E3D4972
:102158002846FFF779FF236DB268A2632833A3648A
:1021680094F85D0002F0F8FE054694F85C0002F071
:10217800F3FE18F0080F824696F819B01AD0CDB1C0
:1021880018F0110F4FF00B0307F1010714BF4E2190
:102198003E21EF715A46AB71284602F03DFB18F01C
:1021A800010F45D0636B5BB3A36B4BB3204603B001
:1021B800BDE8F08F18F0010F0CBF4FF02E084FF05C
:1021C8004E0819F0020F09D045B10B227B1CAA71E9
:1021D800EB7128465A46414602F01EFB19F0010FE2
:1021E800E0D0BAF1000FDDD001370C238AF8077070
:1021F8005A4641468AF80630504602F00DFBD1E7B0
:10220800337FB27E8DF804209B090021012201A8AA
:102218008DF805308DF806108DF807202CF0C4FCD9
:10222800204603B0BDE8F08FCDB288E7C8B26FE7AB
:10223800284604F07BF8B5E7642F0020E051030836
:10224800700B00206109000800B97047F0B595B01F
:10225800054626F0B1F96E4EC3680268326004463E
:10226800002B00F0C380284602F076FE694B186107
:1022780018B1292200238271C371227A664D2E215A
:1022880002F0CAFA306803F03DF825F0B5FE306870
:10229800624A038823F001031B041B0C038014A962
:1022A8001E232B8001270F230025138021F84C7D46
:1022B8002D230293ADF80C50ADF80650ADF80E5032
:1022C80026F028F9E379ADF8145060229907ADF8A3
:1022D80016500695ADF81C50ADF81E50ADF82050BC
:1022E800ADF82250049200F1838013F0010F14BF5F
:1022F800022200224FF48073ADF81470ADF81C2050
:10230800ADF82030002304AA61793068069302F002
:1023180087F83068617926F0DDF83068436C43F45B
:102328000043436403889BB243F080030380E3794E
:102338009B0768D56179026A04238B4022EA03026D
:102348000262026A134303623268354F13889BB2F4
:1023580043F001031380207C00222921FFF798FE17
:102368003049207C00236022FFF76EFEE068386069
:102378002CF086FB386803684FF6FE721340036042
:102388002CF07EFB09A81DF0B7FF33686279264957
:1023980038680A91343313440993802210230025A6
:1023A80009A940F22A3E0E920B934FF400724FF4A3
:1023B80000530D951095139511950F921293ADF842
:1023C80030E01DF0A7FF627933680C2A98BF1749DF
:1023D800D86898BF31F812503A6815490543DD604E
:1023E8001368012043F002031360087015B0F0BDB4
:1023F80013F0010F14BF08222A460423ADF81E204B
:10240800ADF816307EE7012261791DF057FE9BE793
:10241800F0360020C8220020E6360020E4360020EE
:10242800EC36002029080008643A00209C73030851
:10243800E83600200348D0F83C3113B100F59A7013
:1024480018477047700B00200348D0F8203113B1AB
:1024580000F58C7018477047700B00200348D0F8BF
:1024680004310BB1FC301847704700BF700B0020D7
:102478000348D0F8E8300BB1E0301847704700BF88
:10248800700B00200348D0F8CC300BB1C43018478B
:10249800704700BF700B00200348D0F8B0300BB174
:1024A800A8301847704700BF700B00200348D0F8C9
:1024B80094300BB18C301847704700BF700B002068
:1024C8000248836F0BB1703018477047700B0020BB
:1024D8000248C36D0BB1543018477047700B002089
:1024E8000248036C0BB1383018477047700B002056
:1024F8000248436A0BB11C3018477047700B002024
:102508000248836803B11847704700BF700B00206A
:10251800F8B505015A4C5B4B625961199A4204EBB4
:10252800050704BF01230B730646387A25F064FDBE
:102538003B7A03F01F015B090122022B02FA01F228
:1025480078D0032B71D0012B67D063190136187925
:1025580002F002FDF6B2074610B11223C67183716C
:102568006319587902F0F8FC10B11323C67183710E
:102578006319987902F0F0FC10B11423C6718371C5
:1025880066190E21F279384602F046F9707902F0A0
:10259800E3FCF2790E2102F03FF9B07902F0DCFC9D
:1025A800F2790E2102F038F96359374A934251D033
:1025B800344A934259D0354A934240D02C44227B26
:1025C800002A2FD1012002249A8822F48052120472
:1025D800120C9A80998889B241F4805199801A889E
:1025E80002F4415242F44572024322431A809A8807
:1025F80022F470621204120C42F4E0629A809A8B00
:1026080022F400621204120C07219A8319821A8894
:1026180092B242F040021A80F8BD1D4B996A0A43F3
:102628009A6292E700200446CEE7194B19690A43DB
:102638001A618AE7164BD9680A43DA6085E702F51A
:10264800EA32116941F400411161116921F4004134
:102658001161B3E702F56042D16841F48051D1605D
:10266800D16821F48051D160A8E702F5EC321169F4
:1026780041F480411161116921F4804111619DE7A4
:10268800644400200038004000300140003C004015
:1026980000100240F0B53A4C059D00EB800004EBB9
:1026A80080046468002C69D0364E49004FF42040FD
:1026B800CFB23060A169090453D46068DFF8D0E074
:1026C80047F4903100EA0E0001434FF42040616066
:1026D800306003E0411E002847D00846A1698907F9
:1026E800F8D54FF42040A262306003E0421E002873
:1026F8003BD01046A2695106F8D5234A6168DFF835
:1027080090E0306042EA0342174301EA0E021743A1
:102718006760BBB1013BDBB201332B444FF420416E
:10272800A269316052074FF4204005D4421EE0B13F
:102738001046A2695207F9D5626A306005F8012B84
:102748009D42EDD14FF42040306002E0431E60B15D
:102758001846A3699B06F9D520233060E361012060
:10276800F0BD411E08B10846A4E7084A13880133A2
:102778009BB24FF0FF3113803160F0BD2046F0BDB1
:1027880050620020345D002000240002385D0020E3
:10279800009800FCF0B50D460178012983B0044685
:1027A800164618D0022902D0002003B0F0BD806878
:1027B8001F4603F0BBFD45F080016068FFF7BCF9D8
:1027C8003B46324600216068FFF7D3F9A06803F062
:1027D800B3FD0120E9E790F90400421CE4D0022887
:1027E800E2DC617900962A46FFF754FFDDE72DE920
:1027F800F04F90F8553089B00646002B40F02785F9
:10280800A84B0293029B1B7D002B00F0228170696C
:10281800038823F040031B041B0C038003889BB22E
:1028280023F0380343F03803038003889BB243F056
:1028380040030380B36996F84E1013B11A689B8859
:10284800138540F2E93302E0002B00F09C850289F1
:10285800013B12F0020F9BB2F6D01A23037340F229
:10286800E93302E0002B00F08E850289013B12F06B
:10287800010F9BB2F6D0037B706940F2E93302E0A6
:10288800002B00F084850289013B12F0020F9BB2F5
:10289800F6D0017340F2E93302E0002B00F07785AF
:1028A8000289013B12F0010F9BB2F6D0037BB3699A
:1028B80013B11A689B88936102F094FE044602F0F3
:1028C80091FE8442FBD07069038823F040031B0407
:1028D8001B0C0380038823F038031B041B0C0380A4
:1028E80003889BB243F040030380337C012B00F044
:1028F8009980022B40F0A580B36913B11A689B88B0
:10290800138540F2E93302E0002B00F04885028984
:10291800013B12F0020F9BB2F6D0C323037340F2BF
:10292800E93302E0002B00F03A850289013B12F0FE
:10293800010F9BB2F6D0037B70690627838906AD29
:102948004FF47A734FF6FF714FF0FF0E04E0013B2E
:102958009BB28B4200F01F8502899407F7D580F857
:102968000CE04FF47A7303E0A3B28B4200F01385B6
:102978000289D20703F1FF34F6D5027BD2B20DB13A
:102988002A700135013FE7D1B36913B11A689B88F2
:1029980093619DF81A509DF81B309DF818409DF8DA
:1029A80019109DF81C009DF81D2043EA05231BB251
:1029B80073875BB241EA042142EA0022013331877E
:1029C800B28743D196F9383001333FD10A263220F5
:1029D80025F0D0FF4FF4FA7502F004FE044602F029
:1029E80001FE001BB0F57A7FF9D3013DF4D1072031
:1029F80025F030FE4FF47A7502F0F4FD044602F03B
:102A0800F1FD001BB0F57A7FF9D3013DF4D1013E09
:102A1800DDD12549254B2648264A0860DA6009B0E9
:102A2800BDE8F08F96F91400431C0AD0022808DC90
:102A380006AB717D009343220623FFF72BFE002887
:102A4800A7D1B6F93A305BB20133BBD009B0BDE8C3
:102A5800F08F7069038823F040031B041B0C03806C
:102A680003889BB223F0380343F0380303800388BC
:102A78009BB243F040030380B36913B11A689B8883
:102A8800138540F2E93302E0002B00F09B840289B1
:102A9800013B12F0020F9BB2F6D06B23037340F296
:102AA800E9330CE0C8220020FC9F002000ED00E084
:102AB800EFBEADDE0400FA05002B00F08384028926
:102AC800013B12F0010F9BB2F6D0037B706940F214
:102AD800E93302E0002B00F079840289013B12F00F
:102AE800020F9BB2F6D08023037340F2E93302E071
:102AF800002B00F06B840289013B12F0010F9BB29E
:102B0800F6D0037BB36913B11A689B889361962347
:102B1800A94CAA4DDFF8ACA2A948DFF8ACC20396CD
:102B28004FF010084FF47A779946DAF80430C3F377
:102B38000803002B40F06E83EFF31183002B40F065
:102B480069832368816800BF22689342F9D12A68A3
:102B580007FB02FEAEEB010EBEFBF2FE07FB03EE27
:102B68000126DAF80430C3F30803002B40F017837A
:102B7800EFF31183002B40F012832368816800BFB4
:102B880022689342F9D1D5F800B007FB0BF2521A2C
:102B9800B2FBFBF207FB0323A3EB0E03B3F57A7F2B
:102BA800DFD3B9F10109C0D1039EB36913B11A6823
:102BB8009B881385706940F2E93302E0002B00F02E
:102BC800FB830289013B12F0020F9BB2F6D0682307
:102BD800037340F2E93302E0002B00F0ED83028931
:102BE800013B12F0010F9BB2F6D0037B706940F2F3
:102BF800E93302E0002B00F0E2830289013B12F086
:102C0800020F9BB2F6D00323037340F2E93302E0CC
:102C1800002B00F0D4830289013B12F0010F9BB214
:102C2800F6D0037BB36913B11A689B889361962326
:102C3800DFF890A16248DFF890C103964FF01008C2
:102C48004FF47A779946DAF80430C3F30803002B77
:102C580040F0C382EFF31183002B40F0BE8223685B
:102C6800816800BF22689342F9D12A6807FB02FEF7
:102C7800AEEB010EBEFBF2FE07FB03EE0126DAF80F
:102C88000430C3F30803002B40F06B82EFF3118389
:102C9800002B40F066822368816800BF2268934257
:102CA800F9D1D5F800B007FB0BF2521AB2FBFBF2D0
:102CB80007FB0323A3EB0E03B3F57A7FDFD3B9F148
:102CC8000109C0D1039EB36913B11A689B881385A3
:102CD800706940F2E93302E0002B00F07B8302893F
:102CE800013B12F0020F9BB2F6D06B23037340F244
:102CF800E93302E0002B00F06D830289013B12F0FA
:102D0800010F9BB2F6D0037B706940F2E93302E011
:102D1800002B00F062830289013B12F0020F9BB284
:102D2800F6D00323037340F2E93302E0002B00F0EE
:102D380054830289013B12F0010F9BB2F6D0037B4A
:102D4800B36913B11A689B8893610F2002F096FC4F
:102D5800B36913B11A689B881385706940F2E93327
:102D680002E0002B00F03C830289013B12F0020FC5
:102D78009BB2F6D06A23037340F2E93302E0002BDA
:102D880000F02E830289013B12F0010F9BB2F6D0AE
:102D9800037B706940F2E93302E0002B00F02383E3
:102DA8000289013B12F0020F9BB2F6D01023037385
:102DB80040F2E9330DE000BFB0620020B4620020A9
:102DC80010E000E000ED00E0AC620020002B00F015
:102DD8000A830289013B12F0010F9BB2F6D0037BF4
:102DE800B36913B11A689B8893610F2002F046FCFF
:102DF800B36913B11A689B881385706940F2E93387
:102E080002E0002B00F0F2820289013B12F0020F6F
:102E18009BB2F6D06C23037340F2E93302E0002B37
:102E280000F0E4820289013B12F0010F9BB2F6D058
:102E3800037B706940F2E93302E0002B00F0D9828D
:102E48000289013B12F0020F9BB2F6D000230373F4
:102E580040F2E93302E0002B00F0CB820289013B0B
:102E680012F0010F9BB2F6D0037BB36913B11A6855
:102E78009B8893610F2002F001FCB36996F850100B
:102E880013B11A689B881385706940F2E93302E030
:102E9800002B00F0B1820289013B12F0020F9BB2B5
:102EA800F6D01923037340F2E93302E0002B00F057
:102EB800A3820289013B12F0010F9BB2F6D0037B7B
:102EC800706940F2E93302E0002B00F09882028931
:102ED800013B12F0020F9BB2F6D0017340F2E933C6
:102EE80002E0002B00F08B820289013B12F0010FF7
:102EF8009BB2F6D0037BB36913B11A689B889361C0
:102F08000F2002F0BBFBB36913B11A689B881385C5
:102F1800706940F2E93302E0002B00F07382028905
:102F2800013B12F0020F9BB2F6D01B23037340F251
:102F3800E93302E0002B00F065820289013B12F0C0
:102F4800010F9BB2F6D0037B706940F2E93302E0CF
:102F5800002B00F05A820289013B12F0020F9BB24B
:102F6800F6D01823037340F2E93302E0002B00F097
:102F78004C820289013B12F0010F9BB2F6D0037B11
:102F8800B36913B11A689B8893610F2002F076FB2E
:102F9800B36913B11A689B881385706940F2E933E5
:102FA80002E0002B00F034820289013B12F0020F8C
:102FB8009BB2F6D01C23037340F2E93302E0002BE6
:102FC80000F026820289013B12F0010F9BB2F6D075
:102FD800037B706940F2E93302E0002B00F01B82AA
:102FE8000289013B12F0020F9BB2F6D01023037343
:102FF80040F2E93302E0002B00F00D820289013B28
:1030080012F0010F9BB2F6D0037BB36913B11A68B3
:103018009B8893610F2002F031FBB36913B11A68E2
:103028009B881385706940F2E93302E0002B00F0B9
:10303800F5810289013B12F0020F9BB2F6D03723CB
:10304800037340F2E93302E0002B00F0E7810289C4
:10305800013B12F0010F9BB2F6D0037B706940F27E
:10306800E93302E0002B00F0DC810289013B12F019
:10307800020F9BB2F6D01023037340F2E93302E04B
:10308800002B00F0CE810289013B12F0010F9BB2A8
:10309800F6D0037BB36913B11A689B8893610F203C
:1030A80002F0ECFAB36913B11A689B88138570694A
:1030B80040F2E93302E0002B00F0B6810289013BBF
:1030C80012F0020F9BB2F6D03823037340F2E933B3
:1030D80002E0002B00F0A8810289013B12F0010FE9
:1030E8009BB2F6D0037B706940F2E93302E0002B13
:1030F80000F09D810289013B12F0020F9BB2F6D0CD
:103108000123037340F2E93302E0002B00F08F81C2
:103118000289013B12F0010F9BB2F6D0037BB36921
:1031280013B11A689B8893610F2002F0A7FA72699D
:10313800138823F040031B041B0C1380138823F00F
:1031480038031B041B0C138013889BB243F0400305
:103158001380012002F092FA029A01231375FFF7F7
:1031680056BBEFF3118188F31288D0F808B00368D2
:10317800DB0344BFCCF80060D0F808B02368DCF863
:103188000020C9B281F3118829681A4407FB01F3AA
:10319800A3EB0B03B3FBF1F307FB02338AE5EFF371
:1031A800118188F31288D0F808B00368DB0344BFA4
:1031B800CCF80060D0F808B02368DCF80020C9B269
:1031C80081F3118829681A4407FB01F3A3EB0B0369
:1031D800B3FBF1F307FB0233DEE4EFF3118288F36C
:1031E800128881680368DE0303D50123CCF8003018
:1031F80081682368DCF80060D2B282F311882A68FB
:1032080006EB030E07FB02F35B1AB3FBF2F307FBB3
:103218000E3E33E5EFF3118288F312888168036864
:10322800DE0303D50123CCF8003081682368DCF87D
:103238000060D2B282F311882A6806EB030E07FBFE
:1032480002F35B1AB3FBF2F307FB0E3E88E41D0999
:10325800013D052D03F00F0300F2A880864A32F8DD
:10326800150040FA03F2D40740F1A080012404FAC3
:1032780003F3013B184030F0BBFA804BDFF81882AB
:103288005F5D074418EBC70500F0908020220023FB
:10329800AA71EB7158F83700794A00F138439B0A54
:1032A800D25C02F01F035209022A04FA03F300F069
:1032B800DD80032A00F0D580A24200F0CD80AB88E3
:1032C800069306A9002407942BF0A4FCAB886D4A4A
:1032D800F260B3FA83F2C2F11F02511C63D0D1B27B
:1032E80001F0FC0303F1804303F5803301F003018F
:1032F800D3F808E088004FF00F0C58F83710DFF8C3
:103308009C810CFA00F72EEA070E06F10C0748F824
:103318002270C3F808E0D3F808C05B4FDFF880E1FB
:10332800C1F38721814041EA0C01B8184FF0010828
:10333800996008FA02F3554990F80891029106A895
:10334800CEF80030082306928DF81D308DF81E80C7
:103358008DF81C4023F056FD029901EB09031A7AF7
:10336800F02A67DCAB88B3FA83F3C3F11F035F1C51
:103378003FF448AA012202FA03F345490A681343B5
:103388000B60FFF73FBAFDF72FFCFFF775BAFDF7A3
:103398002BFCFFF78CBAFDF727FCFFF7F5BAFDF712
:1033A80023FCFFF7C9BA394A0292DCE7354B374AA2
:1033B800F36002920123E0E7FDF716FC16E4FDF73F
:1033C80013FC2FE4FDF710FCFFF780BBFDF70CFCA6
:1033D800FFF798BBFDF708FC96E4FDF705FCAFE4A2
:1033E800FDF702FCD5E4FDF7FFFBF9E4FDF7FCFB74
:1033F8001FE5FDF7F9FB38E5FDF7F6FB60E5FDF79E
:10340800F3FB78E5FDF7F0FB9EE5FDF7EDFBB7E58F
:10341800FDF7EAFBDDE5FDF7E7FBF6E5FDF7E4FB85
:103428001CE6FDF7E1FB35E6FDF7DEFB5BE6FDF7A5
:10343800DBFB74E64F44F02197F818218DF814202F
:1034480005A803228DF816408DF8178019728DF89B
:1034580015202BF0A9FB85E70E4A51690B435361F0
:103468002DE70C4AD1690B43D36128E7094A9169D2
:103478000B43936123E700BF787303088473030841
:10348800F4730308A907000800510308C8220020A4
:103498000004014000100240545300201C23002067
:1034A80014040140F0B5037A012B85B0044663D0BB
:1034B800022B67D1036913B11A689B881385E068EA
:1034C80040F2E93301E0002B6CD00289013B12F095
:1034D800020F9BB2F7D0BB23037340F2E93301E03C
:1034E800002B5FD00289013B12F0010F9BB2F7D08D
:1034F800037BE0684FF0060E838902AE4FF47A73BF
:103508004FF6FF71FF2703E0013B9BB28B423CD093
:1035180002899507F8D507734FF47A7302E0ABB2C6
:103528008B4232D00289D20703F1FF35F7D5027BEF
:10353800D2B20EB132700136BEF1010EE8D1236964
:1035480013B11A689B8893619DF80C009DF8086078
:103558009DF809109DF80A509DF80B209DF80D3034
:1035680041EA062143EA002342EA05220120E182DA
:103578002283638305B0F0BD90F90C00431C01D091
:10358800022805DD002005B0F0BDFDF72DFBD6E7CC
:1035980002AB617B00933B220623FFF77BF80028F0
:1035A800D2D1EFE7FDF720FBA3E71749174B184ADD
:1035B800184810B4D1F8884044F47004C1F8884021
:1035C8001C6844F001041C605C6822405A601A6858
:1035D80022F0847222F480321A601A6822F480225F
:1035E8001A605A6822F4FE025A60DA6A22F00F0260
:1035F800DA621A6B002410404FF0006218639C6076
:103608008A605DF8044B704700ED00E0001002404E
:103618000CC07FF8CCFC00FF38B50B4C23688BB18D
:103628005A68821A002A054604DA0CE05A68AA1A6F
:10363800002A07DB9A68226018461A6890472368B0
:10364800002BF3D138BD38BD886B00200B4B00220E
:1036580010B4027203F18C04012102E0072A09DC8C
:103668009979890702D51979815401329C4203F16D
:103678001403F3D15DF8044B704700BFFC730308D3
:1036880024230370704700BF0123102111224170C9
:103698004271037203700371704700BF2DE9F04156
:1036A8000B78057BDB43DFB200F1130200F11D0349
:1036B80002F8015F9342FBD1DFF890E000F12701A7
:1036C800002203F8012F9942FBD11421052400267A
:1036D80047FA04F303F00103002B1E4414BF4FF014
:1036E80019084FF00A0814F0010FF6B214BFAC46DF
:1036F8004FF0000C0023CA1810FA82F20133434538
:1037080082F814C0F7D15A1E92B20132013C8B18CC
:10371800621C9BB201D01946DAE716F0010F14BFFC
:1037280019240A240022991810FA81F10132A242C0
:103738000D75F8D113449BB25A1C0344002192B270
:103748001975AEF800200261BDE8F0811023002051
:103758002DE9F04FDFF890A0BAF802300B3383B0B0
:103768001FFA83F901F1060B4FF001084FF0000C26
:10377800002711F801EB3E464C460122A4F10B0349
:103788009BB2019105E001339BB2017B29759C42F4
:1037980008D0C518002AF6D1C51801339BB29C423F
:1037A8002A75F6D103190136092F019983F814C037
:1037B800F6B20CD0092E15D008FA07F313EA0E0F4B
:1037C80014BF012200220C34A4B20137D6E709F154
:1037D800780959451FFA89F9CAD1AAF802C003B075
:1037E800BDE8F08F0022EEE7102300202DE9F04716
:1037F800DFF85C80B8F8043004331FFA83FC01F169
:1038080009094FF0010E11F8017B64460026231FB9
:103818000EFA06F29BB23A40C2B1B0F80CA0C51835
:1038280001339BB29C4285F814A0F5D101360434CB
:10383800082EA4B2EBD10CF1200C49451FFA8CFCE0
:10384800E1D10023A8F80430BDE8F0879246E6E706
:103858001023002010B50168047B0A680223A340E6
:103868001A420AD0054A406800241470026822F0FF
:1038780001021204120C02604B6010BDBB2700202D
:10388800436A8269D154436A0169826B01338B426E
:1038980028BF00234362002A2FD0EFF31181502361
:1038A80083F31288836B1A68D2072CD470B45E68CD
:1038B8006EB9456A826A954217D084691444DC60FF
:1038C8000ED9AA1A5A608562002280F854201A6814
:1038D80042F00102C9B21A6081F3118870BC7047C6
:1038E8000469A21A5A608662EEE7012380F8543010
:1038F800C9B281F3118870BC7047026D136843F038
:10390800800313607047C9B281F31188704700BF04
:10391800426B10B462B1436CC2684469D11A013B6E
:10392800615C5DF8044B08BF13464364C8B2704736
:10393800016A4369C4685B5C0131A14228BF114632
:1039480001625DF8044BD8B2704700BF836B13B1B6
:1039580090F854007047836A406A181AB0FA80F0E9
:1039680040097047416A836A99420AD3CB1A816B2E
:10397800026961B14968501E0B4483420AD2C01AD9
:10398800704702691144CB1A816B0029F2D1501E8D
:10399800C01A704700207047436B43B1426C5B68A4
:1039A80093422FBF981AC0689B1AC0187047C26903
:1039B800036A9A422FBFD01AC0688018C01A70478D
:1039C8000A4B30B503F1140493F900205D78072AF7
:1039D800C8BF143A811804330D7313F8025C855478
:1039E80013F8012C0A76A342EED130BD2052030809
:1039F80003682DE9F041DF691FB13B46BDE8F0419E
:103A08001847002A164611DD04460D460E4400E00C
:103A180023689B68204698470028F9D0236815F842
:103A2800011B1B6820469847AE42F1D1BDE8F081E2
:103A380000232322027043708370C370704700BF55
:103A48002DE9F0470569C3681D4028D00F46064692
:103A58004FF000484FF00009B5FA85F328FA03F251
:103A6800D2431B3B32611540042B16D8DFE803F024
:103A78003129211903007B6A002B32D003F1FF3A68
:103A88001FFA8AFAC7F824903C6A34B123682046A2
:103A9800514698476468002CF8D1002DDCD1BDE868
:103AA800F0873868716B036889B29847002DD3D1C5
:103AB800F5E77868B16B036889B29847002DCBD1D8
:103AC800EDE7B868F16B036889B29847002DC3D158
:103AD800E5E7F868316C036889B29847002DBBD1D7
:103AE800DDE7F36A1FFA83FACEE700BF30B5044674
:103AF800006D61710368A26823F00103036087B059
:103B0800A379009213F004023DD04FF4805213F0D1
:103B18000203019244D102934FF48063002203937D
:103B280011F00103059237D1049308238D076946E4
:103B380048BF04931CF070FB6079236DA17900F0F5
:103B48000202002A15BF4FF440324FF480324FF47E
:103B58000034002410F0010F586808BF2246CC0733
:103B68004CBF024320EA02025A609A6809074CBF18
:103B780042F0080222F008029A601A6842F0010234
:103B88001A6007B030BD13F0020301920BD04FF456
:103B9800005513460295C1E7042304930C23C5E797
:103BA8004FF40053B7E70293B8E700BF10B50446D7
:103BB800006DA160036823F001030360A37986B058
:103BC80013F00402009141D04FF4805213F0020325
:103BD800019244D102934FF4806362790393D10731
:103BE8004FF000030493059345BF0423049308236F
:103BF8000C236946920748BF04931CF00DFB6079BB
:103C0800236DA17900F00202002A15BF4FF440325B
:103C18004FF480324FF40034002410F0010F58683C
:103C280008BF2246CC074CBF024320EA02025A6072
:103C38009A6809074CBF42F0080222F008029A600D
:103C48001A6842F001021A6006B010BD13F00203B0
:103C5800019207D04FF4005113460291BDE74FF48B
:103C68000053B7E70293B8E7022828BF022010B430
:103C7800084C094B207000EB8002C0EBC2020749D8
:103C88005DF8044B013003EB4203C0B20B602AF02D
:103C9800AFBC00BF1C6200202435002084680020CF
:103CA80008B529F0B1FBFDF7DBF8BDE8084029F0BD
:103CB80093BB00BF2DE9F04F013085B0C3B2039329
:103CC8008E4D8F4F8F4C904E0A2302933220DFF88F
:103CD800409224F04FFE4FF4FA7A4FF0100C4FF454
:103CE8007A70D9F80430C3F30803002B40F0C88079
:103CF800EFF31183002B40F0C3802968A26800BF4E
:103D08002B689942F9D1D7F800E000FB0EF39B1A13
:103D1800B3FBFEF300FB01314FF0010E0191D9F81E
:103D28000430C3F30803002B40F08E80EFF31183B7
:103D3800002B40F089802B68A16800BF2A68934255
:103D4800F9D1D7F800B000FB0BF2521AB2FBFBF224
:103D580000FB0323019A9B1AB3F57A7FDFD3BAF1EC
:103D6800010ABED1039B002B40F0C4804FF47A7A3D
:103D7800DFF89C9150464FF0100CD9F80430C3F38B
:103D88000803002B40F09980EFF31183002B40F0DB
:103D980094802968A26800BF2B689942F9D1D7F8A6
:103DA80000E000FB0EF39B1AB3FBFEF300FB0131AE
:103DB8004FF0010E0191D9F80430C3F308033BBB5F
:103DC800EFF3118323BB2B68A16800BF2A689342D5
:103DD800F9D1D7F800B000FB0BF2521AB2FBFBF294
:103DE80000FB0323019A9B1AB3F57A7FE3D3BAF158
:103DF800010AC2D1029B013B02937FF467AF43499A
:103E0800434B4448444A0860DA6005B0BDE8F08F87
:103E1800EFF311888CF31288A1682368DB0344BF91
:103E2800C6F800E0A1682B6832685FFA88F888F362
:103E38001188D7F800801A4400FB08F35B1AB3FB1B
:103E4800F8F300FB0233CDE7EFF311888CF3128807
:103E5800A1682368DB0344BFC6F800E0A1682B68AB
:103E680032685FFA88F888F31188D7F800801A4416
:103E780000FB08F35B1AB3FBF8F300FB023369E7B6
:103E8800EFF311828CF31288D4F808E02368D90381
:103E980003D501233360D4F808E02B683168D2B227
:103EA80082F311883A68194400FB02F3A3EB0E036E
:103EB800B3FBF2F300FB01312EE7EFF311828CF331
:103EC8001288D4F808E02368D90303D501233360A6
:103ED800D4F808E02B683168D2B282F311883A68C6
:103EE800194400FB02F3A3EB0E03B3FBF2F300FB50
:103EF80001315DE7184624F0ADFB37E7B0620020DA
:103F0800B462002010E000E0AC620020FC9F0020BA
:103F180000ED00E0EFBEADDE0400FA0538B5434B16
:103F28005A899989914224BF00225A81198ADA89CB
:103F3800914224BF0022DA81DA788AB3072A2FD087
:103F48003B493C4D91F85300012400210A282C706C
:103F58009C70D9713DD00C2865D0DFED377A8ABBCB
:103F6800364C9FED370AA278002918BFF0EE407A48
:103F7800062A04D8334901EB820191ED050A21791B
:103F880059B3013A032A4DD8F7EE007A87EE800A32
:103F980030F086F82388984228BF1846208038BD1C
:103FA800D97921B198780428B8BF0420987020489E
:103FB80090F853000A280CD00C28CED1DFED227AD5
:103FC800002ACDD0072ACBD00A282CD1DFED1F7AC2
:103FD800C6E70A20DFED1E7AC1E79B78154A07EE8F
:103FE800103A1178B8EEC77A27EE277A07EE901ABA
:103FF800F8EEE77A67EE877AB4EEE70AF1EE10FAA0
:1040080010DDC0EE077AFDEEE77A17EE903A102B36
:10401800A8BF1023012BB8BF0123DBB28B4238BFE6
:104028000B46137038BDDFED0B7A99E784540020F6
:1040380098540020844600206F120339205900202C
:104048006F120338205203080AD7A3390F506E3A6B
:104058005304E9386F12833A2DE9F047A64FA74E6B
:1040680029F0D2F9BE421ED2DFF80C83DFF80C9398
:104078004446258862197DB14A450DD2052D0BD9D4
:1040880033886188C3F30B03994200F0DA80144641
:1040980025886219002DEFD1716830461436FCF777
:1040A8006BFEBE42E4D3964A1378A3F117010229A6
:1040B8000FD9944911F83300002840F0EE80D80059
:1040C8000144497829B1904911F83330002B00F0A8
:1040D8000C818E4B5A78022A40F2D98000228C49F2
:1040E8005A701A788B48022A016000F2CC8002EBE1
:1040F8008201894BC2EBC10203EB4203998C5A8CB3
:10410800864C9142236001D300225A84844B9A78CA
:10411800042A00F0E18032B91A88B2F5F07F84BF32
:104128004FF4F0721A807F4DFFF7F8FE2B687E4A35
:104138001A40002A00F0DC80D80700F1C880590432
:1041480000F1C0801A0700F1B8809B0400F1AE802E
:1041580023F0B8FC10B9754829F0A8FC8020FCF7BA
:1041680041FE4FF40070FCF73DFE4FF40030FCF7C1
:1041780039FE4FF00070FCF735FE4FF08060FCF719
:1041880031FE1EF06DF900213022694830F045FFFC
:1041980020681DF067F8674B276803F1500102E0BB
:1041A800043399426DD01A78002AF9D19C78D878CE
:1041B8008442F5D26049614B0D79614961480A70C2
:1041C800614E624C0460C822642111FB0521002263
:1041D80059609A60DA601A615A619A61DA6183F803
:1041E800202083F82120376018F060FA584B9FEDA3
:1041F800595A1B88584A9FED596A5079584906EE12
:10420800903AF8EEE66A1388C5EE265A07EE103A99
:1042180053881279C1ED005A07EE903AB8EEC77A82
:10422800504BF8EEE77A18725A7227EE067A67EE64
:10423800867ABDE8F04783ED017AC3ED007A29F06C
:10424800CBB863799B077FF422AF716894F804A018
:104258003046FCF791FD3388BAEB133F04D014368F
:10426800BE42FFF405AF1EE773887068AA1FC3F348
:104278000B039A4204F10601A8BF1A462FF03AFD33
:10428800EDE7012296E700221A70234B36E7204912
:1042980002EB420201EB820123E7D8000C186468A4
:1042A800002C7FF40DAF1724147009E72E48FCF793
:1042B80099FD4020FCF796FD4AE72C48FCF792FD53
:1042C8002B6842E72A48FCF78DFD2B683AE7294816
:1042D800FCF788FD2B6832E79A8AB2F57A7FBFF43B
:1042E80022AF4FF47A729A821DE718231370F0E612
:1042F80043F001032B601FE734B9030898B403089F
:1043080054440020B4780308247103081C62002078
:10431800303600208868002024350020846800207A
:1043280020590020C0360020096000022C5E0020C1
:1043380048240020B072002094490020C04B00207F
:10434800EF2000208C2400207C24002096460020AA
:1043580088260020C0C9FB48BC24002017B7D138E4
:104368008C260020944700200940000201600002CA
:10437800092000020860000202F003080000040897
:1043880008B529F041F8FCF76BFD29F025F8FFF78F
:1043980063FE0120BDE808402AF02AB938B50C4C64
:1043A8000C4DAC4206D2616820461434FCF7E4FC9C
:1043B800AC42F8D3084A094B094C14600022094959
:1043C8001A705A7008480860BDE8384020F08CBD63
:1043D80098B4030834B90308846800201C620020DC
:1043E80024350020886800203036002008B5FFF703
:1043F800D5FF29F009F8FCF733FDBDE8084028F09F
:10440800EBBF054B10B59A68044C2178501C09B9CC
:104418009A6010BD0246F8E710230020BB27002051
:10442800F0B50C292BD8DFE801F06F2A2A2A4C2A8C
:104438002A2A2B2A2A2A0700046AB2F80CE097884D
:104448001668674D24F480540462036A4468C1699D
:1044580023F4005343EA0E3321F4E641A84243EA29
:10446800073341EA062100F0B58005F50065A8424A
:1044780000F0B08092684460C16102640362F0BDDC
:10448800046A96899588D2F800E0554F24F4807420
:104498000462036A4468C16923F4007343EA06238B
:1044A80021F07301B84243EA052341EA0E017ED0A8
:1044B8004C4DA8427BD092684460C161C2630362DC
:1044C800F0BD046A96899588D2F800E0444F24F03C
:1044D80010040462036A4468816923F0200321F010
:1044E800807143EA061321F4E641B84243EA051312
:1044F80041EA0E2148D03B4DA84245D0926844601D
:10450800816182630362F0BD046A9389B2F804E0B2
:104518001768334E24F001040462056A446881690F
:1045280043EA0E0321F4803125F002059BB221F005
:104538007301B04243EA050341EA070114D0294D4B
:10454800A84211D005F54065A8420DD005F5806553
:10455800A84209D005F58065A84205D09268446054
:10456800816142630362F0BDD689158A578A23F0B8
:10457800080333433D43D68824F4407423F00403EE
:10458800ADB233432C43E9E7D589178AD68823F09F
:10459800800343EA051324F44064558A23F040035A
:1045A80044EA870443EA061344EA8504A6E7D58962
:1045B800178AD68823F4006343EA052324F4405479
:1045C800558A23F4806344EA071443EA062344EA3D
:1045D800051470E7158A24F4804444EA851449E7F1
:1045E800002C0140003401402DE9F04FF022002159
:1045F80083B07948794CDFF80892794D794E7A4F33
:10460800DFF8008230F009FD78487949DFF8F8E1F1
:10461800DFF8F8C100221359834200F0C280B3F1D9
:10462800804F00F0CA80AB4200F0C980B34200F06E
:10463800C880BB4200F0C780734500F0C680634560
:1046480000F0C580434500F0C480DFF8C4A153459D
:104658007AD00AF5806A534508BF092375D0143209
:10466800A02AD8D15D4C634D634E614F04F1A00878
:1046780002E01434A04564D0A379002BF9D0237943
:104688004FEA131909F1FF39B9F1050F03F00F03C8
:10469800EFD835F8190040FA03F2D207E9D54FF000
:1046A800010A0AFA03F3013B18402FF0A1F816F8A3
:1046B80009305249184411EBC002DAD051F83000E1
:1046C800DFF850E1217A00F138439B0A1EF80330E5
:1046D80003F01F0E5B09022B0AFA0EFA63D0032BB4
:1046E80066D0012B58D093880093B3FA83F3C3F1B3
:1046F8001F039BB2DA0800EB820203F00703D2F82B
:1047080020E09B004FF00F0C0CFA03FC2EEA0C0E75
:10471800C2F820E0D2F820E001FA03F343EA0E03DE
:10472800136269460023022214348DF804208DF8A0
:1047380005308DF806308DF807302AF06BFAA04561
:104748009AD103B0BDE8F08F082309EBC3034FF0FB
:10475800010B93F834A00AF01F034FEA5A1ABAF172
:10476800020F0BFA03F311D0BAF1030F08D0DA45A0
:104778007FF475AFD1F814A043EA0A034B616EE7E2
:10478800D1F81CA043EA0A03CB6168E7D1F818A066
:1047980043EA0A038B6162E77B694AEA03037B61A8
:1047A800A1E70023D1E7BB694AEA0303BB619AE7A3
:1047B800FB694AEA0303FB6195E70123C5E7022386
:1047C800C3E70323C1E70423BFE70523BDE70623A7
:1047D800BBE70723B9E700BF3C5D0020FC73030873
:1047E800000400400008004000100040002C014078
:1047F80000100240787303088473030854530020A0
:1048080020520308004001400014004000340140D9
:1048180000440140F4730308002867D003682DE9B9
:10482800F04F03F138445C4EA40A0125345D04F0CE
:104838001F066409022C05FA06F558D0032C00F06F
:10484800A580012C58D08088B0FA80F4C4F11F04E8
:10485800A4B2E50803EB850504F007042E6AA4005A
:104868000F27A74026EA07062E622E6A01F00307E3
:10487800A2407C1E3243012CC1F3810CC1F3001805
:104888002A62C1F341113CD9C60700F18980850726
:1048980000F19580440700F1A380020700F1B18080
:1048A800C60600F1BF80850600F1CD80440600F100
:1048B800DB80020600F1E980C60500F1F780850576
:1048C80000F10581440500F11381020500F1218101
:1048D800C60400F12F81850400F13D81440400F1F4
:1048E8004B81020400F15981BDE8F08F70472B4CD1
:1048F800A6693543A561A6E7284C66693543656115
:10490800A1E7002422464FF0010E4FF0030904E00E
:104918000132102A04F10204E6D00EFA02F636EA51
:104928000005F5D1D3F808A009FA04F5ED430AEA21
:10493800050AC3F808A0D3F808B00CFA04FA4AEA42
:104948000B0AC3F808A0B3F804A01FFA8AFA2AEAE7
:1049580006069E80B3F804A008FA02F646EA0A069C
:10496800B6B29E801E682E401E60D3F800A007FADB
:1049780004F646EA0A061E60D3F80CA001FA04F60B
:1049880005EA0A0A46EA0A05DD60C1E7034CE6695A
:104998003543E56157E700BFF47303080010024090
:1049A8001A6822F003021A601A683A431A60DA6831
:1049B80022F003020A438507DA607FF56BAF1A68B5
:1049C80022F00C021A601A6842EA87021A60DA6852
:1049D80022F00C0242EA81024407DA607FF55DAFFB
:1049E8001A6822F030021A601A6842EA07121A603E
:1049F800DA6822F0300242EA0112DA6002077FF533
:104A08004FAF1A6822F0C0021A601A6842EA871289
:104A18001A60DA6822F0C00242EA8112C606DA6039
:104A28007FF541AF1A6822F440721A601A6842EAA8
:104A380007221A60DA6822F4407242EA01228506E7
:104A4800DA607FF533AF1A6822F440621A601A6898
:104A580042EA87221A60DA6822F4406242EA812236
:104A68004406DA607FF525AF1A6822F440521A60CE
:104A78001A6842EA07321A60DA6822F4405242EAB7
:104A88000132DA6002067FF517AF1A6822F4404255
:104A98001A601A6842EA87321A60DA6822F44042D9
:104AA80042EA8132C605DA607FF509AF1A6822F456
:104AB80040321A601A6842EA07421A60DA6822F439
:104AC800403242EA01428505DA607FF5FBAE1A689A
:104AD80022F440221A601A6842EA87421A60DA68A9
:104AE80022F4402242EA81424405DA607FF5EDAEC5
:104AF8001A6822F440121A601A6842EA07521A60C9
:104B0800DA6822F4401242EA0152DA6002057FF5BF
:104B1800DFAE1A6822F440021A601A6842EA875225
:104B28001A60DA6822F4400242EA8152C604DA6066
:104B38007FF5D1AE1A6822F040721A601A6842EA0C
:104B480007621A60DA6822F0407242EA016285045C
:104B5800DA607FF5C3AE1A6822F040621A601A68FC
:104B680042EA87621A60DA6822F0406242EA8162A9
:104B78004404DA607FF5B5AE1A6822F040521A6034
:104B88001A6842EA07721A60DA6822F0405242EA6A
:104B98000172DA6002047FF5A7AE1A6822F040427B
:104BA8001A601A6842EA87771F60DA6822F0404282
:104BB80042EA8171D960BDE8F08F00BF03682DE932
:104BC800F04F03F13845644EAD0A0124755D05F0D8
:104BD8001F066D09022D04FA06F400F0A280032DC9
:104BE80000F0A480012D52D08088B0FA80F4C4F17E
:104BF8001F04A4B2E50803EB850504F007042E6A38
:104C0800A4000F27A74026EA07062E622E6A01F0A5
:104C1800030702FA04F47A1E3443012AC1F3810C13
:104C2800C1F300182C62C1F3411135D9C60700F150
:104C38009780850700F1A380440700F1B18002073F
:104C480000F1BF80C60600F1CD80850600F1DB804B
:104C5800440600F1E980020600F1F780C60500F17C
:104C68000581850500F11381440500F121810205C4
:104C780000F12F81C60400F13D81850400F14B81CC
:104C8800440400F15981020455D4BDE8F08F334D36
:104C98006E6934436C61A7E7002422464FF0010E89
:104CA8004FF0030904E00132102A04F10204ECD0A9
:104CB8000EFA02F636EA0005F5D1D3F808A009FA8B
:104CC80004F5ED430AEA050AC3F808A0D3F808B0CA
:104CD8000CFA04FA4AEA0B0AC3F808A0B3F804A0CD
:104CE8001FFA8AFA2AEA06069E80B3F804A008FA90
:104CF80002F646EA0A06B6B29E801E682E401E607C
:104D0800D3F800A007FA04F646EA0A061E60D3F8AC
:104D18000CA001FA04F605EA0A0A46EA0A05DD606B
:104D2800C1E70E4DAE693443AC615DE70B4DEE69EA
:104D38003443EC6158E71A6822F040421A601A6856
:104D480042EA87771F60DA6822F0404242EA8171BE
:104D5800D960BDE8F08F00BFF4730308001002406B
:104D68001A6822F003021A601A683A431A60DA686D
:104D780022F003020A438507DA607FF55DAF1A68FF
:104D880022F00C021A601A6842EA87021A60DA688E
:104D980022F00C0242EA81024407DA607FF54FAF45
:104DA8001A6822F030021A601A6842EA07121A607A
:104DB800DA6822F0300242EA0112DA6002077FF56F
:104DC80041AF1A6822F0C0021A601A6842EA8712D4
:104DD8001A60DA6822F0C00242EA8112C606DA6076
:104DE8007FF533AF1A6822F440721A601A6842EAF3
:104DF80007221A60DA6822F4407242EA0122850624
:104E0800DA607FF525AF1A6822F440621A601A68E2
:104E180042EA87221A60DA6822F4406242EA812272
:104E28004406DA607FF517AF1A6822F440521A6018
:104E38001A6842EA07321A60DA6822F4405242EAF3
:104E48000132DA6002067FF509AF1A6822F440429F
:104E58001A601A6842EA87321A60DA6822F4404215
:104E680042EA8132C605DA607FF5FBAE1A6822F4A1
:104E780040321A601A6842EA07421A60DA6822F475
:104E8800403242EA01428505DA607FF5EDAE1A68E4
:104E980022F440221A601A6842EA87421A60DA68E5
:104EA80022F4402242EA81424405DA607FF5DFAE0F
:104EB8001A6822F440121A601A6842EA07521A6005
:104EC800DA6822F4401242EA0152DA6002057FF5FC
:104ED800D1AE1A6822F440021A601A6842EA875270
:104EE8001A60DA6822F4400242EA8152C604DA60A3
:104EF8007FF5C3AE1A6822F040721A601A6842EA57
:104F080007621A60DA6822F0407242EA0162850498
:104F1800DA607FF5B5AE1A6822F040621A601A6846
:104F280042EA87621A60DA6822F0406242EA8162E5
:104F38004404DA607FF5A7AE1A6822F040521A607E
:104F48001A6842EA07721A60DA6822F0405242EAA6
:104F58000172DA6097E600BF10B50409013C052C20
:104F680017D80D4B33F8142000F00F0042FA00F365
:104F780013F001030DD0012303FA00F001381040AB
:104F88002EF036FC054A064B125D104403EBC000B8
:104F980010BD002010BD00BF787303088473030898
:104FA8005453002001490248FEF74ABD045E002020
:104FB8000040014001490248FEF742BDDC5D002087
:104FC8000034014001490248FEF73ABDDC5D00208B
:104FD8000034014001490248FEF732BDB45D0020AB
:104FE8000008004001490248FEF72ABD8C5D0020F8
:104FF8000004004002494FF08040FEF721BD00BF89
:10500800645D002001490248FEF71ABD3C5D00209E
:10501800002C014001490248FEF712BD3C5D00200A
:10502800002C01402DE9F04104684E4DA30AAB4223
:105038007AD00AD94C4DAB425FD00335AB4277D01A
:10504800053DAB425DD0BDE8F081B3F5801F67D068
:10505800013DAB4259D14FF0700E022647794FEA15
:10506800970C002968D0B000634685190227D4F848
:105078000C809F400CEB4503BFB23C4D03F1040C80
:1050880047EA080745F8231045F82C20E760EFF3B6
:105098001181502282F31288821905EBC20213692A
:1050A800002B34D013620433821905EBC20257690E
:1050B80017B11F6053690433821905EBC20297695F
:1050C80017B11F6093690433821905EBC202D769CF
:1050D80017B11F60D36904330027CAB21F6082F377
:1050E8001188304405EBC000036A9BB9E3684FF6AA
:1050F800FE721340E360BDE8F0814FF0C00E042655
:10510800ACE74FF0200E0026A8E7BDE8F08105EBDC
:105118000E03C9E7E36843F00103E360BDE8F081EB
:105128004FF0480E012699E74FF0980E032695E7B1
:105138004FF0E80E052691E7BF08022306FA03F0B0
:10514800BB40DB43E768094D9BB23B4087190CEB3A
:10515800470CE3600CF1040345F82C1045F82320B4
:1051680095E700BF020010004D0010003C5D0020D4
:1051780030B503685C4D18885C4CB4FBF2F2013919
:10518800013AAB4294B283B089B282B266D0584831
:10519800834263D0B3F1804F60D0A0F5983083424A
:1051A8005CD000F58060834258D0524883425BD07F
:1051B80000F5806083427DD022F4407200F58C3087
:1051C80092B283421A80D9621C850ED0484A934213
:1051D8000BD002F54062934207D002F580629342F9
:1051E80003D002F58062934201D100221A8601227F
:1051F8005A611A883C4992B242F001028B421A80E5
:1052080062D0B3F1804F61D03B4A934260D002F53F
:10521800806293425ED002F5006293425CD002F550
:10522800806293425AD002F59032934258D002F5E8
:105238004062934256D002F5806293421ED002F536
:105248008062934208BF092219D002A84FF00123B7
:1052580040F8043D29F0A8FC03B030BD254822F0F1
:105268007002834292B2A3D101201A80D9621C85B0
:1052780058611A8892B202431A80C5E708221F4B68
:1052880003EBC20301A893F835408DF804400123CD
:1052980000228DF805308DF807308DF8062029F0AA
:1052A80083FC1B2CD8D1164B019301A829F07CFC58
:1052B80003B030BD01201A80D9621C8558611A8854
:1052C80092B202431A809CE70022D8E70122D6E76F
:1052D8000222D4E70322D2E70422D0E70522CEE750
:1052E8000622CCE70722CAE7002C014000A24A04A4
:1052F8000034014000100040000400402052030820
:1053080019010001204B98422DD0B0F1804F2CD0CC
:10531800A3F5943398422AD003F58063984228D0A5
:1053280003F50063984226D003F58063984224D0A1
:1053380003F59033984222D003F54063984220D079
:1053480003F58063984207D003F58063984208BF4D
:10535800092202D00020704708220C4B03EBC2033D
:1053680093F8340070470022F7E70122F5E702229C
:10537800F3E70322F1E70422EFE70522EDE706222F
:10538800EBE70722E9E700BF002C014020520308A1
:105398002DE9F04F013085B0C3B203930B4602915B
:1053A8008B4C8C4E002B00F09A8032208A4D8B4F0C
:1053B800DFF82C9223F0DEFA4FF4FA7A4FF0100C53
:1053C8004FF47A70D9F80430C3F30803002B40F087
:1053D800DE80EFF31183002B40F0D9802968A268A2
:1053E80000BF2B689942F9D1D7F800E000FB0EF313
:1053F8009B1AB3FBFEF300FB01314FF0010E019144
:10540800D9F80430C3F30803002B40F08780EFF38A
:105418001183002B40F082802B68A16800BF2A68A6
:105428009342F9D1D7F800B000FB0BF2521AB2FB45
:10543800FBF200FB0323019A9B1AB3F57A7FDFD3B3
:10544800BAF1010ABED1039B002B40F0BD804FF496
:105458007A7ADFF88C9150464FF0100CD9F8043066
:10546800C3F30803002B75D1EFF31183002B71D11F
:105478002968A26800BF2B689942F9D1D7F800E0E3
:1054880000FB0EF39B1AB3FBFEF300FB01314FF058
:10549800010E0191D9F80430C3F3080313BBEFF3ED
:1054A8001183FBB92B68A16800BF2A689342F9D120
:1054B800D7F800B000FB0BF2521AB2FBFBF200FB6C
:1054C8000323019A9B1AB3F57A7FE3D3BAF1010A51
:1054D800C4D1029B013B0293002B7FF466AF05B059
:1054E800BDE8F08FEFF311888CF31288A168236868
:1054F800DB0344BFC6F800E0A1682B6832685FFA96
:1055080088F888F31188D7F800801A4400FB08F35C
:105518005B1AB3FBF8F300FB0233D2E7EFF3118811
:105528008CF31288A1682368DB0344BFC6F800E047
:10553800A1682B6832685FFA88F888F31188D7F871
:1055480000801A4400FB08F35B1AB3FBF8F300FB76
:10555800023370E7EFF311828CF31288D4F808E075
:105568002368D90303D501233360D4F808E02B68F6
:105578003168D2B282F311883A68194400FB02F309
:10558800A3EB0E03B3FBF2F300FB01317FE7EFF36C
:1055980011828CF31288D4F808E02368D90303D564
:1055A80001233360D4F808E02B683168D2B282F363
:1055B80011883A68194400FB02F3A3EB0E03B3FB0E
:1055C800F2F300FB013118E7184623F043F83EE7F1
:1055D80010E000E0AC620020B0620020B46200205D
:1055E80000ED00E0204B5B68C3F3080330B4BBB99F
:1055F800EFF31183A3B91D4B1D4C1868A16800BFB8
:105608001A689042F9D11B4B1C684FF47A7202FB5E
:1056180004F3591AB1FBF4F130BC02FB00107047D7
:10562800EFF31182102383F3128811498C680B68F9
:1056380013F4803F104B02D0012018608C680B498E
:10564800D2B20D68186882F311880A4B19684FF4B2
:105658007A72284402FB01F31B1B30BCB3FBF1F345
:1056680002FB0030704700BF00ED00E0B062002090
:1056780010E000E0B4620020AC6200202DE9F84F91
:105688008046FFF7AFFF254E2549DFF8A0E0254A01
:10569800254D844610274FF47A740120DEF8043033
:1056A800C3F30803D3B9EFF31183BBB90B68D2F87E
:1056B80008A000BFD1F800904B45F7D1D6F800B04C
:1056C80004FB0BF9A9EB0A09B9FBFBF904FB0393EB
:1056D800A3EB0C034345E1D3BDE8F88FEFF3118A40
:1056E80087F31288D2F808B01368DB0344BF286038
:1056F800D2F808B00B68D5F800905FFA8AFA8AF3F6
:105708001188D6F800A0994404FB0AF3A3EB0B0315
:10571800B3FBFAF304FB0933DAE700BFB4620020F5
:10572800B062002010E000E0AC62002000ED00E074
:105738002DE9F04FDFF830C1474A4849484E494DF6
:105748008046102718F1FF38C0F08480DCF8043058
:10575800C3F30803002B5CD1EFF31183002B58D15E
:105768000B68946800BF08688342F9D1D6F80090A6
:105778004FF47A7000FB09FEAEEB040EBEFBF9FE97
:1057880000FB03EEDCF80430C3F308034FF47A742B
:105798000120FBB9EFF31183E3B90B68D2F808A035
:1057A80000BFD1F800904B45F7D1D6F800B004FB04
:1057B8000BF9A9EB0A09B9FBFBF904FB0393A3EB6B
:1057C8000E03B3F57A7FBDD2DCF80430C3F30803C7
:1057D800002BDFD0EFF3118A87F31288D2F808B0D4
:1057E8001368DB0344BF2860D2F808B00B68D5F80B
:1057F80000905FFA8AFA8AF31188D6F800A09944D3
:1058080004FB0AF3A3EB0B03B3FBFAF304FB093322
:10581800D5E7EFF3118487F31288D2F8089013685C
:10582800D80303D501232B60D2F808900B682868A9
:10583800E4B284F31188D6F800A04FF47A7400EB30
:10584800030E04FB0AF3A3EB0903B3FBFAF304FB0F
:105858000E3E97E7BDE8F08F10E000E0B062002050
:10586800B4620020AC62002000ED00E030B4EFF339
:105878001183102282F312880649074C0A680748E8
:10588800013200250A602560DBB2026883F31188C3
:1058980030BC7047B0620020AC62002010E000E02D
:1058A8001D4B70B59C68236D626BDD69C2B1A36B3B
:1058B8002BB12B0702D5236D08221A6270BD2A0668
:1058C800F7D5A26A616A8A4220D0511CA069A162F8
:1058D800825C2069266D81423285EAD3A362E8E7BB
:1058E800A906E4D5E26A22B1988C216B80B2904770
:1058F800DDE7E1699B8C6069DBB24E1CE6614354CD
:10590800E169E368994228BFE261D0E7226D136834
:1059180023F080031360CCE7642F00201D4B70B583
:105928005C68236D626BDD69C2B1A36B2BB12B0779
:1059380002D5236D08221A6270BD2A06F7D5A26A1D
:10594800616A8A4220D0511CA069A162825C2069E8
:10595800266D81423285EAD3A362E8E7A906E4D539
:10596800E26A22B1988C216B80B29047DDE7E16949
:105978009B8C6069DBB24E1CE6614354E169E368C5
:10598800994228BFE261D0E7226D136823F08003B3
:105998001360CCE7642F00201D4B70B51C68236D85
:1059A800626BDD69C2B1A36B2BB12B0702D5236DE6
:1059B80008221A6270BD2A06F7D5A26A616A8A426D
:1059C80020D0511CA069A162825C2069266D8142A9
:1059D8003285EAD3A362E8E7A906E4D5E26A22B1F0
:1059E800988C216B80B29047DDE7E1699B8C6069F8
:1059F800DBB24E1CE6614354E169E368994228BF73
:105A0800E261D0E7226D136823F080031360CCE7CE
:105A1800642F002070B4EFF31186502383F31288AB
:105A2800836B1A68D20720D45D686DB9446A826AAC
:105A3800944217D081691144D9600ED9A21A5A60CC
:105A48008462002280F854201A6842F00102F1B200
:105A58001A6081F3118870BC704701698A1A5A600C
:105A68008562EEE7012380F85430F1B281F31188A2
:105A780070BC704703685B6A03B11847704700BF82
:105A880003681B6A03B11847704700BF03682DE914
:105A9800F041DF691FB13B46BDE8F0411847002AD5
:105AA800164611DD04460D460E4400E023689B6847
:105AB800204698470028F9D0236815F8011B1B6871
:105AC80020469847AE42F1D1BDE8F0810368DB6813
:105AD800184700BF03689B68184700BF03685B68E6
:105AE800184700BF03681B68184700BF054B53F8E9
:105AF800203033B11A689B88918A0B4218BF1B0467
:105B0800936170477C620020036803F138422DE9F5
:105B1800F04F920A584DAA5C02F01F055209012461
:105B2800022A04FA05F400F08C80032A00F08E8023
:105B3800012A3CD001F003077A1E012AC1F3810C27
:105B4800C1F300188088C1F3411135D9C60700F1A7
:105B58009780850700F1A380440700F1B180020710
:105B680000F1BF80C60600F1CD80850600F1DB801C
:105B7800440600F1E980020600F1F780C60500F14D
:105B88000581850500F11381440500F12181020595
:105B980000F12F81C60400F13D81850400F14B819D
:105BA800440400F15981020455D4BDE8F08F334A0A
:105BB80055692C435461BDE7002422464FF0010E7D
:105BC8004FF0030904E00132102A04F10204ECD07A
:105BD8000EFA02F636EA0005F5D1D3F808A009FA5C
:105BE80004F5ED430AEA050AC3F808A0D3F808B09B
:105BF8000CFA04FA4AEA0B0AC3F808A0B3F804A09E
:105C08001FFA8AFA2AEA06069E80B3F804A008FA60
:105C180002F646EA0A06B6B29E801E682E401E604C
:105C2800D3F800A007FA04F646EA0A061E60D3F87D
:105C38000CA001FA04F605EA0A0A46EA0A05DD603C
:105C4800C1E70E4A95692C43946173E70B4AD569FD
:105C58002C43D4616EE71A6822F040421A601A6831
:105C680042EA87771F60DA6822F0404242EA81718F
:105C7800D960BDE8F08F00BFF4730308001002403C
:105C88001A6822F003021A601A683A431A60DA683E
:105C980022F003020A438507DA607FF55DAF1A68D0
:105CA80022F00C021A601A6842EA87021A60DA685F
:105CB80022F00C0242EA81024407DA607FF54FAF16
:105CC8001A6822F030021A601A6842EA07121A604B
:105CD800DA6822F0300242EA0112DA6002077FF540
:105CE80041AF1A6822F0C0021A601A6842EA8712A5
:105CF8001A60DA6822F0C00242EA8112C606DA6047
:105D08007FF533AF1A6822F440721A601A6842EAC3
:105D180007221A60DA6822F4407242EA01228506F4
:105D2800DA607FF525AF1A6822F440621A601A68B3
:105D380042EA87221A60DA6822F4406242EA812243
:105D48004406DA607FF517AF1A6822F440521A60E9
:105D58001A6842EA07321A60DA6822F4405242EAC4
:105D68000132DA6002067FF509AF1A6822F4404270
:105D78001A601A6842EA87321A60DA6822F44042E6
:105D880042EA8132C605DA607FF5FBAE1A6822F472
:105D980040321A601A6842EA07421A60DA6822F446
:105DA800403242EA01428505DA607FF5EDAE1A68B5
:105DB80022F440221A601A6842EA87421A60DA68B6
:105DC80022F4402242EA81424405DA607FF5DFAEE0
:105DD8001A6822F440121A601A6842EA07521A60D6
:105DE800DA6822F4401242EA0152DA6002057FF5CD
:105DF800D1AE1A6822F440021A601A6842EA875241
:105E08001A60DA6822F4400242EA8152C604DA6073
:105E18007FF5C3AE1A6822F040721A601A6842EA27
:105E280007621A60DA6822F0407242EA0162850469
:105E3800DA607FF5B5AE1A6822F040621A601A6817
:105E480042EA87621A60DA6822F0406242EA8162B6
:105E58004404DA607FF5A7AE1A6822F040521A604F
:105E68001A6842EA07721A60DA6822F0405242EA77
:105E78000172DA6097E600BF2DE9F04F4A484B4BB4
:105E88004B4C4FF090414FF0010A4FF002094FF090
:105E980004084FF0080C4FF0100E202740268025EC
:105EA80030F8022B12F0010F03D01960A3F804A0F8
:105EB800083312F0020F03D01960A3F804900833D6
:105EC80012F0040F03D01960A3F80480083312F00D
:105ED800080F03D01960A3F804C0083312F0100F9C
:105EE80003D01960A3F804E0083312F0200F02D0A1
:105EF80019609F80083312F0400F02D019609E800D
:105F0800083312F0800F02D019609D80083312F414
:105F1800807F05D04FF4807B1960A3F804B0083364
:105F280012F4007F05D04FF4007B1960A3F804B089
:105F3800083312F4806F05D04FF4806B1960A3F812
:105F480004B0083312F4006F05D04FF4006B1960E9
:105F5800A3F804B0083312F4805F05D04FF4805BD7
:105F68001960A3F804B0083312F4005F05D04FF4A9
:105F7800005B1960A3F804B0083312F4804F05D011
:105F88004FF4804B1960A3F804B00833D20B04D047
:105F98004FF4004219609A80083301F58061A142EC
:105FA8007FF47EAFBDE8F08F787303085453002068
:105FB80000180048002852D0036803F138422DE940
:105FC800F04F920A504DAA5C02F01F0552090124B5
:105FD800022A04FA05F443D0032A00F09080012A2B
:105FE80043D001F003077A1E012AC1F3810CC1F3E3
:105FF80000188088C1F341113CD9C60700F1888098
:10600800850700F19480440700F1A280020700F19F
:10601800B080C60600F1BE80850600F1CC8044063B
:1060280000F1DA80020600F1E880C60500F1F6808A
:10603800850500F10481440500F11281020500F193
:106048002081C60400F12E81850400F13C814404BE
:1060580000F14A81020400F15881BDE8F08F7047D1
:106068002A4A95692C439461BBE7284A55692C4311
:106078005461B6E7002422464FF0010E4FF00309A1
:1060880004E00132102A04F10204E6D00EFA02F606
:1060980036EA0005F5D1D3F808A009FA04F5ED436E
:1060A8000AEA050AC3F808A0D3F808B00CFA04FAFB
:1060B8004AEA0B0AC3F808A0B3F804A01FFA8AFA40
:1060C8002AEA06069E80B3F804A008FA02F646EA11
:1060D8000A06B6B29E801E682E401E60D3F800A045
:1060E80007FA04F646EA0A061E60D3F80CA001FA7D
:1060F80004F605EA0A0A46EA0A05DD60C1E7034A2A
:10610800D5692C43D4616CE7F4730308001002408E
:106118001A6822F003021A601A683A431A60DA68A9
:1061280022F003020A438507DA607FF56CAF1A682C
:1061380022F00C021A601A6842EA87021A60DA68CA
:1061480022F00C0242EA81024407DA607FF55EAF72
:106158001A6822F030021A601A6842EA07121A60B6
:10616800DA6822F0300242EA0112DA6002077FF5AB
:1061780050AF1A6822F0C0021A601A6842EA871201
:106188001A60DA6822F0C00242EA8112C606DA60B2
:106198007FF542AF1A6822F440721A601A6842EA20
:1061A80007221A60DA6822F4407242EA0122850660
:1061B800DA607FF534AF1A6822F440621A601A6810
:1061C80042EA87221A60DA6822F4406242EA8122AF
:1061D8004406DA607FF526AF1A6822F440521A6046
:1061E8001A6842EA07321A60DA6822F4405242EA30
:1061F8000132DA6002067FF518AF1A6822F44042CD
:106208001A601A6842EA87321A60DA6822F4404251
:1062180042EA8132C605DA607FF50AAF1A6822F4CD
:1062280040321A601A6842EA07421A60DA6822F4B1
:10623800403242EA01428505DA607FF5FCAE1A6811
:1062480022F440221A601A6842EA87421A60DA6821
:1062580022F4402242EA81424405DA607FF5EEAE3C
:106268001A6822F440121A601A6842EA07521A6041
:10627800DA6822F4401242EA0152DA6002057FF538
:10628800E0AE1A6822F440021A601A6842EA87529D
:106298001A60DA6822F4400242EA8152C604DA60DF
:1062A8007FF5D2AE1A6822F040721A601A6842EA84
:1062B80007621A60DA6822F0407242EA01628504D5
:1062C800DA607FF5C4AE1A6822F040621A601A6874
:1062D80042EA87621A60DA6822F0406242EA816222
:1062E8004404DA607FF5B6AE1A6822F040521A60AC
:1062F8001A6842EA07721A60DA6822F0405242EAE3
:106308000172DA6002047FF5A8AE1A6822F04042F2
:106318001A601A6842EA87771F60DA6822F04042FA
:1063280042EA8171D960BDE8F08F00BF10B10368FF
:1063380082881A85704700BF10B1036882889A6105
:10634800704700BF38B100298388026814BF002154
:1063580010218B40936170470E4B1B8801463BB957
:106368000D4B0E4A1B7810680BB981F00101E9E763
:106378000B4B5A691AB118B91A68106058747047EB
:10638800084A18681188084A92FBF1F20121026054
:1063980059747047886200208A6200208C6200204D
:1063A80090620020A862002020A1070010B40A4BC8
:1063B8000A4A1C7801238340234052F8200029B957
:1063C800B3FA83F149095DF8044BBBE7191C18BF00
:1063D80001215DF8044BB5E7786200207C6200205B
:1063E8001C4C08B501210220FFF7E0FF237803F0D9
:1063F8000502052A2AD003F00903092B08D0002139
:106408000120FFF7D3FF00210846FFF7CFFFFEE783
:10641800114A124B11681A680B68114C4FF6FE703E
:1064280003400B601388206823F001031B041B0C36
:10643800138018B12A2200238271C37102224E21CF
:10644800FEF7EAF92068FFF771FFD8E71BF0A4FA16
:106458002378D0E7582F0020C4270020C827002021
:10646800AC2F002030B1036882881B8A1A4214BFFF
:1064780001200020704700BF2DE9F0410B4E356820
:1064880073691D4010D0DFF828800127B5FA85F41C
:10649800C4F11F0408EB840307FA04F4D8680368FE
:1064A8009847A5437461F1D1BDE8F081000401402B
:1064B800102300202DE9F04FBF4B1E788BB0002E23
:1064C80040F0BC80BD4BBE4C1D78DFF814A3DFF84C
:1064D8001493DFF8148305F00105A4F10A0B54F8AE
:1064E8000A3CBBB1CC2707FB06B71846FFF7F6FAFC
:1064F80080B154F80A0CFFF7E9FA14F8023C8BB99A
:10650800242831D0F5B154F80A3C1846FFF7E6FACA
:106518000028EED10136032E04F1CC04DFD10BB0F4
:10652800BDE8F08F012B23D0022B2BD0032B37D0C3
:10653800042B67D0052B40D0062B4FD054F80A2CDB
:106548001346D2E754F80A3C23281A4600F08781FC
:106558009C4991F832108142C7D19B4BCAF80090F0
:10656800C3F80C801346C0E7012304F8023CCAE7CD
:106578004D2854F80A2C0CBF0223002304F8023CCF
:106588001346B2E700233C2804F8023C45D03E28D5
:10659800D4D10122032304F8012C04F8023CB2E709
:1065A800C02814D80022042304F8050C04F8040CAD
:1065B80004F8062C04F8023CA5E714F8063C14F885
:1065C800052C9A422FD814F8043C834203D00023A8
:1065D80004F8023C97E7062304F8023C14F801EC9F
:1065E800BEF1000F00F08081BEF1010F00F0C48100
:1065F80001360023032E04F8023C04F1CC047FF496
:106608006EAF8CE714F8043C04F8030C58400523DB
:1066180004F8040C04F8023C75E7032204F8013C72
:1066280004F8022C6FE714F8042CF91842400133DF
:1066380004F8042C04F8063C887264E7634B186875
:1066480000283FF46CAFFAF743FBDFF8A0A1604DD8
:10665800DFF89C91DAF80000FFF740FA00283FF4D1
:106668005EAFDAF80000FFF731FA09281BD03F289F
:1066780019D02B68002B66D1042800F0A8810C28BB
:1066880000F0E6807F28E5D0A0F12002D2B25E2A91
:10669800E0D80BB92028DDD05A1C09F803002A607D
:1066A8001CF068F9D6E72C68002C5AD1494B2646CD
:1066B80003F59478002E08BF1E4608334345F9D1E8
:1066C800002E00F07881A3F1080B3068DBF8002079
:1066D800075D135D9F42204402EB040140F069818D
:1066E800671E4F4422460BB9FD2A5CD907F8013FC3
:1066F80001322A6010F8013F11F801EF9E45F2D0EF
:106708000AB1B34512D034481CF03CF9B34508D35C
:1067180056F8080B1CF036F909201CF02BF95E45D9
:10672800F6D92E481CF02EF92A680024944291D2FA
:10673800661E4E4416F8010F1CF01CF92B68013434
:106748009C42F7D386E70C2800F082800A2851D0B3
:106758000D284FD07F2800F0FC80FF2B3FF67AAF42
:1067680092E71C4F4FF0000B07F594785E4602E065
:10677800083747450DD0224639684846FAF7B6FD2E
:106788000028F5D1BB46002EF2D13E4608374745D2
:10679800F1D1002E99D1BBF1000F3FF45BAF0E4849
:1067A8001CF0F0F8B4E7511C202009F80200296019
:1067B80009F801300A46A4E71C4E002009710020A0
:1067C800068F00202C5E002000ED00E098330020AA
:1067D800A0340020145503083C7C0308447C0308BB
:1067E800FC9F0020EFBEADDE0400FA059C330020BC
:1067F800A03300201CF047F923217D482EF024FC0B
:10680800002800F0E280A0EB0900286088B1431E50
:1068180019F80310202940F0E88009EB030204E08E
:1068280012F8011D202948D10346581E002BF7D124
:106838002B604FF48072002148462EF0EEFB6D4B22
:106848001B78002B3FF46BAE6B481CF09BF801E7FC
:106858006A481CF097F868481CF094F8FAE668490A
:106868006848C978684ADFF8D0E1D364003118BFB6
:1068780001210170654911654021536582F858105E
:1068880082F85950624963480B605032CEF80020B4
:10689800584A012313701CF089FB57481CF072F802
:1068A8004FF400600AF0AEFE5B4B93F83230232BB6
:1068B80000F0938014F8023C3EE62B60574C00220F
:1068C80004F5947809F8032002E00834444578D0A8
:1068D8002168484611F0E4FC0028F6D0444570D2FF
:1068E800636898470023A3E74D4BADF822E00FCB30
:1068F8000DF1280C02AF87E80F004CF824ED14F8CE
:10690800051C14F8033C069404EB010E6246394654
:106918004FF0010C06A8CDF81CE0ADF820308DF83A
:1069280024C002F057FFE8B9019F002304F8023C95
:10693800002F3FF4EFAD54F80A0C0BF0E7FC0136DA
:1069480054F80A0CB847032E04F1CC047FF4C7AD01
:10695800E5E5013B002233482B6009F803201CF0D1
:1069680011F877E6029A304B03923946A4F10A00EF
:1069780002930BF00BFCD7E714F8053C14F8032C32
:106988000694234407936E2A4FF000030893099353
:10699800ADF820207FF42CAE06A8FAF726FD06A84D
:1069A800FAF718FD06A8FAF715FD06A8FAF712FD7A
:1069B8001EE62246A4E61D48A3F1080B1BF0E2FFE1
:1069C800A6E61B481BF0DEFF8CE728681EE7084890
:1069D80010F04DFB0BB0BDE8F08F164A14F8023CDE
:1069E800C2F80C80CAF80090A6E5034666E700BF27
:1069F800A03300201C4E0020447C03084C7C030874
:106A08001C6200202828002010230020F9390008E3
:106A18009C330020787C03082C5E00201455030862
:106A2800A0520308747C0308349300203C7C0308BC
:106A3800587C030800ED00E0983300202DE9F04F62
:106A48002DED068BAB4BAC4A1C7897B000F59C41FA
:106A5800203181460B911160002C00F0D186A74AA5
:106A68001268904240F28380A54A06921668A549AA
:106A7800A54A0591013C1C70A44B049206F480566B
:106A88000893002E40F08180A14B1B78022B01F067
:106A98008B81042B01F07A81012B01F0FA809D4B48
:106AA8009945089B9B7800F27C85002B40F07D85FA
:106AB800994B0793069B1E6816F4805740F06E8624
:106AC800DFF894A2049BB3F90610059B5D8BA942DD
:106AD800B4BF00250125914B1B6813F080535ED08D
:106AE800079A127812F001025FD00598408C88420C
:106AF80041F3AF82002D5ED1894C94F88C100029A7
:106B080059D188488849006890F82D0000240C6005
:106B18004C608C60854900284ED10870002A4FD0FF
:106B2800F2064DD5824A1278D40649D4002F47D1AF
:106B3800002B45D1700243D47E4B1B78002B02F00A
:106B480018827D4B9B78002D42F0AB823BB17B4A8B
:106B58007B4B12681B689B1A002BC2F2AE82102076
:106B68006F4C27F05FFC012384F88D3028E0644BDC
:106B780006931E68644B634A049306F48056634B7D
:106B880005920893002E3FF47FAF00216348FAF77F
:106B9800C6FF00287FF478AF0DF044F874E7700260
:106BA8009ED4079A127802F001025D4C002184F805
:106BB8008C10002DA5D05D4901200870002AAFD1A6
:106BC800604B1A78002A79D10599049C488BB4F94E
:106BD8000070898BB4F90240B842B4BF8026002601
:106BE80046F04003B942D8BF33469B0843F08006BD
:106BF800A042B8BF3346049F43F04006A142C8BF35
:106C080033469B08B7F90440B7F9066043F080079C
:106C1800A042B8BF3B4643F04007A142C8BF3B462D
:106C28009B0843F080073E4C8642C8BF3B4643F072
:106C3800400794F88EE08E42B8BF3B469E4501F06F
:106C48002B84A4F8902084F892203A4984F88E3056
:106C58000E78002E01F035835F2B01F0A8836F2B8F
:106C680001F0BD83079B1B78DF0727D494F89210A7
:106C780021BBB4F99030322B20DD94F88E2001200E
:106C8800572A84F8920001F05A87069B1B685D0713
:106C980041F183825A2A41F0808294F89430002B83
:106CA80042F07B8194F8963083F0010384F89630A3
:106CB800002B42F0C0810C2027F0B4FB224B099333
:106CC800224B234D0A93069B1B685F0700F1E2865F
:106CD8000DF150091F4E0B950022C9F804203446C7
:106CE800149240F6330B4FF0190840F28337049D95
:106CF80037E000BF846B00208C6A0020806B002086
:106D080020570020307400202C3E0020C04B00206B
:106D1800EE6A0020404B4C00097100205C460020C0
:106D2800AC23002084680020C84300205826002097
:106D3800683E0020EF200020B0460020B06200200E
:106D48000030002088640020246800208868002023
:106D580080680020B072002000730020043454457D
:106D680022D0A178E378994218FB0170F6D294F802
:106D780001E00EF1040E18FB037135F91E305B4576
:106D8800A8BF5B46B3F5617FB8BF4FF46173984203
:106D9800E4DA9942E2DB21782729DFD8484604342F
:106DA800FAF7AEFE5445DCD1614A0B9D1378614A6F
:106DB80099E8030082E80300002B40F0E4855E4B6D
:106DC8001A78002A00F05E8501215A48FAF7A7FED2
:106DD800002840F0DA82089BDB78002B40F0D5824F
:106DE8002B881FB227F001071FFA87F84345A5F83B
:106DF800008001F00880514F4FF002090E204FF03B
:106E0800140B4FF0FF0A87F8009087F801B087F855
:106E180002A027F007FB49464648B5F80080FAF774
:106E28007EFE002841F0928228F002039BB243457F
:106E38002B800BD0414B02201421FF2218700E200A
:106E480059709A7027F0EEFAB5F800803C4B3D4A2D
:106E5800197850680B9318F0030F08BF81F00201EE
:106E6800C1F340010C92FFF76DFA24213148FAF77B
:106E780056FE30B9079A13785F0744BF23F004031E
:106E88001370099B1B6813F00A0F11D006212948BB
:106E9800FAF745FE002801F0B3802B88580641F127
:106EA8001D8207212348FAF73AFE002840F0CE87D2
:106EB8000C212048FAF733FE2A88002800F0458381
:106EC80042F480739A422B8009D01C4B0222142171
:106ED8001A700E20FF2259709A7027F0A3FA1A4BE5
:106EE8001B78082B00F03D830E2B00F03A83069B9D
:106EF800D3F8008018F4806F60D0144B1B79002BF6
:106F080000F0258214210B48FAF709FE002840F00A
:106F1800238213F027F8012027F0C6F900284AD069
:106F2800DFF82CA000274FF0CC0BA14615E000BFDE
:106F3800445900205C4600201C4E002030330020BD
:106F4800786200207C6200205444002004680020FD
:106F5800FC8E0020DFB2022F2CD80BFB07F87B1C1D
:106F68005AF80840002CF5D1032290F90230029417
:106F78000192C278E24951F822200092184622462E
:106F88002346012126F0D0FD034607EB470000EB1E
:106F98000010099353B121460AEB8000CC222EF051
:106FA8003CF8099B4AF808300137FFB220F0CAFFC5
:106FB8000028D0D14C46069BD3F80080079B93F855
:106FC80000A0D04B1AF0010A00F0408201221A708A
:106FD8000A9B04991B68B1F906105A89CA48012707
:106FE8009142077080F21882C84B4FF07E521A60A7
:106FF800059BC74FB3F81890049B97F90420B3F981
:107008000030387897F801C0002AA3EB090714BFAD
:1070180001224FF0FF32002FB8BF7F42B7F5FA7F49
:10702800A8BF4FF4FA77B84280F2F3813F1A07EE0F
:10703800907AF8EEE77AB74F4B45C7ED007A03DA56
:10704800F1EE677AC7ED007A049BB3F902E0AEEB84
:107058000903002BB8BF5B42B3F5FA7FA8BF4FF412
:10706800FA73984280F2D2811B1A07EE903AF8EE32
:10707800E77AF145C7ED017A03DDF1EE677AC7EDEE
:10708800017A049BB3F90400A0EB0903002BB8BFF5
:107098005B42B3F5FA7FA8BF4FF4FA736345CCBFE0
:1070A800A3EB0C03002302FB03F207EE902AF8EE91
:1070B800E77A4845C7ED027ABCBFF1EE677AC7EDBB
:1070C800027A18F4805800F07E81B1F5FA6F924B7D
:1070D800A8BF4FF4FA61B1F57A7F1A78B8BF4FF4B8
:1070E8007A71A1F57A71002A41F020818B4ADFF884
:1070F80044E282FB0130CB17C3EB6013581C6FF0DE
:10710800630C3EF910003EF913E00CFB0313A0EBEF
:107118000E0003FB00F382FB0312DB17C3EB6213C1
:107128009E440FFA8EFE07EE90EAB8EEE78A87EDE6
:10713800038AB8F1000F40F04D842B885A0640F1BD
:10714800FB807749774A91ED018AD2ED019A92ED59
:10715800026A91ED034A92ED030A91ED029A92EDCB
:10716800007AD1ED005AD7ED011A97ED002A6E4A40
:107178006E4938EE445A79EEC63A77EE007A65EEF3
:10718800233A75EEC96A75EE890A37EE401A66EE3B
:10719800A76AB0EE633AA0EE813A13F00303B0EEAB
:1071A800665A78EE044A79EE867AA0EE815AF0EEB5
:1071B800638AA4EEA73AD4EEA78AA4EEE75A33EE80
:1071C800263AF0EE687AF0EE674AF6EE008A35EE77
:1071D80088AAE0EEC14A28EEC33A35EE635A77EE44
:1071E800293A77EEE67AAAEE233A25EE285A76EE81
:1071F800403A34EE49AAE0EE817A74EEA64AAAEE45
:10720800235A34EE094A37EE697A64EEA84A63EEE7
:10721800036AE4EE074A75EEC85A36EE006A67EE6E
:10722800A87AB0EE667A95EE057AE5EE056AE5EE9F
:10723800867AB1EE648AF0EE665AF0EE476AB1EEED
:10724800674AE8EE246A63EE270A67EEA43AE4EE9A
:10725800275AB1EE450AB0EE606AB0EE631AA4EEA2
:10726800277A23EE244AE7EEA76AA5EE246AA0EE61
:10727800031AE8EE245AB0EE448A31EEA19AE0EE01
:10728800240AA5EE278A66EEA16A72EE028AE5EE66
:10729800033A61EE211A26EE096AA4EEA47AA0EE5A
:1072A800274A0CBFD7ED022ADFED212A82ED005ACA
:1072B800A2EE256AE0EEA86AE2EE081A73EEA33A97
:1072C80027EE227A34EE044AF0EE005AE3EEA26A80
:1072D800A4EE226AA1EEA57AC7ED016AC1ED366A6D
:1072E80081ED356A87ED006A81ED377A82ED013AE2
:1072F800C2ED027AC2ED034AF3B987ED027A1BE0C8
:10730800406D03080A710020902600200C260020FA
:1073180088460020A84B0020B02700201F85EB518D
:10732800580000201C0B0020540B0020AC23002028
:10733800000000009C490020BAF1000F40F02481B1
:107348002BF06CFB17B0BDEC068BBDE8F08F079BEC
:107358001B78D9077FF5DDAD4FF40F702AF0F2F8EE
:1073680000283FF428AE0BF09BF84FF40F702AF07A
:107378008BF800283FF41FAE0BF092F84FF40F7013
:107388002AF082F80028EED115E6099B1B689B07B6
:107398007FF526ADB5F8008018F0010F7FF444ADF5
:1073A80048F0010398452B803FF43EADC14B0222C3
:1073B80014211A700E20FF2259709A7027F032F8A3
:1073C800B5F8008030E5059B5A8B9142C0F21885CC
:1073D800B1F5FA6FD4BFC2EB0101C2F5FA614FF4FF
:1073E8007A7303FB01F1B4480378C2F5FA62B1FB82
:1073F800F2F1002B3FF47AAE4378B04A01FB03F177
:1074080082FB0123C917C1EB63116FE6DFEDAC7A8C
:107418002FE6DFEDAB7A0EE6B1F5FA6F80F2E9847C
:10742800187A8B1A03FB00F3C2F5FA6293FBF2F3A6
:10743800C3F1640307EE903AF8EEE77A9FEDA17A7C
:10744800A14B67EE877AC3ED007AD1E51B780693E6
:10745800002B7FF4BDAD9D4A1268002A3FF4B8ADF9
:107468009B4A079212F8030CDFF8A0B21146D71E08
:107478001AF05AFF9BF80090079A002800F034860B
:10748800069BB9F1000F41F0298507F108017879C9
:107498001AF04AFF002841F034858E49B87A1AF06C
:1074A80043FF002800F03386B9F1020F41F031851F
:1074B8008949F87B1AF038FF002841F0268587496A
:1074C800387D1AF031FF002800F03386B9F1040F37
:1074D80041F02F858249787E1AF026FF002841F076
:1074E80024858049B87F1AF01FFF002800F03386F2
:1074F800B9F1060F41F015857B4997F823001AF07A
:1075080013FF002841F00985784997F828001AF0F8
:107518000BFF002800F03386B9F1080F41F0ED8425
:10752800734997F82D001AF0FFFE00283FF450AD7C
:107538000922134602EB820217446E4A7878B9781A
:107548008BF800301070517042E522F480739BB2C2
:107558009A422B807FF4B9AC674B1B78082B7FF4D9
:10756800C3AC2A8822F040039BB29A422B803FF496
:10757800BEAC504B022214211A700E20FF22597003
:107588009A7026F04FFFB2E40B9B19780C9B01F020
:1075980001011868FEF7D6FE17B0BDEC068BBDE8F2
:1075A800F08F13B9089A01239370544B089A1D78E9
:1075B80092F8214007931B201AF0EEFE012C05F0EB
:1075C8000108814600F0088705F00205089A4C4E2C
:1075D80092F82030DFF838A14A4F09959346052BD9
:1075E80000F29887DFE813F0BF00B5000600FD0041
:1075F800FF00F200012C04BF05238BF82030B8F1FE
:10760800000F12D0059B3088B3F9181000221346DA
:1076180061F30F0260F31F4261F30F03049861F3F3
:107628001F430360032342600993374DDBF81410AE
:107638002A68914280F0358647F230510322CBF810
:107648001C108BF82020022009F0DCFF0CF0EAFA6D
:107658002968DBF81C200A440421CBF818208BF891
:107668002010012C40F0A7872A68DBF818109142F7
:1076780080F050879AF8000020B91AF08DFE002893
:1076880040F048873A6822F002023A602A68738814
:10769800642101FB03234FF480600022CBF81030F3
:1076A8008BF820208BF8032009F07CFF9BF8203012
:1076B80095E700BF30330020B02700201F85EB512D
:1076C800000000000AD7233C0C2600200C71002083
:1076D800E6320020F0320020F5320020FA32002095
:1076E800FF32002004330020093300200E3300202D
:1076F8001333002010710020544400200971002029
:10770800944900207C680020B06200201500002009
:10771800EF2000201AF046FE012807D1B14D7288EB
:107728002B68642101FB0233CBF81030B9F1000F4C
:1077380002D0B379002B4BD1012C00F0EB86A94D78
:10774800DBF810102A689142C0F02A8701238BF8D1
:107758002030012C3AD0F379012B46D01AF0A2FD43
:107768009BF820303BE7B8F1000FD3D1099D4FF4C7
:107778008060B9F1000F00F0668309F02BFF089ACA
:1077880000231361002D3FF495A9284626F04AFEF0
:10779800069B1E6816F480573FF492A91D21924853
:1077A800FAF7BDF900287FF48BA9904B03F1500A32
:1077B80003E004339A4500F0B3861A78262AF8D1F4
:1077C8009978DA789142F4D2FFF77CB9854D5DE774
:1077D8001AF068FD03224FF47A738BF82020CBF857
:1077E8001C30804D2FE77F4D3BE71AF05BFD0322ED
:1077F80040F6B8338BF82020CBF81C30794D22E7BF
:107808007B4F3B78002B01F080827A4BDFF8F881C0
:10781800DFF8F8B1DFF8F8A1059345465E46049015
:1078280099460EE019F804109847032C28DC88B90B
:107838003B782AF8020F01349C4205F1040580F2D6
:107848004E81072CE1B23046DBF80430EADD984778
:1078580000B2EDE738F824206B88801A4FF47A716B
:107868009B1A01FB00F040F6CA0290FBF3F00844B3
:10787800904240F2EE23A8BF10469842B8BF18467F
:1078880000B2D5E7DFF88C91DFF88CA15A4F0B9244
:1078980009F15A084FF0010B494619F8010C1AF082
:1078A80043FD00B399F8040099F8023099F803E011
:1078B80000EB400107EB8101013BD1F8A02003EB6D
:1078C8004303534493420ED097F8CC20C1F8A0301C
:1078D8000BFA00F022EA00000B9B81F89CE0C1F84B
:1078E800A43087F8CC0009F10609C145D4D1434B2F
:1078F8003C4A1B780B930A9BDFF820A112681B688F
:107908000C93AAF19C094FF0000B9046DAF804306A
:1079180083B31F7877B3DAF80820A8EB0202002AAD
:107928000CDB99F8CC20012101FA0BF122EA0102C3
:1079380008F5FA7189F8CC20CAF808100B9ACAB170
:107948009AF8002059780432D2B2002940F087838F
:1079580005990498098B30F9122001F1C800824278
:1079680040F3F08599F8CC109A7841FA0BF3D807D0
:1079780040F17A860BF1010BBBF1040F0AF10C0AF6
:10798800C4D1FFF721BA194B03E004339C423FF4FA
:1079980016AA19782329F8D19878DA789042F4D27F
:1079A8001148FAF7BCF800283FF409AA144B1B68E1
:1079B80013F4003341F089820022124B1046995C7F
:1079C800142902F10C0201F0378101301828F6D190
:1079D800FFF7F5B91D210448FAF7A1F820B300F024
:1079E80073BD00BFB06200205C460020B07200206A
:1079F8007073002030740020AC230020A54B0020B9
:107A0800F0310020AC58030888730020786A002001
:107A1800AA230020FD310020B0520308482400208A
:107A28000436B4423FF489AB31782629F8D1B278CC
:107A3800F3789A42F4D2089BDB78002B7FF47DAB75
:107A4800B848FAF76CF8DFEDB87A002801F07481CD
:107A580038EE678AB54AB649FDEEC87ACDED047AA4
:107A6800BDF910301B0382FB0302DB17C3EBA21224
:107A7800C9F57A731BB203FB02F343F30F334B448C
:107A880007EE903AF8EEE77A0123C7ED037A0B7018
:107A9800FFF753BBA74C94F896305BB1079B1B7854
:107AA800DE0707D5049BB3F90620059B5B8B9A423A
:107AB80000F3CC8511219B48FAF731F8002800F033
:107AC800B68294F89A302BB994F8943013B93223CB
:107AD800A4F89830012384F89A30FFF7F9B8DDF854
:107AE8001090954A06929149126842F2010AA1FB48
:107AF800091B12EA0A0A4FEA9B1B00F095828F4D78
:107B08008F48904C90492E780078267008701EB1E6
:107B18008D490E7886F00106864C0F2184F82410D2
:107B2800002B00F0E383059D884BB5F826C0B5F817
:107B380024E0059D109318462D8B0078844B1295F0
:107B480094F825500995834D0495A3FB00535B08D1
:107B580003EB4303C31ADBB20F90CDF834C002F431
:107B680080520C9304F128000BF59673CDF84490DD
:107B780097F80080DDF82490DFF808C20994754C66
:107B88000E91139200210A930896CDF81CE0089BE9
:107B9800002B00F02883099B079D33F911201FFA59
:107BA80082FEAE454FEA410303D30D9DAE4540F238
:107BB8005F835CF82120934580F01F83E25EBAF171
:107BC800000F40F0348301314145E25200F10600D4
:107BD800DDDB0E9A099C604B84F824200F2A494665
:107BE8000CBF01220022DDF8449084F825101A7099
:107BF80000F08383594B5249534ADFF88CB10893FC
:107C08001C46042001230B70137009F0FBFCDBF801
:107C18000030A1686268E3605B1A934284BF002366
:107C280084F82130069B3C781E68002C01F0A58062
:107C3800059A4B4DB2F824E0178B464916F4805646
:107C4800284640F0968332460EE0437803EB8303E0
:107C580003EB830303F2EE239BB20132A24221F825
:107C6800023B00F102000ED015F81230002B00F094
:107C78000383022BE9D001320B8821F8023BA24290
:107C880000F10200F0D1109A137801331370FEF757
:107C9800F8BE284CD4F88830A9EB0303002BFEF675
:107CA800FEAE304A304B527C059933F812308A7D4B
:107CB800DFED2E6A9FED2E6AC97D9BB207EE102A72
:107CC80007EE903AB8EEC77AF8EEE77A27EE267A0A
:107CD80067EE867A0B9AC4F88820C7EE876A40F266
:107CE800FF32FCEEE67ACDED077ABDF81C30934200
:107CF80028BF134609B1D31A9BB21E481E4D0178FE
:107D08001E4C35F81160226825F81130921B134477
:107D180001311B4D236001F00F021B0902702B80FB
:107D2800FEF7BDBE5C46002000007A44D34D6210C9
:107D380084260020AC23002020570020546A00200D
:107D48003C200020A54B00203D200020657200202B
:107D5800ABAAAAAA2C3E002060440020C04B0020F9
:107D6800BC73002028620020486200200000C8423E
:107D780000008044EF6A0020F46A0020F06A0020C6
:107D8800183E002068720020B0620020FDF72AFC2F
:107D9800BD4BBE4A1B68C31A93427EF780AEBC4BEC
:107DA80000221A80FEF77BBE059A0499537DD27D86
:107DB800013B31F913301AB1C3F53B6308331BB2E9
:107DC800A3F57A7307EE903A9FEDB27AB04AF8EECF
:107DD800E77A40F2FF3167EE877AFCEEE77ACDED7D
:107DE800077ABDF81C308B4228BF0B461380FEF77C
:107DF80056BE1B7AC3F1640307EE903AFFF71CBB2B
:107E08004146FFF7F0BA0221A348F9F788FE002897
:107E18003FF40AA82F8018F0020F7FF417A848F043
:107E2800020343452B803FF411A89C4B02221421E6
:107E38001A700E20FF2259709A7026F0F3FAB5F8DE
:107E48000080FFF703B809F0ADFB98E4944AB2F953
:107E58000030002BB8BF5B42B3F5E17FBFF628A81E
:107E6800B2F90230002BB8BF5B42B3F5E17FBFF631
:107E78001FA88C4B93ED096AD3ED076A93ED057A39
:107E8800D3ED037A76EE866A77EE877A76EEA66A7F
:107E9800B7EE007A37EE666A77EEA77AB0EEC66A72
:107EA800F0EEE75AB4EEE56AF1EE10FAB4BFB0EEC0
:107EB800655AB0EE465AB5EE405AF1EE10FA40F067
:107EC80096839FED797AB4EEE56AF1EE10FA44BF35
:107ED8009FED766A36EE477AB7EE006AF4EEC66A28
:107EE800F1EE10FAC8BFDFED726AF5EEC07AC8BFCE
:107EF80036EEC77AF1EE10FA48BFB1EE477AF6EEE1
:107F0800007A27EE677ADFED697A77EE276ABDEEA9
:107F1800E66A16EE103A2033402B40F24586DFED34
:107F2800656A654ADFED637AC2ED006AFDEEC76AED
:107F3800C2ED017A16EE903A2033402BC2ED027A58
:107F480049D8DFED5B7AB4EEE77AF1EE10FA41F347
:107F58000C809FED5A6ADFED5A6A01E0B0EE677A4D
:107F6800B4EEE67AF1EE10FA77EE467AF6DC9FED9B
:107F7800557AF4EEC77AF1EE10FA41F10A809FEDD6
:107F88004F6ADFED516A01E0F0EE477AF4EEE67AE7
:107F9800F1EE10FA37EE867AF6D4DFED447AB4EED5
:107FA800E77AF1EE10FA40F39A86DFED417A37EE80
:107FB800C77A27EE076ADFED455ADFED456ADFED40
:107FC800457AE6EE256A67EE065AE6EE267AA5EECB
:107FD800A77AF0EE477A404BC2ED037A1A6812F49A
:107FE800003240F059863D4B1046995C0A2902F14F
:107FF8000C0200F0408501301828F6D1FEF758BF72
:108008002A8822F040039BB29A422B803EF449AF63
:10801800224B022214211A700E20FF2259709A70E6
:1080280026F000FAFEF73DBF2D490E786FE594F86B
:108038009430002B3EF44CAE079B1B7813F00103E1
:108048007EF446AE012284F8943084F89520FEF739
:108058003FBE244C012184F88C10FEF7ACBD0129E9
:1080680000F0308599F8CC20012303FA0BF30BF1CB
:10807800010B1343BBF1040F89F8CC300AF10C0A49
:108088007FF444ACFEF7A0BED024002060E31600C5
:10809800183E00206F12833F5C46002030330020DA
:1080A800306800202C0B0020A7DFA834DB0FC93F65
:1080B800DB0F49400000000058000020DB0FC940DA
:1080C800E4CB1641DB0F49C0E4CB16C192E741B9B6
:1080D8009730083C15A82ABEF0310020AC58030898
:1080E800A54B0020AC230020511D78791AF01CF90B
:1080F80000283FF4D2A9B9F1010F40F0028707F137
:108108000D01B87A1AF010F9002840F00287BE492C
:10811800F87B1AF009F900283FF4D1A9B9F1030F47
:1081280040F0F386B949387D1AF0FEF8002840F08F
:108138000087B749787E1AF0F7F800283FF4D1A9EC
:10814800B9F1050F40F0F186B249B87F1AF0ECF8A2
:10815800002840F0E686B04997F823001AF0E4F8C2
:1081680000283FF4D1A9B9F1070F40F0D686AB49F2
:1081780097F828001AF0D8F8002840F0BE86A849D9
:1081880097F82D001AF0D0F800283EF421AFB9F185
:10819800090F3EF41DAFFFF7CBB95D2A00F06982E5
:1081A8005B2A00F0B6855E2A00F03386562A00F076
:1081B8007786972A00F0C186A72A00F01E86994D77
:1081C8002B889B0740F0E985A2F1B703072B00F243
:1081D8008A82DFE813F07A028802880288026C0239
:1081E80088025E025E02079B002B3FD05CF82120CC
:1081F80093454FEA4103FFF4E1AC8B4A8A4DD25CC8
:1082080005EB030E002A00F09480022A47D19EF85D
:10821800012002EB820202EB820202F2EE2292B20B
:10822800032933DD12B2BAF1000F3FF4CCAC0C9D38
:1082380020F81520B9F1000F03D10F9D022D7FF60C
:10824800C2ACB0F802900288B0F804E04A44964400
:10825800764A0FFA8EFE82FB0E52754DA2EBEE7235
:1082680025F803E012B24FF00109ACE41A464B00BE
:108278000A9D4CF82150A2E4D3B2022B04D9032B57
:108288007FF4F9AC7346E8E43B46E6E4012505FAD9
:1082980001FE0E9D25EA0E0512B20E958FE4E25AF4
:1082A800BEE7644A1278002A7FF4C6A9B8F1000F25
:1082B8003FF4C2A9012C40F02D819BF82030FFF734
:1082C8008EB931465C48F9F72AFC002800F0C080D6
:1082D80084F893600CF0C8F8FEF7C4BC43F0400281
:1082E80093422A807FF494AEFEF7DBBD534B544A89
:1082F800109201221A70534B04931B214E48F9F730
:108308000EFC00287FF476AC4F4BDFF840B10893A1
:108318001946DBF80030CA688B609B1AC82B00F23C
:10832800FC84069B1E6806F48056ACE45B78FFF775
:1083380064B8CAB2022A40F2B983032AAFD1129AAA
:10834800139D079E002D08BF324669E728F00103F8
:108358009BB243452B803FF45EAD0E2087F800901A
:1083680087F801B087F802A026F05CF8B5F800801D
:1083780051E500220FE0437803EB830303EB83030B
:1083880003F2EE239BB20132A24221F8023B00F134
:1083980002003FF478AC15F812301BB1022BEAD07A
:1083A8000B88F0E7D3B2032BFAD83B46EBE7B2F5DC
:1083B800FA7FFEF683AC94F89230002B7EF47EAC04
:1083C800079B1B7801210B4084F8921000F0D4839E
:1083D8000BF028FCFEF772BC0025FFF7F7B8B2F5E2
:1083E800FA7FFEF66BAC94F89230002B7EF466AC04
:1083F800079A12780121D20784F8921000F17C8440
:108408000CF032F8FEF75ABCF5320020FA320020A0
:10841800FF32002004330020093300200E330020EF
:108428001333002080680020BC7300205655555532
:108438001C240020482600205C46002060440020C0
:10844800657200202C3E0020C04B0020B062002046
:10845800079BC14A1B781060D9077EF507ACBF4B54
:108468001B78002B3EF42AAC089BDB78002B7EF4AB
:1084780025AC94F893300133DBB2032B84F89330A6
:108488007EF61CACB64B5B7813B9002D7EF416ACA7
:108498000BF0C8FBFEF7E6BBB24AB3491068B4F963
:1084A8009020C66981FB06018911F617701A00F53C
:1084B800FF407F3082423EF7C8AB891B0A4412B2A4
:1084C800A4F89020FEF7C1BB089BDB78002B7FF453
:1084D800ABAADFEDA67AA44938EE678AC9F5FA6334
:1084E800FDEEC87A1BB2CDED047ABDF91020120357
:1084F80081FB0201D217C2EBA11203FB02F343F383
:108508000F334B4407EE903AB8EEE78A87ED038ABB
:10851800FFF78ABA099D002D3EF4CCAAFFF735B9BA
:10852800934A059BD588049A1B8BB2F906105A1BEF
:10853800914240F388802B449942B4BF002501251D
:10854800FEF7C9BAC8398A4242DA99F8CC109A7843
:1085580041FA0BF3D9073FF50DAA524201200D92BB
:1085680026F046F87B1E0D9A162B00F28881DFE86C
:1085780013F00A021E02F201430232025702DD0121
:10858800C801B3019E01890186014302780157029F
:10859800DD01C80163014F013B016C022501DE00CA
:1085A80019F080FE032140F6B8328BF82010CBF882
:1085B8001C20FFF748B8AB460899DBF80020CB69C8
:1085C800099D13448B61002D3EF474AAFFF7DDB8B2
:1085D80099F8CC30012202FA0BF223EA020308F5DB
:1085E800FA7289F8CC30CAF80820FFF7C3B9B4EE9C
:1085F800E56AF1EE10FA8CBFB0EE654AB0EE464A75
:10860800C4EE054A9FED5B2A9FED5B5ADFED5B1ACE
:10861800DFED5B2A9FED5B3ADFED5B3A9FED5B4A4E
:10862800A4EE825AE4EEE12AA4EE857AA4EEA23AF8
:10863800B0EE475AB0EE637AA4EE837AA4EE874A86
:1086480084EE057A3FE40125FEF745BA002150483B
:10865800F9F765FA00287FF42DAA322384F89600EA
:10866800A4F89830FFF726BA002A0CBF0120022090
:1086780075E7484B002201204749484C0B60484B9E
:108688000993484B2270484D0A9325F0B1FFFEF735
:108698001ABB444A414B0A921146444A0A600222D4
:1086A8005A703F4B099319F0DBFEFEF70CBB3D4AAD
:1086B8003A4B0A9211463E4A0A6000225A70384BD9
:1086C800099319F0CDFEFEF7FEBA364A334B0A92EB
:1086D8001146384A0A6001225A70314B099319F041
:1086E800BFFEFEF7F0BA9E2A00F09D849D2A00F096
:1086F8009284AE2A00F08784AD2A00F07C84EF2AA9
:1087080000F07684FD2A00F06184FB2A00F09C8446
:10871800FE2A00F09684F72A00F090847B2A00F065
:108728004E841F4B09931F4B0A93FEF7CCBAD9F816
:10873800D000214B90F836109B7811446429A8BFCB
:10874800642121EAE17180F83610002B40F0918411
:1087580018F0DEFE86E400BF04300020A54B0020A0
:10876800B046002074330020D34D621000007A44D4
:108778007849002099FB243F69A2163E39094E3DED
:10878800E3B59E3E88FA163E45FE7F3FA7DFA83434
:108798005C46002024350020846800201C620020EC
:1087A800246800208868002080680020483600205F
:1087B800303600203C3600206A3E0020D9F8D00030
:1087C800BC4B90F837109B781144FE29A8BFFE21B6
:1087D80021EAE17180F83710002BB9D0162019F082
:1087E80025FED9F8D000B3E7D9F8D000B14B81788D
:1087F8001144C829A8BFC82121EAE17181709B787A
:10880800002BA5D0142019F011FED9F8D0009FE74D
:10881800D9F8D000A74B41781144C829A8BFC8216E
:1088280021EAE17141709B78002B91D0132019F057
:10883800FDFDD9F8D0008BE7D9F8D0009D4B017821
:108848001144C829A8BFC82121EAE17101709B78A9
:10885800002B3FF47DAF122019F0E8FDD9F8D000C5
:1088680076E7944B0C989B78417911446429A8BF0A
:10887800642121EAE1714171002B40F02684D9F886
:10888800D00065E7D9F8D0008A4B017A9B7811446B
:10889800C829A8BFC82121EAE1710172002B3FF461
:1088A80057AF0B2019F0C2FDD9F8D00050E7D9F81E
:1088B800D000804BC1799B781144C829A8BFC82132
:1088C80021EAE171C171002B3FF442AF0A2019F08F
:1088D800ADFDD9F8D0003BE7D9F8D000754B8179C8
:1088E8009B781144C829A8BFC82121EAE171817188
:1088F800002B3FF42DAF092019F098FDD9F8D000CE
:1089080026E7D9F8D0006B4B417993F802E011447F
:10891800C829A8BFC82121EAE1714171BEF1000F41
:1089280040F09583112F7FF462AF11E7D9F8D0009A
:10893800604B017993F802E01144C829A8BFC82107
:1089480021EAE1710171BEF1000F40F0A083102F00
:108958007FF461AFFCE60C99564B0F790D931744E1
:10896800642FA8BF642727EAE7770F7119F078FD0D
:108978000D9B9B78002B82D00320394619F056FDB9
:10898800D9F8D000E4E60C984A4B01781144FA294A
:10899800A8BFFA2121EAE17101709B78002B3FF40E
:1089A8006EAF012019F042FDD9F8D000D0E60C983E
:1089B800404B817811446429A8BF642121EAE17100
:1089C80081709B78002B3FF45AAF022019F02EFDDE
:1089D800D9F8D000BCE60C98364BC1799B78114485
:1089E80081F30801C171002B3FF449AF052019F04C
:1089F8001DFDD9F8D000ABE60C982E4B817993F881
:108A080002E011446429A8BF642121EAE17181715F
:108A1800BEF1000F40F025830D2F7FF423AF2EE722
:108A2800D9F8D000234BC17893F802E01144C82943
:108A3800A8BFC82121EAE171C170BEF1000F40F062
:108A48001C830F2F7FF4FBAE82E60C98194B4178FC
:108A58001144B1F5967FA8BF4FF4967121EAE171F0
:108A680041709B78002B3FF40AAF152019F0DEFC0B
:108A7800D9F8D0006CE61049D1F800E04200BEF108
:108A8800000F08D0171803EB87079EF801E07F78DE
:108A98007745BEF40DAA1044084F094A03EB80033A
:108AA80000200B6038801060FEF702BA129AFFF7B8
:108AB800B7BB00BF6A3E002004260020EC26002039
:108AC800F026002004999B7831F91220B2F5617FD5
:108AD8004FF4966191FBF3F3C0F2E68040F6330160
:108AE8009142A8BF11460C2FA1F5617191FBF3F1DA
:108AF80000F00182182F7FF4B5AAC9B2C8290B4625
:108B0800A8BFC823D9F8D020D77DD8B2B8423FF43F
:108B1800A9AADF1BC14BD07548BF0737FF109B7848
:108B28000137FFB23BB9002F3FF49CAA384625F025
:108B38005FFDFFF797BA182019F078FCF3E7B84AF9
:108B4800B84B099210461A68B7494FF47A73B3FBC9
:108B5800F2F3C3EB431203EB82030268DB00560710
:108B6800A1F8A8307EF5ACA8B04BB14D0A221A8006
:108B7800B04B0A93FEF7A7B8AF49096811F4003162
:108B880040F09D81AD4B08465D5C0F2D01F10C0155
:108B98006DD001301828F7D1FA3A0023A4F89020B4
:108BA80084F89230FEF78AB8B4EEE77AF1EE10FA5C
:108BB80040F3D881DFEDA25A9FEDA26A01E0F0EE02
:108BC800676AF4EEC66AF1EE10FA76EEE57AF6DC3C
:108BD800DFED9D6AF4EEE67AF1EE10FA40F1B88125
:108BE800DFED975A9FED996A01E0F0EE667AF4EEB0
:108BF800C67AF1EE10FA77EEA56AF6D4DFED947A2C
:108C0800F4EEE76AF1EE10FA40F3BB80DFED917AFB
:108C180077EEE66A66EEA65A9FED8F5A9FED8F6A49
:108C2800DFED8F7AA5EE856A26EEA55AE5EE867AFF
:108C3800E5EE276AFFF775B98A49D1F800E04200E6
:108C4800BEF1000F08D0171803EB87079EF801E064
:108C58007F787745BEF4B3A80244834F834803EB7B
:108C6800820300220B603A800260FEF7A8B87D49B3
:108C78000F68450037B12E1803EB86067F787678A3
:108C8800BE4289D20544784E784803EB8503002517
:108C98000B60358005607FE7754B1B78032B00F070
:108CA80026810022FFF79FB90C2F40F01A81002778
:108CB8003946704B0E915B78BB423FF4D3A9574BB2
:108CC8000D9338460CF03EFA0D9B0E999B781BB11C
:108CD800C9B20C2019F0AAFB0137FFB223E7DFED78
:108CE800667AB4EEE77AF1EE10FA44BFDFED567A11
:108CF80037EEC77AFFF75DB9604A494913604D4BB3
:108D080009914B4D0A93FDF7DEBF5D4A0592FEF7C8
:108D1800E8BE5C4B01220220AEE45B4A069B1E685B
:108D2800136823F004031360089A012306F480569D
:108D380082F82130FEF7A7BF38EE678A534B5449B3
:108D48001870FDEEC87AC9F5FA63CDED047ABDF95D
:108D58001020120381FB0201D217C2EBA1121BB231
:108D680003FB02F343F30F334B4407EE903AF8EE5C
:108D7800E77AC7ED037AFEF7E0B906F48056FEF706
:108D880082BFDFED3D7AF4EEE76AF1EE10FA44BFF8
:108D9800DFED2D7A77EEE66A3CE70023BB2A1493D1
:108DA80000F00A81B72A00F00381BE2A00F0D880BB
:108DB800BD2A7FF498AC4FF6FE71364A1848D6891A
:108DC8000990908933440144D381918124F01CFB9C
:108DD800F8F746F824F000FBFBF73EF9012025F0F0
:108DE80007FCB4F89030134A0A92FA3B0022A4F820
:108DF800903084F89220FDF766BF274A084B099304
:108E080013780B4D43F0040313700A4B0A93FDF7D4
:108E18005ABF224B022203202EE400BF6A3E0020E4
:108E28002468002010570020985400202A9300201E
:108E38008068002088680020F0310020AC580308C2
:108E4800DB0FC940E4CB1641DB0F49C0E4CB16C1A8
:108E5800DB0FC93FDB0F494092E741B99730083C27
:108E680015A82ABE04260020EC260020F0260020A3
:108E78007C3800201C620020DB0FC9BF04300020B2
:108E880030740020723500207C6800208426002081
:108E9800D34D621090460020683E0020C035002067
:108EA80024F0B2FAF7F7DCFF24F096FAFBF7D4F8CF
:108EB800012025F09DFB94F88E20FFF77AB98649AA
:108EC8000978032947D019465CE6834B1B78032BA6
:108ED8007EF472AD25F08AFAFDF771BF1A46FEF7E7
:108EE80029BB182F7FF4BEA800210B460AE625F0FF
:108EF8007DFAFDF7DDBFCFB2DBE608221346FEF7A9
:108F080019BB01221346FEF715BB03221346FEF7D1
:108F180011BB02221346FEF70DBB07221346FEF7CC
:108F280009BB06221346FEF705BB05221346FEF7CA
:108F380001BB04221346FEF7FDBA684B684A099242
:108F48004FF4C8721A80674B674D0A93FDF7BBBE92
:108F5800F0EE676A52E625F049FAB4F990201BE66C
:108F680002212AE7F0EE667A32E6F0EE477AFEF75B
:108F7800FEBF002D3DF4F3AD5C4C94F88D30002B12
:108F88003DF41EAE25F032FA002384F88D30FDF74B
:108F980017BEB0EE677AFFF700B8514B0993514BF3
:108FA80084F8941084F895004F4D0A93FEF773BD2A
:108FB80019464FF6FE7300E719460223FDE64FF403
:108FC800FA6102200BF0E8FFFFF7ABBB002101209C
:108FD8000BF0E2FFB4F89030414A0992963B414ABF
:108FE800A4F8903000230A9284F89230FDF76BBE03
:108FF80000210846ECE7FF21002026F055F894F8F8
:109008008E20FFF77CBB0121002026F04DF894F854
:109018008E20FFF771BB0021FF2026F045F894F859
:109028008E20FFF766BB0021012026F03DF894F85A
:109038008E20FFF75BBB0B20FDF73EBE002104200E
:10904800C6E700210320C3E700210220C0E7112062
:109058000E930D9219F0EAF9D9F8D0000E9B0D9AEB
:1090680060E40D200E930D9219F0E0F90E9B0D9A15
:10907800D2E4172019F0DAF901E40F200E930D92CB
:1090880019F0D4F9D9F8D0000E9B0D9AD9E4102024
:109098000E930D9219F0CAF9D9F8D0000E9B0D9ACB
:1090A80055E4002B3FF468AF1149124A09684FF4A0
:1090B8007A7000FB031313605EE70C4C0AF0B2FDF4
:1090C800002384F88D30FDF77BBD0E2019F0AEF932
:1090D800D9F8D000FFF73CBB7C3800202C93002047
:1090E800246800208868002080680020AC230020C5
:1090F800B0620020003000202DE9F047C74C6368BB
:1091080020469847002800F0C380C54B1B780122F1
:10911800042B84F83C2000F0BD80B4F91610B4F993
:109128001820B4F91A3021636263A363BD4B1B880E
:10913800002B69D0BC4DD4ED0C7AD5ED004A95EDE5
:10914800050A95ED015A95ED067AD5ED035A95ED88
:10915800026AF8EEE76AD5ED047AA4EEA60AA5EE4F
:10916800267A67EEC07AA5EEC07AE6EE267A85ED15
:10917800057AC5ED067A2AF093FFD4ED0D6AD5ED90
:10918800094A95ED0E0A95ED0A5A95ED0F7AD5ED37
:109198000D7AD5ED0C5A95ED0B6A2063F8EEE66A68
:1091A800A4EEA60AA5EE267A67EEC07AA5EEC07AE6
:1091B800E6EE267A85ED0E7AC5ED0F7A2AF070FF75
:1091C800D4ED0E6AD5ED124A95ED170A95ED135AAE
:1091D80095ED187AD5ED167AD5ED155A95ED146AF0
:1091E8006063F8EEE66AA6EEA40AA6EE857A67EE54
:1091F800C07AA0EE657AE6EE867A85ED177AC5ED37
:10920800187A2AF04DFFA063884FA17F884813F091
:10921800CFF93B88002B40F08480864ED6F8E0508A
:10922800854B1B685B0743D4B5F90070216B636BF2
:10923800A06B824A824E92ED026AD2ED006AD2EDAC
:10924800015AC91B2163B5F90270DB1B6363B5F9C9
:1092580004703568C01B07EE900AB8EEE75A07EEAF
:10926800901AB8EEE77A07EE903AF8EEE77A36EE1B
:10927800056A36EE877A77EEA57A0135A06382ED26
:10928800026A82ED007AC2ED017A3560BDE8F087A6
:10929800BDE8F0876B4BB4F91600B4F91810B4F9AF
:1092A8001A2018802063598061639A80A2633DE781
:1092B800B6F89820322A00F08880002A66D196F8FD
:1092C8009530002BB0D06048D6F8FC205F4980FB71
:1092D8000273D217C2EB23122A80D6F8002180FB32
:1092E8000273D217C2EB23126A80D6F80431A78A18
:1092F80080FB0302DB17C3EB2213DB1BAB800023CD
:10930800CB6086F8953024F07FF8F7F7A9FD24F0B4
:1093180063F8FAF7A1FE012025F06AF9D6F8E050C3
:1093280082E7444E226BD6F8E050B3F5C87F4FF081
:10933800000323632B80398818BFD6F8E400B7F8F8
:10934800008008BF0020B1F5C87F18BFD6F8E83004
:10935800616B02440B440020B8F5C87F6063C6F80F
:10936800E420C6F8E830688052D0D4F838E0D6F85F
:10937800EC10A0637144B8F1010FA880C6F8EC1096
:1093880068D008F1FF38A7F8008049E7D6F8FC0054
:10939800236B00210344C6F8FC3021632980D6F8EA
:1093A8000001636B61630344C6F800316980A36BF5
:1093B800D6F80401A1630344012AC6F80431A98040
:1093C80075D0013AA6F8982079E72B8820491F48DC
:1093D800276BA6F8F0300023B5F802E0B5F804C012
:1093E800C0684B608B602363C6F8FC702B80616B90
:1093F800C6F8001163636B80A16BC6F80411A36300
:10940800A6F8F2E0A6F8F4C0C6F8F800AB80D8E7F2
:10941800A36BC6F8EC30A063A880B2E738680020D8
:10942800E864002030400020344000202C930020C5
:1094380068680020AC2300202057002088470020BF
:1094480084470020EC6400201F85EB5190460020E3
:10945800A8240020DFF804C1DFF8F0E0C8328CFB54
:1094680002A9C833D217C2EBE9128CFB03A9DB1798
:10947800C3EBE913C8316B802A808CFB013CA28ABC
:10948800CB17C3EBEC139B1AAB80CEF80C0023F080
:10949800BBFFF7F7E5FC23F09FFFFAF7DDFD404639
:1094A80025F0A6F8B7F80080D6F8E05069E7254B14
:1094B80086F89A101B6886F8942013F4003334D188
:1094C80019462148475C0B2F01F10C0110D00133DC
:1094D800182BF7D1B6F8F0101C4B2980B6F8F270AB
:1094E800B6F8F400D6F8F8106F80A880D96068E75D
:1094F800174FD7F800C05900BCF1000F09D001EB95
:10950800030E00EB8E0E9CF801C09EF801E0E645C4
:10951800E0D20B44DFF848E00E4900EB830000235B
:109528003860AEF800300B60D4E70B4B1B78032B88
:1095380001D00B46C5E724F059FFD6F8E050B6F83D
:109548009820C7E7F0310020AC5803089046002067
:1095580004260020F02600207C3800201F85EB51CF
:10956800EC2600202DE9F0478C4B1B78DB070746DB
:1095780044D58B4B8B4D1C788B4E012C59D01CD36A
:10958800022C07D189498A4A09881288914201D94F
:1095980001241C70EB7AE3B12B89D3B1854B1B787E
:1095A800BBB108F0E5FB002800F09B802B7B8342D1
:1095B8002CBF0121002131700CE07C497E4A0988CA
:1095C80010886A7B801A8842E2DAEB7A0024002B42
:1095D800E2D131782A79632A06D8022C774E00F036
:1095E800BA803378002B5DD1754AAB7A8C4238BF8C
:1095F8000C461470002B4CD1BDE8F0876B4B694DBD
:1096080019885B88E878CB1A83EAE3728142A2EB77
:10961800E3721DD32B788B421AD3614B1C78E01E62
:10962800012861D96749097802294FD0012C5E4E7B
:10963800A5D15F4A5D491288687B0988121A914250
:1096480039DD5D4A12888A42A4D200241C70A1E741
:10965800B1EB400FE1DC524B1C78E11E012940F2CE
:109668009480022ADEDC57494F4E0878DFF844819F
:10967800DFF844C1DFF838E1002103240228347000
:109688001C7088F80010ACF80010AEF8001081D1FA
:109698001FE0012C71D0022C0BD10720BDE8F04748
:1096A80024F0C0BE7068381A474B984258DD727073
:1096B8009AE7BDE8F08702241C706BE7022AD2DD26
:1096C8004049097802294FF0040464D13949364EDB
:1096D80009783E48022ACCBF00220122C28081803C
:1096E8004BE70221317075E7022A9BDC95F800C030
:1096F80091FBFCFC0CF1010CBCF1080FDFF8B4A0E5
:10970800304EA87895F801E096F800802A4CDFF8EA
:10971800A090254EA8BF4FF0080C8AF800C01FFA89
:109728008CFA10FB0AF01EFB0AFE80B2DFF88CA050
:109738002080A9F800E000244FF0640EB8F1020F71
:1097480034701C70CAF804408AF801E07FF439AF1D
:109758000FFA8CF1BDE73078A0B901237760337038
:10976800C2F164021A4B00FB02F083FB0023C0170E
:10977800A0EBA3506430707036E70820BDE8F047CE
:1097880024F050BE7368F81A8EE7032C96D10D4961
:10979800097802299AD0044EFCE600BF097100201E
:1097A800A827002014680020B8270020046600209D
:1097B800AC27002012680020AA270020B02700202C
:1097C8007C380020E86400207F969800EC64002034
:1097D8006BCA5F6B2DE9F04FB0F908500D81EDB2FF
:1097E800442D93B00C46174600F06D82064642D9C8
:1097F800812D00F0AB8200F29580542D00F0C980D5
:1098080040F2FC816E2D00F02C82802D40F01D81ED
:10981800994B93F8009009F1020919F0FF0900F03B
:109828009580964B964F974EDFF88CA2994403F19A
:1098380001080A2516E0322D01F03884A5F13C0014
:10984800C0B2132841F23C8400232268511C2160D5
:1098580015702268C14502F101012160137075D0AD
:1098680018F8015B0A2DE6D1BAF80030FF2BA8BF23
:10987800FF23DBB2E9E7052D00F013821ED8022D85
:109888007FD040F2A881032D00F0E081042D40F044
:10989800DC802A467C492046F7F7ACFD00212046AB
:1098A800F7F7D6FD22680221531C012523602846BC
:1098B8002B461170638113B0BDE8F08F242D5ED064
:1098C80040F24081282D00F00682382D40F0BD80FE
:1098D8000A686E4B0125511C21601570226805210C
:1098E80050192060117022680A21501920601170E7
:1098F80022680021501920601170226819785019C7
:1099080020601170226859785019206011702268FF
:109918009978531923602B4611702846638113B038
:10992800BDE8F08FA02D18D040F22A81B82D00F0A4
:109938000B82FE2D40F08980554D05F1080635F85B
:10994800021B2046F7F784FDAE42F8D101252B46CD
:109958002846638113B0BDE8F08F4E4B084619685E
:10996800F7F75FFD4C4B20461968F7F75AFD4B4B4C
:10997800196820460125F7F754FD2B46E8E7484BC0
:10998800F6E70422474920460125F7F733FD2B4621
:10999800C3E70B68444A454F581C112120601970D1
:1099A80023681278591C21601A70236897F855208B
:1099B800591C21601A70236897F85420591C21609B
:1099C8001A70B7F850102046F7F742FD23680022B6
:1099D800591C21601A7023682822591C21601A70AA
:1099E800B7F852102046F7F733FDBD1E07F14E06B3
:1099F80035F8021F2046F7F72BFDB542F8D122684B
:109A08002B4B0D21501C20605D181170226813F833
:109A1800011F501C9D4220601170F7D1236802225B
:109A2800591C21601A70B7F856102046F7F710FD38
:109A3800B7F858102046F7F70BFD0125B7F85A106C
:109A48002046F7F705FD2B4667E72146284606F02E
:109A5800ADFD014600287FF479AF742D00F0EC804D
:109A6800772D2BD1336872689A4240F0DA81114A17
:109A7800204624F06FFE69E7C9640020F852030805
:109A88006766666658270020226200200F3500208E
:109A9800EC640020ACF7FF1FB0F7FF1FB4F7FF1FFF
:109AA800C0360020807C0308C061002010380020E8
:109AB8006D380020A9DA020880270020F52D00F073
:109AC800DD8170683768A5F12103C21B362B00F2CF
:109AD8006583DFE813F03D026303630363036303F5
:109AE8006303630363035C02630363036303630346
:109AF800630363036303630363036303630363032E
:109B08006303630363032D02630363036303630354
:109B1800630363036303630363036303630363030D
:109B280063036303630363036303630363036303FD
:109B3800630363036303630363030E036303E802BE
:109B480063037102202D80D10B68B84D591C6A78C7
:109B580021601A7023682A78591C21601A702368BA
:109B6800AA78591C21601A7029892046F7F770FCD9
:109B780023686A79591C21601A702268A97993E6CA
:109B8800822D7FF462AF0B68A94AAA4D1178A74AC3
:109B9800581C2060197011892046F7F759FCA64B0C
:109BA80022681B88FF2B02F10101A8BFFF23216057
:109BB8001370A96881F3100189B22046F7F748FCB1
:109BC800296801F30F0189B22046F7F741FC9B4B46
:109BD8002268197868E6012D7FF437AF0B680022F8
:109BE800591C21601A7023685A1C22601D70226853
:109BF8002521531C23602B4611708EE6522D7FF4CD
:109C080024AF0A688E4E531C0321236006F10C070B
:109C180033461170062501202268511C21601070FE
:109C28002268BB4202F101012160157000F0D68064
:109C38009879DD790633EFE7336872689A4240F025
:109C4800EC80804A204624F085FD7FE60B685A1C8C
:109C58000A601D700B685A1C0A601D700A68002192
:109C680022E6754B0A681B88724DFF2BA8BFFF239D
:109C7800511C21601370A96881F3100189B2204634
:109C8800F7F7E6FB704B20461988F7F7E1FB2968E0
:109C980001F30F0189B220460125F7F7D9FB2B46BE
:109CA8003BE60B2269492046F7F7A4FB08226849DE
:109CB8002046F7F79FFB0125072266492046F7F75C
:109CC80099FB2B4629E6002A3FF440AE624B13600D
:109CD80001252B4621E60B68DFF89C815F4E591C55
:109CE800022221601A70236806275A1C22601F70FE
:109CF80023680A22591C21601A70236801255A1901
:109D080022601D70B8F800102046F7F7A1FBB8F8DC
:109D180002102046F7F79CFB23685A1922601F702F
:109D280023685022591921601A7023680022591992
:109D380021601A7031882046F7F78AFB718820461F
:109D4800F7F786FB2B46E8E5454B11E6454B1E78B1
:109D5800033616F0FF063FF4F9AD434B434F1E445C
:109D680003F101094FF00A0820E0B8F1500F01F0A3
:109D7800A481B8F1320F01F0B981A8F13C00C0B25A
:109D8800132841F2B7810025294623685A1C22600E
:109D9800204683F80080F7F75BFB29462046F7F753
:109DA80057FB4E453FF4D2AD19F8018BB8F10A0FB5
:109DB800DBD12F4B9D68196805EB85054FF6FF73BE
:109DC8006D009D42A8BF1D469942A8BF194625EAC5
:109DD800E57521EAE171ADB289B2D6E7254B216874
:109DE8001A78481C20600A70002A3FF4AFAD013A87
:109DF800D2B202EB420206EB42025278002A3FF44A
:109E0800A5AD0132D5180133226813F8011F501C83
:109E1800AB4220601170F7D198E55A1C326019786E
:109E28000FE75A1C3260197821E600BF1468002039
:109E380012680020F0650020046600207C380020AD
:109E48007053030809DB0208183E0020887C0308C9
:109E5800947C0308A07C0308ED0201084027002039
:109E6800F0310020C964002008530308502700205F
:109E78000C270020B45E00208046002033687268FA
:109E88009A4241F05081B64BFF221A704FF00009F8
:109E9800B44D09F08BFE49462022B34885F800905E
:109EA8002BF0BBF88DF808909DF80830072B01F2CD
:109EB800EA81DFF8DC82AC4E4A469DF8083003EBB5
:109EC800430308EBC3035B7CE3B19DF8083003EB65
:109ED800430308EBC30320215B699BB19DF808305D
:109EE80003EB430308EBC303586946F82200FCF769
:109EF80061F82B7856F82300FCF71EFA2A7801320D
:109F0800D2B22A709DF808300133DBB28DF80830E0
:109F18009DF80830072BD0D92368591C21601A7086
:109F2800002F3FF413AD914B3B6001252B46F4E421
:109F38007B1C33603B780A2B01F023813046F7F70E
:109F480054FA3046F7F751FA3046F7F74EFAFDE47F
:109F58003B467A1C3260864D13F8022B6A703360D8
:109F68007B782B70FB1C3360BB78AB703046F7F7FF
:109F780031FA33682881591C1A46316012F8021BDD
:109F8800697132605B78AB7101252B46C5E47B1C97
:109F980033603B780A2B01F0EE80502B40F08F8520
:109FA8003046F7F717FA734F38803046F7F712FA4A
:109FB800012578802B46B0E47B1C3846336010F8C6
:109FC800375B0DF107020133336013F8011C02F807
:109FD800011F9842F7D1DFF8BCA19AF80070002F52
:109FE800FDD1DFF8B4B16448634E4FF00108042195
:109FF8008AF80080F7F7ECFDDBF80000FCF796F92B
:10A008005E4B3946304683F80080F7F795FD3946B0
:10A018003046F7F791FD09213046F7F78DFD2946BF
:10A028003046F7F789FD0DF1080845460DF13E0960
:10A03800A5EB0807FFB20A213046F7F77DFD394640
:10A048003046F7F779FD15F8017B0B213046F7F715
:10A0580073FD39463046F7F76FFD0020FBF746FDE4
:10A06800A945E5D1444808210546F7F765FDA02133
:10A078002846F7F761FDA0212846F7F75DFD002186
:10A088002846F7F759FD10F02006F4D1DBF8000058
:10A09800FCF752F9012502213748F7F799FD8AF8AC
:10A0A80000602B4639E47B1C336097F80080B8F1D8
:10A0B800FF0F01F0B080B8F1FE0F01F07380304659
:10A0C800F7F788F996E80C009B1A002B07DD531C5C
:10A0D800336013781BB9B8F10C0F41F2C980B8F19D
:10A0E800270F00F2DC82264B012523F818002B46A7
:10A0F80013E47B1C33603878032800F2D082431EB7
:10A10800204D2149DBB203EB430305EB4303087001
:10A118005D7800283FF41AAC531EDBB2AB4240F026
:10A12800BE820022C1F80620C1F802208A725BB103
:10A13800581C336808444A1C0133336013F8011C67
:10A1480002F8011F9042F7D1104B1B78002B3FF407
:10A15800FDAB01251DF052FE2B46FFF7DEBB00BF0D
:10A16800B82400202F33002038720020095F01082E
:10A17800146800204027002000300140254E0020B0
:10A188001038002070530308B45E0020B92700205F
:10A19800605800201D4E0020B86100200B3DEF2DB7
:10A1A80000F27D8201A353F825F000BFA7AD000897
:10A1B800A7A60008A7A60008A7A60008A7A6000843
:10A1C800A7A60008A7A60008A7A60008A7A6000833
:10A1D800A7A60008A7A60008A7A60008A7A6000823
:10A1E800A7A60008A7A60008A7A60008A7A6000813
:10A1F800A7A60008A7A60008A7A60008A7A6000803
:10A20800A7A60008A7A60008A7A6000837AD00085B
:10A21800A7A600081DAD0008A7A60008FBAC00080B
:10A22800A7A60008A7A60008A7A60008D3AC0008A0
:10A23800A7A6000879AC0008A7A60008F5AB000897
:10A24800A7A60008CFAB0008A7A60008A3AB000884
:10A25800A7A600084FAB0008A7A6000803AB000894
:10A26800A7A60008A7A60008A7A60008A7A6000892
:10A2780055990008A7A60008D7AA0008A7A60008AD
:10A28800A7A60008B5AB0008A7A600087DAA000885
:10A29800A7A60008A7A60008A7A60008A7A6000862
:10A2A800A7A60008A7A60008A7A60008A7A6000852
:10A2B8003DAA0008A7A60008EFA90008A7A600085D
:10A2C800A7A6000849B00008A7A60008A7A6000886
:10A2D800A7A60008A7A60008A7A60008A7A6000822
:10A2E800A7A6000871AF0008A7A60008D5AF000808
:10A2F800A7A60008CFAE0008A7A600083FAE000832
:10A30800A7A6000817AE0008F9AD0008DDAD0008E3
:10A31800A7A60008A7A60008A7A60008A7A60008E1
:10A32800A7A60008A7A60008A7A60008A7A60008D1
:10A33800A7A60008A7A60008A7A60008A7A60008C1
:10A34800A7A60008A7A60008A7A60008A7A60008B1
:10A35800A7A60008A7A60008A7A60008A7A60008A1
:10A36800A7A60008A7A60008A7A60008A7A6000891
:10A37800A7A60008A7A60008A7A60008A7A6000881
:10A38800A7A60008A7A60008A7A60008A7A6000871
:10A39800A7A60008A7A60008A7A60008A7A6000861
:10A3A800A7A60008A7A60008A7A60008A7A6000851
:10A3B800A7A60008A7A60008A7A60008A7A6000841
:10A3C800A7A60008A7A60008A7A60008A7A6000831
:10A3D800A7A60008A7A60008A7A60008A7A6000821
:10A3E800A7A60008A7A60008A7A60008A7A6000811
:10A3F800A7A60008A7A60008A7A60008A7A6000801
:10A40800A7A60008A7A60008A7A60008A7A60008F0
:10A41800A7A60008A7A60008A7A60008A7A60008E0
:10A42800A7A60008A7A60008A7A60008A7A60008D0
:10A43800A7A60008A7A60008A7A60008A7A60008C0
:10A44800A7A60008A7A60008A7A60008A7A60008B0
:10A45800A7A60008A7A60008A7A600088BB00008B2
:10A46800A7A60008D9A90008AFA90008A7A6000850
:10A47800A7A60008A7A60008A7A60008A7A6000880
:10A48800A7A60008A7A60008A7A60008A7A6000870
:10A49800A7A60008A7A60008A7A60008A7A6000860
:10A4A80055A90008A7A600081DA90008A7A6000826
:10A4B80081A8000823A8000807A80008A7A6000884
:10A4C800EDA70008A7A60008C5A70008A7A60008CA
:10A4D8006BA70008A7A600083DA70008A7A60008C4
:10A4E800A7A600081BA70008EDA60008D9A6000823
:10A4F800B1A6000889A6000867A60008A7A6000854
:10A50800A7A60008A7A60008A7A60008A7A60008EF
:10A51800A7A60008A7A60008A7A60008A7A60008DF
:10A52800A7A60008A7A60008A7A60008A7A60008CF
:10A53800A7A60008A7A60008A7A600084DA6000819
:10A54800A7A60008A7A60008F5A50008A7A6000862
:10A55800A7A60008A7A600088FA50008A7A60008B8
:10A56800A7A60008A7A6000875A50008B14B1B7888
:10A57800DB0700F194800125F9F792FBF9F76CFDF0
:10A588002B46FFF7CAB93046F6F724FF3368ADF813
:10A5980008001A46591C316012F8021B32608DF807
:10A5A8000A105A788DF80B20DA1C32609A788DF8E8
:10A5B8000C201A1D3260DA788DF80D205A1D326091
:10A5C8001B798DF80E3002A80023ADF81030F6F78D
:10A5D8005DFE994A994B1268801A4FF0010561F1A6
:10A5E8000001C3E904012B46FFF797B97B1C3360D0
:10A5F8003B780F2B53D8BA1C3260C3EBC303904A85
:10A608007978D154F91C31601344BA785A703A1DDC
:10A618003260FA789A707A1D32603A79DA70BA1D27
:10A6280032607A791A71FA1D3260BA795A7107F173
:10A6380008023260FA799A71012519F0D7FA2B4687
:10A64800FFF76BB93046F6F7C5FE7E4FF881304606
:10A65800F6F7C0FE0125B8812B46FFF75EB93046F4
:10A66800F6F7B8FE784F38823046F6F7B3FE7882B0
:10A678003046F6F7AFFE0125B8822B46FFF74DB9F5
:10A688003B467A1C326013F8020B3360FB1C797866
:10A698003360BA781AF0BEFB00287FF457A94FF050
:10A6A800FF352B46FFF739B93B467A1C3260674ABB
:10A6B80013F8021B11703360624A7B789370FB1C9D
:10A6C8003360634BBA789A7001252B46FFF725B99A
:10A6D800604B614918684E22012529F00BFB2B4677
:10A6E800FFF71BB93A467B1C33605C4B12F8021B20
:10A6F800197032607A785A70FA1C3260BA789A7097
:10A708003046F6F767FE564B0125D8802B46FFF7F3
:10A7180004B93046F6F75EFE514F38803046F6F7FA
:10A7280059FE78803046F6F755FE0125B8802B464D
:10A73800FFF7F3B8DFF8388198F80030002B3FF4C2
:10A7480005A9484F00253046F6F744FE17F010F8E3
:10A7580098F80030A7EC010A01359D42F3DBFFF7BA
:10A76800F5B80D2A9BD17B1C33603D78072D96D810
:10A77800DFF8008130460C27F6F72CFE07FB05F7BB
:10A7880008EB0705A8803046F6F724FEE880304637
:10A79800F6F720FE336828811A46591C316012F8F2
:10A7A800021BA97232605B78EB723046F6F7FBFD4C
:10A7B800012548F807002B46FFF7AFB87B1C33602C
:10A7C8003878060600F1A4851A4B1B78DD073FF59B
:10A7D800BDA8032828BF00200125F9F745FA2B4614
:10A7E800FFF79BB8134B1B78D8073FF5AFA8012597
:10A7F800F9F7FCFDF9F730FC2B46FFF78EB80D4B47
:10A808001B78DA073FF5A2A8174A1378012543F009
:10A81800040313702B46FFF780B8064B1B78D90743
:10A828003FF594A8114B4FF4C87201251A802B46A6
:10A83800FFF773B809710020B0620020B824002027
:10A848000431002090460020205900208454002024
:10A85800A046002084680020CC70030888460020A9
:10A868007849002078330020683E00202C9300208F
:10A87800C964002044300020092A7FF710AFDFF8B0
:10A88800E8833B467A1CD8F80050326013F8022B54
:10A898002A7033607B78AB70FB1C3360BB78642B09
:10A8A800A8BF64233A1D6B713260FB78642BA8BF84
:10A8B80064237A1DAB7132603B79EB71BB1D336049
:10A8C8007B79642BA8BF6423FA1D2B723260BB7995
:10A8D800EB7007F108033360FB792B713046F6F70C
:10A8E80079FD726833686881D11A00290CDD591C1A
:10A8F800D8F800003160521A002A1978417203DD35
:10A908009A1C32605B784370012517F0A9FD2B462D
:10A91800FFF703B8C24B1868FB1C02462137991E83
:10A92800316013F8031C1170591E316013F8021CB2
:10A938005170336013F8011C917003339F4202F188
:10A948000302ECD116F0E4FDFFF700B8C2F34705A7
:10A95800122D3FF6A4AEB5B112AB0DF1060803EB0C
:10A968004507C146423F3046F6F734FD29F8020F45
:10A978004F45F8D1AB4B38F8022F23F8022FC845C2
:10A98800F9D1112D09D8A84A6B00023B13440021C4
:10A99800223223F8021F9A42FBD1A44A01231D4602
:10A9A8001370FEF7BABF7B1CA14933600A783B7865
:10A9B800002A40F0898404220A709E4A9B00138072
:10A9C800FAF710FE9C4B012598612B46FEF7A5BFB0
:10A9D8009A4F002330463B60F6F7E5FC01253860C6
:10A9E8002B46FEF79ABF7B1C336097F80080B8F1BE
:10A9F800110F3FF654AEBB1C3360914D7B7805F8C0
:10AA080018303046F6F7E6FC40F6CA039842A8BF6D
:10AA1800184640F2EE23984205EB4801B8BF1846A5
:10AA28000125A0F2EE222B46192092FBF0F24A7083
:10AA3800FEF773BF3B467A1C824D326013F8022B37
:10AA48002A7133607B786B713046F6F7C3FC336844
:10AA580028805A1C32601B78AB713046F6F7BAFC76
:10AA6800336868805A1C32601B78EB7101252B46CD
:10AA7800FEF753BF7B1C3360734B3A78DFF8EC81E9
:10AA88001A700023C8F800303046F6F78CFC32689C
:10AA9800D8F800306D496E4D0343501CC8F800309B
:10AAA800306013780B723046F6F794FC2860304615
:10AAB800F6F790FC68603046F6F78CFCA8603046E4
:10AAC800F6F788FC3046F6F785FCFEF73FBF3B46B5
:10AAD8007A1C32605F4A13F8021B917033607978F0
:10AAE800517083423EF432AFFB1C3360524BBA784C
:10AAF8001A7201252B46FEF710BF0723B2FBF3F3AA
:10AB0800C3EBC301521A7FF4CAADDBB203F1FF3ABB
:10AB18005FFA8AFA002B3EF419AFDFF83CB10AF16C
:10AB2800010A90467B1C336097F900104A4B0025B8
:10AB380093F902208A4203F1080300F046830135A5
:10AB4800062DF5D1ABE57B1C33603B780E2B3FF629
:10AB5800A6ADBA1C3260787803283FF6A0AD3F490D
:10AB6800062202FB03F28B18FD1C58713560B87879
:10AB780088543A1D3260FA785A707A1D32603A79F0
:10AB88009A70BA1D32607A79DA70FA1D3260BA7931
:10AB98001A7101252B46FEF7C0BE7B1C33602B4B78
:10ABA8003A785A7501252B46FEF7B7BE2C4B07F1AC
:10ABB80008020137376017F8011C03F8011FBA4271
:10ABC800F7D1FEF7C3BE7B1C33603D781F2D3FF6DF
:10ABD80066AD052A7FF463AD3046F6F7E4FB214BFA
:10ABE80043F825001AF080F9FEF7B0BE1D4D05F1B7
:10ABF80040073046F6F7EEFB3368A5F88000591C8D
:10AC08001A46316012F8021B85F8821032605B78B0
:10AC180085F883300435AF42EBD1FEF797BE00BF0D
:10AC280084680020A2710020A4710020C87100204F
:10AC3800EE6A0020183E0020B8240020F0310020E1
:10AC4800BC73002094490020544400203074002034
:10AC5800902F0020B04600202C5E0020FC31002000
:10AC68002F7400206C39002088680020C03600202E
:10AC78007B1CAF4D33603B782B723046F6F7AAFB4E
:10AC8800A8833046F6F7A6FB28833046F6F7A2FBE2
:10AC980032686883531C33601278EA747268D31A76
:10ACA800032B00F370833368D11A052900F35B8303
:10ACB800D21A002A7EF74AAE5A1C32601B7885F8F1
:10ACC800213001252B46FEF728BE7B1C3360994AAC
:10ACD80039781170C01A00287EF738AEBB1C336073
:10ACE8007B78003318BF0123012553702B46FEF7EC
:10ACF80014BE3046F6F76EFB8F4F38603046F6F7D5
:10AD080069FB78603046F6F765FB0125B8602B468D
:10AD1800FEF703BE894F00233B603046F6F743FB3E
:10AD28003B68012503433B602B46FEF7F6BD7B1CC1
:10AD380033603D780191132D3FF6B1ACBB1C3360F5
:10AD4800787823F041FD00283FF4A9AC7C4B0278C9
:10AD580003F82520FA1C326003EB8505BA786A707F
:10AD68003A1D3260FA78AA707A1D32603A79EA7030
:10AD7800019903F1500202E00433934207D0187896
:10AD88000028F9D19D78D8788542F5D201216D4BFC
:10AD980081F00101012519702B46FEF7BEBD6A4BF3
:10ADA800102A4FF0000128BF1022196059609960DD
:10ADB800D9601974002A3EF4C9AD3168013B0A44D0
:10ADC8000131316011F8010C03F8010F8A42F7D103
:10ADD800FEF7BCBD7B1C33603B78002B00F0BA82C9
:10ADE8004FF40040012506F00DFC2B46FEF795BDFB
:10ADF800564B1B7813F001017FF451AC7B1C336078
:10AE0800387801250AF0C8F82B46FEF786BD3B4680
:10AE18007A1C32604E4A13F8021BD17033604D4AD7
:10AE28007B785371FB1C33604B4BBA78DA70012581
:10AE38002B46FEF772BD3046F6F7CCFA3046F6F7E9
:10AE4800C9FA3046F6F7C6FA3046F6F7CEFA33684E
:10AE5800424D1946581C2A68306011F8020B82F8D6
:10AE68002C003160597882F83610D91C31609B78F3
:10AE780082F837303046F6F7B8FA3046F6F7B5FAC2
:10AE88003046F6F7B2FA30462F68F6F7A3FA788715
:10AE980030462F68F6F79EFA336872683887D11AF9
:10AEA80001290ADD591C2A6831601B7882F82E3086
:10AEB8003046F6F79AFA33687268D31A032B00F310
:10AEC800818228683EE57B1C3360244DDFF894803E
:10AED8003B7888F8053030462F68F6F77BFA3884D7
:10AEE80030462F68F6F776FA72683368F883D11A15
:10AEF800072900F31882D11A032900F3EA81D21A2C
:10AF0800002A05DD591C2A6831601B7882F8263032
:10AF1800F9F704F81AF088FB114B1B68002B00F0B6
:10AF280069822868012515F063FF2B46FEF7F5BCFA
:10AF38003074002054440020902F0020C036002098
:10AF4800B0720020EF2000201A3E00200971002076
:10AF58009046002020400020A04600208468002061
:10AF68003C44002084540020C84B1B68002B3EF44E
:10AF7800EDAC1AF067F9FF283EF4E8AC3046F6F776
:10AF880029FA3F2840F22982C14F00253D703368D5
:10AF98007268B880D21A012A7EF7D8AC1A46591CB2
:10AFA800316012F8021BB97012A8326000225D7875
:10AFB80000F8402D1AF036F89DF80830AB423EF400
:10AFC800C5AC28461AF034F9FEF7C0BC3B467A1CDB
:10AFD8003260DFF8EC8213F8022B88F80220336025
:10AFE800AC4A7B781370FB1C3360AB4DBB782B717C
:10AFF8003B1D3360FB78092BA8BF09233046AB7093
:10B00800F6F7E8F9336872682880D11A012905DD56
:10B018003046F6F7DFF933687268E8819A4240F003
:10B02800F481F8F77BFF336872689A423EF48EAC7D
:10B038005A1C32601B78EB7001252B46FEF76DBC5D
:10B04800964B1B78012B3EF681AC7B1C3A4633604D
:10B05800DFF8708212F8023B88F802303260FB1C7D
:10B0680097F801E03360C31A012BB97840F33E81A9
:10B078003046F6F7AFF90125A8F800002B46FEF791
:10B088004CBC3B467A1C326013F8025B3360FB1CF5
:10B0980078783360B978002D00F03481012D7EF482
:10B0A80055AC0AF033F82B46FEF737BC3388FF2B34
:10B0B800A8BFFF23DBB2FEF7C8BB794BFEF77ABE09
:10B0C80020F010F900283EF4BFAB03780A2B28D8EB
:10B0D800B0F9023087FB0312DB17C3EBA2039BB264
:10B0E800FF2BA8BFFF23DBB2FEF7AFBB97E8220018
:10B0F800FEF762BE20F0F6F800283EF444AE03786E
:10B108000A2B3EF640AEB0F90430B0F9061003EB56
:10B11800830383F3500521EAE171ADB289B2FEF7EA
:10B1280034BE0023DFE75A1C194632605D4811F827
:10B13800022B027031605B784370042A06D9FF2A1B
:10B148003EF4A4AE22680021FEF7AEBB564909784A
:10B15800994203D8022AF5D1FF2BF3D123680125A0
:10B168005A1922601D70002F3EF4F0AB4F4B3B6024
:10B178002B46FEF7D2BB3046F6F72CF94C4FFEF7BC
:10B1880013BFBB1C33604B4B7A781A70FA1C3260C1
:10B19800BA785A703A1D3260FA789A7001252B46AF
:10B1A800FEF7BBBBBB1C33607D78022D3FF677AA48
:10B1B8003046F6F70FF9404B03EB45034FF0FF35E8
:10B1C800A3F856002B46FEF7A8BB0BEBC509304683
:10B1D80089F80210F6F7FEF833682BF835001A469E
:10B1E800591C316012F8021B89F8031032605A7832
:10B1F80089F80420DA1C32609A7889F806201F1D25
:10B20800376008F10108DB7889F80530C2457FF41A
:10B2180089ACFEF79BBBBB1C3360284B7A781A704D
:10B22800FB1C3360DFF89080BB7888F855303B1DF5
:10B238003360FB7888F854303046F6F7CBF8A8F836
:10B2480050003046F6F7C6F83046F6F7C3F896E8E9
:10B258000C009B1A012BA8F852007EF777AB3046FA
:10B26800F6F7B8F80125A8F85A002B46FEF755BBA3
:10B27800114B0030984418BF0120012588F85E0062
:10B288002B46FEF74ABB4A46FEF746BE0C71002025
:10B2980010710020844600202059002066360020C6
:10B2A80044270020B8240020C964002005030108B1
:10B2B800804600200F35002010380020C061002093
:10B2C800845400206A3E0020042A7EF43FABFFF736
:10B2D80074BB3046F6F77EF8A8F80E003046F6F74D
:10B2E80079F833687268A8F8100008E64B4B1A889A
:10B2F800012512FB0EF22B4692FBF1F2A8F8002072
:10B30800FEF70BBB012515F091FF2B46FEF705BB99
:10B3180000F07F00032828BF0020012509F012FF54
:10B328002B46FEF7FABA3046F6F754F8A8F80A00A2
:10B338003046F6F74FF8A8F80C0030462F68F6F7B5
:10B3480049F8788430462F68F6F744F8336872680D
:10B35800B884D0E5324A1368012523F4004313600A
:10B368002B46FEF7DABA5A1C32601B78EB7230466D
:10B37800F6F719F83368E8605A1C32601B782B74AA
:10B388003368726894E43046F6F724F8A8843046A7
:10B39800F6F720F833687268E884D11A03297FF732
:10B3A80083AC1A46591C316012F8021BA977326027
:10B3B8005B7885F820303046F6F70CF83368726809
:10B3C800688471E430462F68F6F704F878863046CA
:10B3D8002E68F5F7FFFFB08673E5C50800F0070390
:10B3E80001350133EDB20F4F284619467B701FF027
:10B3F8001FFFCBE50C480D490D4A0E4B0360012594
:10B408000B6013602B46FEF788BA5A1C32601B7813
:10B41800003318BF012388F8073002E66C46002085
:10B428007C68002010710020B447002008480020E4
:10B43800704800206B0500082DE9F04F2DED0E8BAC
:10B44800DFF8F4B093B0DBF8042004905846904736
:10B45800002800F08E82BBF8A87000218BF85110EC
:10B46800002F6DD1BBF93A00DBF82450DBF8281027
:10B47800BBF93860DBF82040BBF93C20DFF8BCA002
:10B48800401B521ACBF830009BF85210CBF83420EE
:10B49800341B0BF12C00CBF82C4011F089F8DAF8AA
:10B4A8000020910041F1B787DBED0C5A1F4CDBED12
:10B4B8000B7A1F4994ED406AD4ED416A94ED427AC3
:10B4C800D4F80C2109681B4B0293B8EEE58ADBED32
:10B4D8000D5AF8EEE77AF8EEE58A013277EE867AC9
:10B4E80038EE268A78EE878A8A42C4ED407A84ED5F
:10B4F800418AC4ED428AC4F80C2101F0508393F8C4
:10B5080000E0BEF1140F02F092870023D4F8145122
:10B518000393062D01F29D84DFE815F0FA15BC1699
:10B528001D15CF16080C39177F1500BFE024002021
:10B53800A4400020E86400209854002020570020F0
:10B54800DE4BDF481A6805934FF47A75B5FBF2F2C3
:10B55800C2EB421502EB8502D500DA4BDFF8C8834F
:10B5680044780293ADB2AF421E78B8F9060003F0F2
:10B578007880DBF87C30BBF93810DBF8602003F109
:10B58800010E07EE901A0A44BEF1010FCBF87CE0D9
:10B59800CBF86020F8EEE77A03F07080DBED1B5AF9
:10B5A800DBED1D6A07EE10EA37EEE56AB8EEC75A1A
:10B5B800012F86EE057A37EE257A77EEC77A8BED7E
:10B5C8001C7AE7EE866A8BED1B7AF0EE667ACBED95
:10B5D8001E6ACBED1D6A03F00D84DBF89030BBF9D1
:10B5E8003A10DBF8642003F1010E07EE901A0A44C2
:10B5F800BEF1010FCBF890E0CBF86420F8EEE77AC3
:10B6080003F05780DBED205ADBED226A07EE10EAE3
:10B6180037EEE56AB8EEC75A012F86EE057A37EE9F
:10B62800257A77EEC77A8BED217AE7EE866A8BED7D
:10B63800207AF0EE667ACBED236ACBED226A03F02E
:10B64800B183DBF8A430BBF93C10DBF8682003F1C8
:10B65800010E07EE901A0A44BEF1010FCBF8A4E0E0
:10B66800CBF86820F8EEE77A03F03E80DBED255A48
:10B67800DBED276A07EE10EA37EEE56AB8EEC75A3F
:10B68800012F86EE057A37EE257A77EEC77A8BEDAD
:10B69800267AE6EE276A8BED257AF0EE667ACBED10
:10B6A800286ACBED276A03F07083874CA8F8060058
:10B6B800BBF8A820029B013A1E78ABF8A820059990
:10B6C8000022072E4A608A60CA6040F05981F9F763
:10B6D80089FF029BDFF850821E78049BC01A94F8F9
:10B6E8002831A8F800000693002B40F04F81744AD7
:10B6F8005279002A01F08081744A1278013AD2B254
:10B70800072E84F8282102F0EE8100230793704B5E
:10B71800D4F83421D3F800A0684B0593049B9FED1F
:10B728006D6AD4ED4C9A6C49C4F834319A1A07EE14
:10B73800902AF8EE677AB7EE007AC6EE278A0025D7
:10B74800664BDFF8E891DFF8E881654F03932E46F2
:10B75800D1ED006A94ED4BDA9FED629ADFED62AAB3
:10B768009FED62CA9FED62AADFED62BA9FED62BAF1
:10B7780077EE69CA6CEEA6CAF4EEC7CAF1EE10FA03
:10B7880088BFF0EE47CA5D4B99ED008A2B44D3ED94
:10B79800007AF5EE407AF1EE10FA17D0584B2B44A8
:10B7A80093ED007A78EE476AB0EEE66AF4EEC67A70
:10B7B800F1EE10FA08D5F5EEC06AF1EE10FACCBF3A
:10B7C80037EE878A37EE678A83ED008A4D4B1A88F1
:10B7D800930739D0022E37D09AF82E104A4B07EE2D
:10B7E800901A2B4493ED007A4B42F8EEE76A07EE85
:10B7F800903A26EE877AF8EEE77AB4EEE77AF1EE39
:10B8080010FA0AD407EE901AF8EE677AF4EEC77ABF
:10B81800F1EE10FA88BFF0EE477A3C4B3C4903EB57
:10B82800460331F91600B3F90C30C31A07EE103A83
:10B83800B8EEC77AD007E7EE497A41F17980354BFF
:10B8480093ED008A27EE888A059B94F868212B449B
:10B8580093ED01EA78EE4EDA002A00F0F7802E4BDD
:10B86800D4F86C2104991B688A1A9A4240F3EE8036
:10B878009AF84830022B02F08581022E04F0518498
:10B88800264B1B68990700F19780254B87ED00CA66
:10B898001B689342C0F2CA80F7EE007AF4EEE79A8A
:10B8A800F1EE10FA40F1D28005991E4BD1ED017AE4
:10B8B80093ED007AF0EEE77A3CE000BF10570020E5
:10B8C80084540020E8640020E024002084460020FE
:10B8D8008468002000247449C4480020BC43002028
:10B8E800C8430020CDCCCC3DAE47813F00000000CE
:10B8F8000000C84200003443610BB63BB848002042
:10B908002426002080680020302600209046002051
:10B9180030680020A0480020CC480020246800207F
:10B92800C8480020D4480020EC64002018260020D5
:10B93800D4430020F4EEC77AF1EE10FA40F1868085
:10B94800D1ED027AF0EEE77AB4EEE77AF1EE10FA8A
:10B958007CDDD1ED037AF0EEE77AB4EEE77AF1EE2A
:10B9680010FA73DD0F4B1B689B075FD50E490F4B11
:10B9780043E00F4B0F4C1E780293072E3FF4A7AEFF
:10B9880094F828310693002B3FF4B1AE013B84F8BC
:10B998002831012E01F0AF8213B0BDEC0E8BBDE84B
:10B9A800F08F00BF246800203068002090460020F7
:10B9B800E8640020E0240020D34BD449DFF8C8E332
:10B9C80031F916C09EED008ADFF8C0E387ED00CAA2
:10B9D80003EB460028EE098AB0F90C00A0EB0C0036
:10B9E80007EE900AF8EEE77ADEF8000027EE888A7C
:10B9F800904278EE4EDABFF64FAFB3F90C20B1F9AA
:10BA080000E0C348AEEB020E00688EEAEE72A2EBCD
:10BA1800EE7282421ADAB3F90E30B1F90220D21A64
:10BA280082EAE273A3EBE27398420FDDB94B1A88FE
:10BA3800002384F86831002A43F07485B64AB74B6E
:10BA48001178186881F00101FAF77CFCB44B2B449B
:10BA580093ED000A039B2DEE000A022E20EE2D0A1C
:10BA6800A3EC010A039304F0BF83AE4BD7ED006A41
:10BA780093ED007AAC4BD3ED007AAC4B93ED006AB2
:10BA8800AB4B67EE277A2B4427EEAC7AD3ED007ADE
:10BA980067EE277AF0EE665AEDEEA75AB1EE467ACF
:10BAA800B4EEE57AF1EE10FA08DCB4EEE56AF1EEF0
:10BAB80010FA8CBFB0EE657AB0EE467A94ED4C6A17
:10BAC800F7EE007AB4EEE76AF1EE10FAACBF0123A4
:10BAD800002343B1F0EEE66AF0EEC77AF4EEE67AB8
:10BAE800F1EE10FA01D587ED007A022E04F0C98232
:10BAF800904A914B52F826001B68B0EE4E0A9847C0
:10BB08008E4A8F4B52F826001B6898479AF83730B0
:10BB180023B18C4B1B88002B00F07187B0EE4C8A48
:10BB2800894B38EE400A2B4493ED008A83ED000AD6
:10BB38009AF8483030EE480A20EE288A002B33D095
:10BB4800824B1B7813F0010300F0BE86F7EE007AF3
:10BB5800F4EEE79AF1EE10FA94F86831C1F20A852A
:10BB6800002B00F0F187D4F86C31049AD31A784A84
:10BB780012689A4218DD774BD3ED007AF0EEEDDAD1
:10BB8800F4EEE7DAF1EE10FA42F10D80614B1A8813
:10BB9800002384F86831002A00F0A2866E494A69B9
:10BBA80012B10A6813604B746C4B94F878212B44DB
:10BBB80093ED000A2DEE000A20EE088A88ED008A2F
:10BBC80032B9039B87ED00CA03ED01CA88ED00CAAC
:10BBD8000136032E09F1040908F1040807F10407E6
:10BBE80005F104057FF4CFAD029B1A78072A01F00E
:10BBF800C684012A01F064870023039394F8802106
:10BC0800002A41F0AB81DFF888A1554BDAF8002013
:10BC18001968D60491F82C0000F10C87DFF87491AC
:10BC2800504AB9F81A3092ED006A4F4A4F4ED2ED99
:10BC3800005AD6ED036A4E4A84ED646A07EE103A5C
:10BC48004C4B92ED005AD3ED007AD3ED013AD3ED87
:10BC5800024A84ED626AB8EEC77A35EEC64A012216
:10BC680036EEC77A84ED614AC4ED655A84F89821A6
:10BC7800C7EE055A0A8D534206EE103A3E4BDFEDE9
:10BC88003F6A93ED005A3E4B93ED004AB7EE007AB7
:10BC9800F4EEC75A35EE045AF1EE10FA88BFF0EE0A
:10BCA800475A35EE275AB8EEC66AF4EEE65AF1EE70
:10BCB80010FA07EE902AB4EEC65AB8BFF0EE665AEC
:10BCC800F1EE10FAC4ED685AB8EE677A01F13283E2
:10BCD800B4EEC75AF1EE10FA88BFB0EE475A264BB9
:10BCE800DFED286AD3ED017A254B93ED014A77EE13
:10BCF800847A25EE265A77EEA37AB4EEE76AF1EE57
:10BD080010FA52DC48E000BF90460020306800205E
:10BD1800D0480020886200208A6200208C620020BF
:10BD280074480020B047002018000020E848002090
:10BD380080480020B8470020B44700200C48002065
:10BD48000848002080680020502600200971002043
:10BD5800CC480020D8480020906200208C48002061
:10BD680084680020F84400207C460020A84B00206E
:10BD780080490020C8430020BC4300200000000088
:10BD8800D44300206F12833AA0480020C8480020FE
:10BD98002057002030740020B4EEE77AF1EE10FA54
:10BDA8008CBFB0EE676AB0EE476AED4B4A8DD3EDB3
:10BDB800027A9FEDEC7A534204EE103A74EEA77AB9
:10BDC800B8EEC44A26EE076AF4EEC47AF1EE10FA29
:10BDD8000AD407EE102AB8EE474AB4EEE74AF1EE65
:10BDE80010FA88BFB0EE674ADF4ADFEDDE7A527894
:10BDF80024EE274A0AB9B1EE444A002841F00486E5
:10BE0800B7EE003AD94E3278002A02F03A86D8497D
:10BE1800DFEDD87AD1ED024AD1ED016A91ED037ACE
:10BE280066EE244AE5EE264AE4EE074A63EE244A23
:10BE3800F4EEE74AF1EE10FAB4BFF0EE673AF0EE2E
:10BE4800643A98BFF0EE647A012ACDED0A4A02F00E
:10BE5800658691ED067AD1ED052AD1ED076A26EEC1
:10BE6800077AA5EE227AA4EE267A23EE077AB4EEB4
:10BE7800E77AF1EE10FAB4EEE37A8CBFF0EE676A77
:10BE8800F0EE476AF1EE10FA88BFF0EE676AB4BFC9
:10BE9800F0EE637AF0EE477A022A8DED0B7A00F025
:10BEA800DE8091ED0A7AD1ED092AD1ED0B3A26EE22
:10BEB800077AA5EE227AA4EE237A23EE077AB4EE67
:10BEC800E67AF1EE10FAB4EEE77A8CBFF0EE663A55
:10BED800F0EE473AF1EE10FA98BFF0EE636AA8BFA9
:10BEE800F0EE477A032A8DED0C7A00F0B88091EDD8
:10BEF8000E7AD1ED0D2AD1ED0F3A26EE077AA5EE8E
:10BF0800227AA4EE237A23EE077AB4EEE67AF1EEEB
:10BF180010FAB4EEE77A8CBFF0EE663AF0EE473AE4
:10BF2800F1EE10FA98BFF0EE636AA8BFF0EE477A18
:10BF3800042A8DED0D7A00F09280D1ED123AD1ED00
:10BF4800112A91ED137A66EE233AE5EE223AE4EEF1
:10BF5800073A63EE233AF4EEE63AF1EE10FAF4EE1D
:10BF6800E73A8CBFB0EE667AB0EE637AF1EE10FA7B
:10BF780098BFF0EE476AA8BFF0EE637A052ACDEDC8
:10BF88000E3A6CD0D1ED163AD1ED152A91ED177A0B
:10BF980066EE233AE5EE223AE4EE073A63EE233AF8
:10BFA800F4EEE63AF1EE10FAF4EEE73A8CBFB0EEB2
:10BFB800667AB0EE637AF1EE10FA98BFF0EE476A4F
:10BFC800A8BFF0EE637A062ACDED0F3A47D0D1ED3F
:10BFD8001A3AD1ED192A91ED1B7A66EE233AE5EE6D
:10BFE800223AE4EE073A63EE233AF4EEE63AF1EE4B
:10BFF80010FAF4EEE73A8CBFB0EE667AB0EE637AE8
:10C00800F1EE10FA98BFF0EE476AA8BFF0EE637A37
:10C01800072ACDED103A22D091ED1E7AD1ED1D2AD6
:10C02800D1ED1F3A26EE077AA5EE227AA3EE847A9E
:10C0380027EE037AB4EEE67AF1EE10FAB4EEE77A78
:10C048008CBFB0EE666AB0EE476AF1EE10FA8DED7D
:10C05800117A98BFF0EE466AA8BFF0EE477A77EEFD
:10C06800E67AF7EE006AF4EEE67AF1EE10FAC4ED3D
:10C078004C7A43F3868586EEA77A022ADDED0B7AA1
:10C0880067EE244A67EE877ACDED0A4ACDED0B7A42
:10C098002DD0DDED0C7A67EE877A032ACDED0C7A88
:10C0A80025D0DDED0D7A67EE877A042ACDED0D7A7D
:10C0B8001DD0DDED0E7A67EE877A052ACDED0E7A72
:10C0C80015D0DDED0F7A67EE877A062ACDED0F7A67
:10C0D8000DD0DDED107A67EE877A072ACDED107A5C
:10C0E80005D0DDED117A27EE877A8DED117A224998
:10C0F800096811F0805801F0F081F6EE005AC4ED9D
:10C10800685A002A02F0B7841C4B94ED656A1C49F2
:10C118001C4F1D78DFF874E094F9983194ED645A57
:10C12800B7F90670C878DAF80010DEED004A05970E
:10C13800BDEEC66A07EE103AB9F81A70124B0797A7
:10C1480016EE10EABDEEC56A05F0010C01F4805741
:10C1580001F0100501F4800108911B7818E000BF78
:10C16800BC4300206F12833A54440020C964002065
:10C17800F0480020000000005C4600200971002003
:10C18800C04B00202C3E002044590020EC480020E1
:10C19800D4ED616AD4ED627AB8EEC77A16EE101A59
:10C1A800002840F02F87002D41F0FD82D24D9DEDF3
:10C1B8000A5A95ED006AD14825EE866AA5EE076A07
:10C1C800B0EE675AA6EE265ABDEEC56A16EE108A7C
:10C1D80016EE107AF045A8BF77464145C8BF0F460E
:10C1E80006EE107AB8EEC66A012A80ED006A00F001
:10C1F800DC8095ED046A9DED0B5A25EE866AA5EE66
:10C20800076AB0EE675AA6EE265ABDEEC56A16EE64
:10C21800108A16EE107AF045A8BF77464145C8BF88
:10C228000F4606EE107AB8EEC66A022A80ED016A59
:10C2380000F0BB8095ED086A9DED0C5A25EE866AE4
:10C24800A5EE076AB0EE675AA6EE265ABDEEC56A95
:10C2580016EE108A16EE107AF045A8BF77464145CB
:10C26800C8BF0F4606EE107AB8EEC66A032A80EDFC
:10C27800026A00F09A8095ED0C6A9DED0D5A25EE44
:10C28800866AA5EE076AB0EE675AA6EE265ABDEE94
:10C29800C56A16EE108A16EE107AF045A8BF7746E2
:10C2A8004145C8BF0F4606EE107AB8EEC66A042AA2
:10C2B80080ED036A79D095ED106A9DED0E5A25EE52
:10C2C800866AA5EE076AB0EE675AA6EE265ABDEE54
:10C2D800C56A16EE108A16EE107AF045A8BF7746A2
:10C2E8004145C8BF0F4606EE107AB8EEC66A052A61
:10C2F80080ED046A59D095ED146A9DED0F5A25EE2C
:10C30800866AA5EE076AB0EE675AA6EE265ABDEE13
:10C31800C56A16EE108A16EE107AF045A8BF774661
:10C328004145C8BF0F4606EE107AB8EEC66A062A1F
:10C3380080ED056A39D095ED186A9DED105A25EE05
:10C34800866AA5EE076AB0EE675AA6EE265ABDEED3
:10C35800C56A16EE108A16EE107AF045A8BF774621
:10C368004145C8BF0F4606EE107AB8EEC66A072ADE
:10C3780080ED066A19D095ED1C6A9DED115A65EE9F
:10C38800865AE7EE055AE6EEA57AFDEEE77A17EE4D
:10C39800905AAE45A8BFAE46A942D8BF714607EE2F
:10C3A800901AF8EEE77AC0ED077ABCF1000F00F0BA
:10C3B8003687534A1268002A40F03E87514A12785D
:10C3C80092B1307868B14D4FDFF858810025E8B256
:10C3D800D8F80030B7EC010A984730780135854223
:10C3E800F5DB494A12689047029B1A78072A01F040
:10C3F800DC800025DAF80020530501F11080434B5A
:10C408001B78BBB1424AB9F81A30B2F906209A42F1
:10C4180010DC404B1B78012B01F07A83192B01F0BB
:10C4280077830E2B06D0082B04D03B4E0023B36035
:10C43800C4F8403194F8AA6126B1384B1B889F078D
:10C4480041F0288394F8B021002A40F0878799F8B2
:10C458001E70002F00F03084022F01F00A83032F92
:10C4680041F0038399F82030C3EB431103EB8101BA
:10C47800C90089B299F81F300233DBB2002A00F0F4
:10C488008385002900F0808525480768B1FBF7F10E
:10C498000FB2A4F8E071002B03F0548007EE907AF5
:10C4A800F8EEE77AF7EE006A86EEA77A1A4E012BC5
:10C4B800D4ED7D6AD6ED007A77EEE67A67EE877A74
:10C4C800C4ED797A3AD0D6ED017AD4ED7E6A77EE6A
:10C4D800E67A022B67EE877AC4ED7A7A2ED0D6ED0B
:10C4E800027AD4ED7F6A77EEE67A032B67EE877AD5
:10C4F800C4ED7B7A22D017E0F04800201C440020CD
:10C508008C4B00206C5C002040590020EF2000205C
:10C518002C3E002054440020A84B002080680020B6
:10C528003C44002038590020D6ED037AD4ED806AC7
:10C5380077EEE67A67EE877AC4ED7C7A0299097815
:10C54800092903F03B81002F40F3BC839BB394ED92
:10C558007D7AD4ED797A77EE877A012BC4ED7D7AEE
:10C56800C6ED007A21D094ED7E7AD4ED7A7A77EE12
:10C57800877A022BC4ED7E7AC6ED017A15D094ED48
:10C588007F7AD4ED7B7A77EE877A032BC4ED7F7AB6
:10C59800C6ED027A09D0D4ED807A94ED7C7A77EEF4
:10C5A800877AC4ED807AC6ED037A013B022BB8BFC7
:10C5B8000223DBB20693069B002A18BF02239E467D
:10C5C800CC4BDFEDCD6A1A68029B91781878137806
:10C5D80007EE903AF8EEE77AB0EE007A67EEA67AC0
:10C5E800F4EEC77AF1EE10FA40F38F86DFEDC36AF6
:10C5F80037EEC77AB0EE676AA7EE266AF0EE466AAB
:10C6080096ED007A9FEDBE6A27EE066AF0EEC65AEE
:10C6180084ED546AC4ED575A99B107EE101AB8EE72
:10C62800C75A9FEDB57A66EE064A25EE075AB7EE69
:10C63800007A37EE457A64EEA54AA4EE857A26EEAE
:10C64800076A9FEDB07A537926EE877A27EE067A45
:10C65800CBB1DFEDA96A9FEDAC6A65EEA65A06EE8E
:10C66800903AF8EEE66A66EEA56AF4EEC66AF1EE6E
:10C6780010FA01F3A081F7EE005A75EEE66A85EE2E
:10C68800A66A27EE067A0C289FEDA08ADFEDA06A3D
:10C6980000F04A87B4EEC87AF1EE10FA98BFB0EE0F
:10C6A800478AB4EEE68AF1EE10FAB8BFB0EE668AB1
:10C6B80084ED4E8ABEF1000F00F0DD80B0EE007A06
:10C6C800F4EEC77AF1EE10FA05DD37EEC77ADFED42
:10C6D8008B6AE7EE267A96ED017ADFED896A27EE16
:10C6E800267AF0EEC75A84ED557AC4ED585A99B1B6
:10C6F80006EE901A9FED806AF8EEE66A27EE075A72
:10C7080066EE866AB7EE006A36EE666A25EE255A48
:10C71800A5EE266A27EE067ADFED7A6A937967EE48
:10C72800A67A67EE877AABB107EE103AB8EEC77A09
:10C738009FED716ADFED746A27EE257A27EE067A97
:10C74800B4EEE67AF1EE10FA41F33981DFED716A61
:10C7580067EEA67A0C2800F0C786DFED6C6A9FEDBD
:10C768006C7AF4EEE67AF1EE10FA88BFF0EE667AAB
:10C77800F4EEC77AF1EE10FAB8BFF0EE477ABEF1E0
:10C78800010FC4ED4F7A76DD5378DFED5B6A07EE73
:10C79800903AF8EEE77AB0EE007A67EEA67A537A26
:10C7A800F4EEC77AF1EE10FA05DD37EEC77ADFED61
:10C7B800536AE7EE267A96ED027ADFED516A27EEA4
:10C7C800267AF0EEC75A84ED567AC4ED595A9BB1D1
:10C7D80006EE903A9FED486AF8EEE66A27EE075AA9
:10C7E80066EE866AB7EE006A36EE666A25EE255A68
:10C7F800A5EE266A27EE067ADFED426AD37967EE60
:10C80800A67A67EE877AFBB107EE103AB8EEC77AD8
:10C818009FED396ADFED3C6A27EE257A27EE067A26
:10C82800B4EEE67AF1EE10FA01F3D780B5EEC07AED
:10C83800F1EE10FA02F10683B7EE006A36EE477A97
:10C84800C6EE076A67EEA67A0C2800F08B86DFED45
:10C858002F6A9FED2F7AF4EEE67AF1EE10FA88BF90
:10C86800F0EE667AF4EEC77AF1EE10FAB8BFF0EEA1
:10C87800477AC4ED507A092800F0228699F8216099
:10C88800002E40F0D785002384F8B03113F0ECF87F
:10C89800002840F03D83204B1B7823B91F4B9B7821
:10C8A800002B41F0F280049805F0F0F9029B1E7805
:10C8B800072E7FF46EA8F8F795FE194B029A401BD5
:10C8C8001678D880FFF765B894F86821002A3FF4F5
:10C8D8006BA9144A84F868311288002A7FF45EA98B
:10C8E800114A124B1178186881F00101F9F72AFDF5
:10C8F800FFF75AB9886800200AD7233CD7A36841B4
:10C908006F12033B00004843A4707D3F00C0F94408
:10C9180000C0F9C40000C8421C4E00206A3E002036
:10C92800EC640020886200208A6200208C6200206B
:10C9380094ED577AB1F90000D4ED586AB1F902E0E4
:10C94800E24AF4EEC76A80EAE0738EEAEE71A3EB7E
:10C95800E073F1EE10FAA1EBEE71B8BFF0EE476AA2
:10C968008B42B8BF0B4607EE103A1378B8EEC77A79
:10C9780027EE097A002B40F0B880D54B93ED006A7A
:10C98800B4EEEA6AF1EE10FA41F17A80F7EE005A55
:10C9980075EEC65A3BEEC77A65EE8B5ACD4BA7EEBD
:10C9A800256A93ED007A26EE076AB5EEC06AF1EEC5
:10C9B80010FA40F28E85CAEE065AB7EE007AB0EE4B
:10C9C800476AA6EEE56AF0EE466AF4EEC76AF1EE4B
:10C9D80010FA88BFF0EE476AF5EEC06AF1EE10FA79
:10C9E800B8BFF0EE4C6ABC4B93ED007A67EE877ADD
:10C9F800A7EEA68AFEF728BF0122FEF781BEB74B35
:10CA0800B74A2B4493ED007AD2ED007AB54B67EE26
:10CA1800277AF7EE006AF4EEE67AF1EE10FA93ED73
:10CA2800007A88BFF0EE667A67EE877A27EE888A02
:10CA3800FFF776B8AC4BDFF8EC921A78AB4ED50717
:10CA48005CBFB9F81820A4F88C21A94AD6ED037A5E
:10CA5800128807EE102AB8EEC77AF4EEC77AF1EE1C
:10CA680010FA41F2C587A34D2B8807EE103AB8EEAD
:10CA7800C77AF4EEC77AF1EE10FAC1F255809E4AF1
:10CA88009E4D92ED006AD5ED006A94F99821C4EDA7
:10CA9800646A76EE665A012AC4ED626AC4ED615A88
:10CAA80084ED656A01F0D785049BC4F89C310025A4
:10CAB80037EEC77AFCEEE77A914E84ED687A17EE86
:10CAC800902AA4F88C21012296ED005A84F8982126
:10CAD8008C4A954241F2BC878B4BD3ED007AD3ED5B
:10CAE800013AD3ED024AFFF7C3B87A4B93ED005AE7
:10CAF800B5EEC05AF1EE10FA40F3EB84834BD3ED58
:10CB0800004AF5EEC04AF1EE10FA40F3E28434EE42
:10CB1800C77A66EECA5A87EE246AC5EE856AB7EE0A
:10CB2800007AB4EEC76AF1EE10FA88BFB0EE476A31
:10CB3800B5EEC06AF1EE10FA76EE876AB8BFB0EECD
:10CB48004C6A66EE266A40E7714AD2ED007AB0EE8A
:10CB5800C87AB4EEE77AF1EE10FA7FF725A86D4AA5
:10CB6800D2ED007AB0EEED7AB4EEE77AF1EE10FA93
:10CB78007FF71AA8684AD9ED007A92ED007AF0EEAC
:10CB8800E77AF4EEC77AF1EE10FA7FF50DA80122E4
:10CB98000499C4F86C1184F86821FEF7E8BF07EE21
:10CBA800102A1978DFF88081C4F80C71B8EEC77ABA
:10CBB800F7EE006A132986EE879AB8F90400B4F8EC
:10CBC80010619BED070A01F0D284544A544992ED52
:10CBD800001AD2ED053A92ED122A92ED173AD2EDEB
:10CBE800091AD2ED0E4A92ED016A92ED064A92EDCB
:10CBF8000A7AD2ED0F5AD2ED132AD2ED186A92EDC5
:10CC0800045AD2ED030A67EE897A69EE288A29EE7A
:10CC1800088AE1EE273A01EB86070025A2EE283ABA
:10CC2800C4F80051C4F80451E1EE884AA6EE274A38
:10CC3800E7EE085A92ED167A92ED0D6A92ED021A15
:10CC4800D2ED0C1AC7ED003AE2EEA86A25EE635A57
:10CC580027EE437A92ED0B2AD2ED152AC7ED204A2A
:10CC6800A0EEE34A26EE646AD2ED143A82ED054A54
:10CC7800A1EE275AF0EE477AE1EEE45AA2EE086AEE
:10CC8800E2EEC36AE3EEA87A82ED065AC2ED0E5AC6
:10CC980082ED0F6A87ED403AC2ED176AC2ED187A45
:10CCA800C4F80851721C02F01F02A4F81021A8F859
:10CCB8000400029BFEF723BCA4F8E071002A3FF4AD
:10CCC800E5AD0A4E4FF0020E7AE400BFAC480020F2
:10CCD800B4480020A8480020A44800203C26002092
:10CCE8009C4800209848002009710020A84B00208B
:10CCF80084490020864900207C4600207049002095
:10CD08008C4900208FD00300C8430020B048002081
:10CD1800DC480020D8480020E048002034430020A8
:10CD2800C840002030740020EC6400209C4A117830
:10CD3800D4F818719B4B9FED9C7AFE009A1982EDEE
:10CD4800007A002979D09948B0EE476AF0EE476A30
:10CD58000022F0EC017A013267EEA77A05EE902AFC
:10CD6800B4EEE77AF1EE10FAF8EEE55AB8BFB0EE95
:10CD7800677A8A4276EEA76AA7EEA56AE9D1F5EE48
:10CD8800C06A9A19F1EE10FA82ED007A55DDC6EE06
:10CD9800265A874A87490988F7EE007A75EEE75AD6
:10CDA800D2ED007A65EEA77AFDEEE77A17EE902AC3
:10CDB800812A42F357808A42A8BF0A4607EE902A82
:10CDC800F8EEE77A7C4AF01902EB800292ED057AD8
:10CDD800D2ED003A92ED066A92ED014AD2ED046A6C
:10CDE800D2ED034A92ED025AA3EEA77AA4EE276A7F
:10CDF80066EEC76AA7EE646ABDEEC77AE5EE276AF3
:10CE080017EE100A812882ED056AC2ED066A42F320
:10CE180026808142A8BF014607EE901AF8EEE77A0D
:10CE2800FCEEE77ACDED057ABDF8142099198A80D1
:10CE38001FB9BEF1130F02F0AC86BEF1150F41F019
:10CE4800DC801E44DFF89081B28828F81720D4F8D7
:10CE580014515A4A013582FB05325119EA17C2EBBF
:10CE6800A102C2EBC202AD1AC4F814515448D4F856
:10CE78001C11049B534D02682D78C4F81C31591AB3
:10CE88000A440260002D40F0DB8107EE901A4E4EF6
:10CE9800DFF864914D4FB8EEE78A06F5F07506F5B0
:10CEA8001378F6EC017A9BED070ADBF80832F8EE06
:10CEB800E77A284627EE800A9847A5F1E000DBF8D4
:10CEC80028319847A5F17000DBF898319847D6F8D3
:10CED800EC00DBF8AC309847D7ED007AA9EC010AF2
:10CEE800E0EE087A2435A845E7EC017AD9D1029B0F
:10CEF8001E78FEF742BD364B364A19681288364B03
:10CF0800C96919805A8013B0BDEC0E8BBDE8F08F4B
:10CF1800324C12F09FFC6378022B00F0E985032B5A
:10CF28007FF4B9AC41F2B813E35C002B41F01583F0
:10CF380041F2A403E35C002B41F00A8341F2E803C9
:10CF4800E35C002B41F00E8341F22C13E35C002BD1
:10CF58003FF4A1AC224811F02DFC9CE4214B224E59
:10CF68001A7812F0010F327840F04C83002A00F052
:10CF7800458592001D491E48DFF880A0DFF88090A3
:10CF880026F0B8FEFFF715BAB4F8E071013F3FB2DA
:10CF9800002FA4F8E0717FF791AE164EFFF7D6BACE
:10CFA800AA400020A043002000000000E024002048
:10CFB800AC400020A8400020C84200209324499299
:10CFC80074470020A0400020C45400207847002067
:10CFD8007433002026330020EC6400207474002091
:10CFE800A085002009710020C96400207833002042
:10CFF8001C440020A84B0020145700202057002074
:10D0080030740020002D00F0BD86BCF1000F42F006
:10D01800A382CA4D002B42F0378195ED006A9DED41
:10D028000A5AC74825EE866AFDEEE44AA5EE076A65
:10D03800B0EE675AA6EE265A14EE901ABDEEC56AEF
:10D0480016EE10CA16EE107AF445A8BF7746614569
:10D05800C8BF0F4606EE107AB8EEC66A012A80ED00
:10D06800006A00F0DF8095ED046A9DED0B5A25EE0D
:10D07800866AA5EE076AB0EE675AA6EE265ABDEE96
:10D08800C56A16EE10CA16EE107AF445A8BF7746A0
:10D098008C45B8BF0F4606EE107AB8EEC66A022A6B
:10D0A80080ED016A00F0BE8095ED086A9DED0C5A8E
:10D0B80025EE866AA5EE076AB0EE675AA6EE265AEE
:10D0C800BDEEC56A16EE10CA16EE107AF445A8BF72
:10D0D80077468C45B8BF0F4606EE107AB8EEC66A9A
:10D0E800032A80ED026A00F09D8095ED0C6A9DEDA3
:10D0F8000D5A25EE866AA5EE076AB0EE675AA6EEC7
:10D10800265ABDEEC56A16EE10CA16EE107AF44518
:10D11800A8BF77468C45B8BF0F4606EE107AB8EE22
:10D12800C66A042A80ED036A7CD095ED106A9DEDED
:10D138000E5A25EE866AA5EE076AB0EE675AA6EE85
:10D14800265ABDEEC56A16EE10CA16EE107AF445D8
:10D15800A8BF77468C45B8BF0F4606EE107AB8EEE2
:10D16800C66A052A80ED046A5CD095ED146A9DEDC7
:10D178000F5A25EE866AA5EE076AB0EE675AA6EE44
:10D18800265ABDEEC56A16EE10CA16EE107AF44598
:10D19800A8BF77468C45B8BF0F4606EE107AB8EEA2
:10D1A800C66A062A80ED056A3CD095ED186A9DEDA1
:10D1B800105A25EE866AA5EE076AB0EE675AA6EE03
:10D1C800265ABDEEC56A16EE10CA16EE107AF44558
:10D1D800A8BF77468C45B8BF0F4606EE107AB8EE62
:10D1E800C66A072A80ED066A1CD095ED1C6A9DED7B
:10D1F800115A65EE865AE7EE055AE6EEA57AFDEE77
:10D20800E77A17EE905AAE45A8BFAE46A942D8BFF6
:10D21800714607EE901AF8EEE77AC0ED077A002A11
:10D228003FF4C7A892004749454826F063FD464A9F
:10D238001268002A3FF4C2A816F00CF9FFF7BEB82E
:10D2480007EE901A414D424BDFF80881DFF808914C
:10D258000394F8EEE78A05F5B8760027CDF818802C
:10D268001C46029BDBED077A1B78172B51D095EDF6
:10D27800007AB8EEC78A082B28EE278A07D1B0EEC5
:10D28800480A059326F00CFF059BA8F80000DAF879
:10D29800002092000BD5002F02F00787B0EE480A55
:10D2A800DBF8083206F170009847B0EE408AB0EE1D
:10D2B800480ADBF82831A6F170009847DBF8983166
:10D2C80030469847029B1B78032BB0EE408A2CD03F
:10D2D800D5F8F000DBF8AC30B0EE480A9847D9ED45
:10D2E800007AA4EC010AE0EE287A0137032F06F150
:10D2F800240608F1020805F10405E9EC017AB0D129
:10D30800029B039C1E78FEF738BBF0EE676AFFF7B6
:10D3180077B995ED007A0BEB4702B8EEC78A128F02
:10D32800A8F8002028EE278AB1E726F0B9FEA8F869
:10D338000000CDE7B0EE465AFEF7D1BCF048002019
:10D348001C440020783300208C4B0020C45400205B
:10D3580014570020EC640020784700209B499C4B20
:10D36800D1F8EC101B6844F620608142A8BF014642
:10D37800B1F57A7FB8BF4FF47A7189B213F0100F04
:10D38800A4F8B211DAF8003000F0C983DB0441F1E7
:10D398006D85904BD3F800E0BEF832707F088E4E52
:10D3A8008E48D4F8B431D6ED037AA0FB0101880980
:10D3B800642191FBF0F11429BDEEE77A04EB4306F2
:10D3C800A8BF142101339942C4F8B43117EE10CA2A
:10D3D800DCBF0023C4F8B43104EB4303A6F8B8C19A
:10D3E800B3F9B83107EE103AB8EEC77A77EEC77AD4
:10D3F800FDEEE77ACDED037ABDF90C1081EAE17311
:10D40800A3EBE173BB4201F3A48675494FF07E5349
:10D418000B60FFF71CB8734B0293734C26E5DBF8DF
:10D428000830002B3EF4EBAF7049A1F14C0098474F
:10D43800FEF7E5BF1E216648F4F771FB00283FF4AC
:10D4480022AA6B4B1B885A063FF51DAA94F8043292
:10D45800B34242F0D581624BD4ED827AD3ED016AB2
:10D4680094ED505ADFED635A9FED636A27EEC57A53
:10D4780068EE277AA8EE267AE5EE267AB4EEE57A03
:10D48800F1EE10FA88BFB0EE657AB4EEC67AF1EE26
:10D4980010FAF4EEE57AB8BFB0EE467AF1EE10FA7B
:10D4A80088BFF0EE657AF4EEC67AF1EE10FAB8BFEE
:10D4B800F0EE467A84ED4E7AC4ED507AFFF7E3B980
:10D4C800FDEEC87A4D4A17EE903A9780D380FFF761
:10D4D800D5B9DFED4B6AFFF786BADAF800104902D2
:10D4E8003EF50BAEFEF70DBE9FED427ADFED426AC8
:10D4F8004249F4EEC77AF1EE10FA98BFB0EE677AB7
:10D50800FDEEE77AB4EEE67AF1EE10FA17EE903A0D
:10D51800B8BFB0EE667ABEF1010F84ED4F7A4B804A
:10D528003FF732A9FFF7AAB9B4EEC87AF1EE10FABC
:10D5380098BFB0EE478ABDEEC77AB4EEE68ADFF848
:10D54800BCC0F1EE10FA17EE103AB8BFB0EE668A1A
:10D5580084ED4E8AACF80030BEF1000F7FF4AEA81F
:10D56800FFF78CB9BDEEE77A244B17EE102A9A80A4
:10D57800FFF76DB9002B3EF417ABFEF7F4BAF8F7D6
:10D5880031F8029BDFF874801A78079B012AA0EB18
:10D598000300A8F8020000F09582072A7EF42CAB5D
:10D5A800F8F720F80390FEF729BBF8F71BF8029B61
:10D5B80012491A78039B072AA0EB030088807EF49F
:10D5C80018AFF8F70FF80546FEF714BF68000020FB
:10D5D8005C46002084680020A84B0020D34D6210D0
:10D5E80018000020E8640020E0240020E454002013
:10D5F8008068002000C0F94400C0F9C4EC64002031
:10D6080000000000002A00F0F981D4ED583A94EDAA
:10D61800574AD4ED627AF34994ED617A91ED005A54
:10D62800D4ED555A94ED546AEF4DF048F4EEC43AEF
:10D63800F3EE046AF1EE10FA77EEA64A00F1C28220
:10D6480095ED026A26EE656AB0EE674AA6EE074ACD
:10D65800B4EEE44A34EE666AF1EE10FA48BFB0EE72
:10D66800456A012A80ED006A00F0C88195ED066AD6
:10D6780026EE656AB0EE674AA6EE074AB4EEE44ABB
:10D6880034EE666AF1EE10FA48BFB0EE456A022A37
:10D6980080ED016A00F0B28195ED0A6A26EE656AAE
:10D6A800B0EE674AA6EE074AB4EEE44A34EE666A7C
:10D6B800F1EE10FA48BFB0EE456A032A80ED026A1F
:10D6C80000F09C8195ED0E6A26EE656AB0EE674A19
:10D6D800A6EE074AB4EEE44A34EE666AF1EE10FAB2
:10D6E80048BFB0EE456A042A80ED036A00F08681DF
:10D6F80095ED126A26EE656AB0EE674AA6EE074A0D
:10D70800B4EEE44A34EE666AF1EE10FA48BFB0EEC1
:10D71800456A052A80ED046A00F0708195ED166A65
:10D7280026EE656AB0EE674AA6EE074AB4EEE44A0A
:10D7380074EE666AF1EE10FA48BFF0EE456A062A02
:10D74800C0ED056A00F05A81D5ED1A6A66EEE56A01
:10D75800B0EE674AA6EE874AB3EE046AB4EEE44A2E
:10D7680074EE466AF1EE10FA48BFF0EE456A072AF1
:10D77800C0ED066A00F04281D5ED1E6ADFF874A29A
:10D78800DFF8749266EEE55AE5EE877AF4EEE74A3A
:10D7980077EEC67AF1EE10FAC8BFF0EE457AC0ED22
:10D7A800077AFEF706BE904D9DED0A5A95ED006A80
:10D7B800BCF1000F41F0E68125EE866A8B48A5EEA4
:10D7C800076AB0EE675AA6EE265ABDEEC56A16EE8F
:10D7D80010CA16EE107AF445A8BF77466145C8BF4F
:10D7E8000F4606EE107AB8EEC66A012A80ED006A86
:10D7F8003FF418AD95ED046A9DED0B5A25EE866A47
:10D80800A5EE076AB0EE675AA6EE265ABDEEC56ABF
:10D8180016EE10CA16EE107AF445A8BF7746614591
:10D82800C8BF0F4606EE107AB8EEC66A022A80ED27
:10D83800016A3FF4F7AC95ED086A9DED0C5A25EEA8
:10D84800866AA5EE076AB0EE675AA6EE265ABDEEBE
:10D85800C56A16EE10CA16EE107AF445A8BF7746C8
:10D868006145C8BF0F4606EE107AB8EEC66A032AAD
:10D8780080ED026A3FF4D6AC95ED0C6A9DED0D5A29
:10D8880025EE866AA5EE076AB0EE675AA6EE265A16
:10D89800BDEEC56A16EE10CA16EE107AF445A8BF9A
:10D8A80077466145C8BF0F4606EE107AB8EEC66ADD
:10D8B800042A80ED036A3FF4B5AC95ED106A9DED3E
:10D8C8000E5A25EE866AA5EE076AB0EE675AA6EEEE
:10D8D800265ABDEEC56A16EE10CA16EE107AF44541
:10D8E800A8BF77466145C8BF0F4606EE107AB8EE66
:10D8F800C66A052A80ED046A3FF494AC95ED146A73
:10D908009DED0F5A25EE866AA5EE076AB0EE675AB6
:10D91800A6EE265ABDEEC56A16EE10CA16EE107AA5
:10D92800F445A8BF77466145C8BF0F4606EE107A92
:10D93800B8EEC66A062A80ED056A3FF473AC95ED29
:10D94800186A9DED105A25EE866AA5EE076AB0EEB4
:10D95800675AA6EE265ABDEEC56A16EE10CA16EE2E
:10D96800107AF445A8BF77466145C8BF0F4606EE52
:10D97800107AB8EEC66A072A80ED066A3FF452AC00
:10D9880095ED1C6A9DED115A65EE865AE7EE055A2B
:10D99800E6EEA57AFDEEE77A17EE905AAE45A8BFF7
:10D9A800AE46A942C8BF8E4607EE90EAF8EEE77A7F
:10D9B800C0ED077A33E49FED0E6AFEF762BEB5EE5E
:10D9C800C07AF1EE10FA01F14182B7EE006A36EE44
:10D9D800477AC6EE076AFEF7BBBEDFED056AFEF7BB
:10D9E80031BF00BFEC480020F04800201C44002054
:10D9F8000000C8422057002030740020DFF878A3C8
:10DA0800DFF87893FEF7D5BCC8494A79002A3EF476
:10DA1800F7A9C74A1278002A3EF4F2A90B78C5493B
:10DA2800DFEDC54A07EE903A0B88B8EE677A07EE45
:10DA3800902A06EE903AF8EEE77AF8EE666A67EE14
:10DA4800277AB7EE007A87EEA63AB4EEE43AF1EE1A
:10DA580010FA88BFB0EE643AB4EEC73AF1EE10FAA5
:10DA6800B8BFB0EE473AFEF7CDB9B44B5988FEF7C8
:10DA780001BDB4F8B21101F57A7189B2FEF7FABCAA
:10DA8800AF4B93ED006AFEF790BF04980FF0C4FA0D
:10DA9800FEF709BFAB4B9FEDAC7AD3ED087AF4EEF5
:10DAA800C77AF1EE10FA00F2F7849FEDA87AA84E33
:10DAB800D6ED037A77EE877AC6ED037AFEF7C2BC15
:10DAC800DFF8BC82F7F78EFDA249D4F87C210968FB
:10DAD8000390821A511AC4F87C01A8F80420A8F807
:10DAE8000610FEF78BB8F7F77DFD0790FDF70FBE20
:10DAF800A3784FF0010A072B3EF6CDAEDFE813F00E
:10DB08003D0755072D072207BE0682068C063907F2
:10DB1800914B9B7B002B3EF488ACFEF78BBCD80066
:10DB28003FF534ACFEF793BCB4F88C51954240F203
:10DB3800FE8494F8A451002D40F0C687874A884E89
:10DB480092ED007AD6ED007A94F99821C4ED647AC2
:10DB580077EE676A012AC4ED627AC4ED616A84EDE2
:10DB6800657A02F00880049BC4F89C317D4A9FEDD9
:10DB7800777A92ED005A84ED687A012284F8982128
:10DB8800FEF7A6BF784B1B88002B40F0F385774A39
:10DB9800774B11781868F8F7D5FBD4F86C21049BFB
:10DBA8009A1AFDF76ABE734BD9ED007A93ED007AA5
:10DBB800F0EEE77AF4EEC77AF1EE10FA7DF7F4AFFB
:10DBC800FDF7E4BFD5ED015A65EEC65AB0EE674AD7
:10DBD800A5EE874AB4EEE44A74EE665AF1EE10FAFE
:10DBE80048BFF0EE455A012AC0ED005A3FF406AF8F
:10DBF800D5ED055A65EEC65AB0EE674AA5EE874AD6
:10DC0800B4EEE44A74EE665AF1EE10FA48BFF0EE4C
:10DC1800455A022AC0ED015A3FF4F0AED5ED095A33
:10DC280065EEC65AB0EE674AA5EE874AB4EEE44AF6
:10DC380074EE665AF1EE10FA48BFF0EE455A032A20
:10DC4800C0ED025A3FF4DAAED5ED0D5A65EEC65A6C
:10DC5800B0EE674AA5EE874AB4EEE44A74EE665A17
:10DC6800F1EE10FA48BFF0EE455A042AC0ED035A07
:10DC78003FF4C4AED5ED115A65EEC65AB0EE674A08
:10DC8800A5EE874AB4EEE44A74EE665AF1EE10FA4D
:10DC980048BFF0EE455A052AC0ED045A3FF4AEAE2F
:10DCA800D5ED155A65EEC65AB0EE674AA5EE874A15
:10DCB800B4EEE44A74EE666AF1EE10FA48BFF0EE8C
:10DCC800456A062AC0ED056A3FF498AED5ED196A93
:10DCD80066EEC66AB0EE674AA6EE874AF3EE045AC5
:10DCE800B4EEE44A74EE656AF1EE10FA48BFF0EE5D
:10DCF800456A072AC0ED066A3FF480AED5ED1D6A75
:10DD0800DFF874A0DFF8749026EEC66AE6EE077AAC
:10DD1800F4EEE47A77EEE57AF1EE10FAB8BFF0EEB9
:10DD2800457AC0ED077AFEF744BB00BF14680020AF
:10DD38001268002004660020713DAA3F786A00201E
:10DD4800A84800204C4700208FC2753C0000000006
:10DD5800A84B00203C440020845200207C46002030
:10DD6800704900208C490020886200208A620020C7
:10DD78008C620020E04800202057002030740020EA
:10DD8800EC640020D94D002B41F0A08095ED006A8D
:10DD98009DED0A5AD64825EE866AFDEEE44AA5EEC0
:10DDA800076AB0EE675AA6EE265A14EE901ABDEE30
:10DDB800C56A16EE108A16EE107AF045A8BF7746A7
:10DDC8004145C8BF0F4606EE107AB8EEC66A012A6A
:10DDD80080ED006A3EF4E9AA95ED046A9DED0B5AC0
:10DDE80025EE866AA5EE076AB0EE675AA6EE265AB1
:10DDF800BDEEC56A16EE108A16EE107AF045A8BF79
:10DE080077468845B8BF0F4606EE107AB8EEC66A60
:10DE1800022A80ED016A3EF4C8AA95ED086A9DEDD4
:10DE28000C5A25EE866AA5EE076AB0EE675AA6EE8A
:10DE3800265ABDEEC56A16EE108A16EE107AF0451F
:10DE4800A8BF77468845B8BF0F4606EE107AB8EEE9
:10DE5800C66A032A80ED026A3EF4A7AA95ED0C6A09
:10DE68009DED0D5A25EE866AA5EE076AB0EE675A53
:10DE7800A6EE265ABDEEC56A16EE108A16EE107A80
:10DE8800F045A8BF77468845B8BF0F4606EE107A1A
:10DE9800B8EEC66A042A80ED036A3EF486AA95EDB8
:10DEA800106A9DED0E5A25EE866AA5EE076AB0EE59
:10DEB800675AA6EE265ABDEEC56A16EE108A16EE09
:10DEC800107AF045A8BF77468845B8BF0F4606EEDA
:10DED800107AB8EEC66A052A80ED046A3EF465AA8F
:10DEE80095ED146A9DED0F5A25EE866AA5EE076A30
:10DEF800B0EE675AA6EE265ABDEEC56A16EE108A2F
:10DF080016EE107AF045A8BF77468845B8BF0F4689
:10DF180006EE107AB8EEC66A062A80ED056A3EF467
:10DF280044AA95ED186A9DED105A25EE866AA5EE6D
:10DF3800076AB0EE675AA6EE265ABDEEC56A16EE17
:10DF4800108A16EE107AF045A8BF77468845B8BF04
:10DF58000F46FEF708BA674ED4ED017A94ED006AD1
:10DF68003188726977EEA77AF0EE006AB0EE677AC8
:10DF7800A6EE267A4E1E04EBC601D6EE267A08399E
:10DF88001032F6EE003A27EE237A67EEA37A84ED94
:10DF9800207AC4ED217A584C274604F1800091ED8F
:10DFA800027A91ED036AD7ED036AD7ED027A52ED52
:10DFB800014A12ED025A37EE674A76EEC65A77EEF4
:10DFC800277AE4EE845A013EA1F10801E5EE047ACD
:10DFD80007F1080702F1080236EE267A00F1080078
:10DFE800E4EE877AE5EE475A67EEA37A25EEA37A40
:10DFF800C0ED007A80ED017AD1D1BEF1140F7EF424
:10E0080028AFF7F7EFFA039BDFF80081C01AA8F8EA
:10E018000200D4F81451FEF71CBFD4F81831B4F834
:10E0280010C1364ACCF120095FFA89F90CEB431785
:10E0380002EB87075FEA990201F0BC8501321601FD
:10E048002F48304907EB060807F1100212ED024A83
:10E0580012ED035A12ED016A12ED047A50ED024AEC
:10E0680050ED035A50ED016A50ED047A64EE244AEB
:10E0780065EE255A66EE266A67EE277A10329045D5
:10E0880041ED024A41ED035A41ED016A41ED047A3E
:10E0980000F1100001F11001D8D11B48A6F11001C0
:10E0A8000F4400EB0108214419F0030209D0B7EC32
:10E0B800017AF8EC017A67EE277A013AE1EC017A05
:10E0C800F5D1BCF1000F41F05380BEF1140F7EF47E
:10E0D800C0AEF7F787FA039BDFF83080D4F8145105
:10E0E800C01AA8F80200FEF7B4BE00BFF04800202E
:10E0F8001C440020B0400020E0240020C84000203C
:10E1080058420020F024002048420020EC640020FF
:10E11800D04E318873684FEA51094FEA89005FEAA7
:10E12800D10C04EB000204EB810500F0A18000F1A2
:10E1380010010CF1010CC84F02EB0C1C29441032E1
:10E1480003F1100E05F1100050ED032A50ED043ACA
:10E1580017ED043A17ED032A50ED026A10ED016A33
:10E1680017ED021A57ED010A11ED044A11ED035A91
:10E1780052ED044A52ED035A12ED027A52ED017A39
:10E1880051ED021A11ED010A73EE238A32EE228A4A
:10E1980047ED048A07ED038A71EE268A30EE868AF7
:10E1A80047ED028A07ED018A74EE848A35EE858A86
:10E1B80042ED048A02ED038A77EE218A37EE808ADF
:10E1C80042ED028A02ED018A73EE633A75EE655AF2
:10E1D8001EED035A32EE623A74EE644A25EE638A03
:10E1E8001EED044A23EE052A64EE652AA3EE048A8E
:10E1F8001032944524EE843AA3EE842A07F11007DE
:10E208000EF1100EA5EE853A00F1100001F1100193
:10E21800E4EE852A00ED078A00ED082A01ED073AA9
:10E2280041ED082A5EED055A1EED065A71EE666A42
:10E2380030EEC66A31EEC77A70EE677A26EE253A76
:10E2480065EEE63A25EE674A67EE054AE6EE053AD8
:10E25800A6EE853AA7EE254AE7EEA54A00ED063A6E
:10E2680040ED053A01ED064A41ED054A7FF46CAFF1
:10E278001FFA89F91A464946784818F01BFF726850
:10E288004946284618F016FF029B1A78142A7FF48C
:10E29800C0AEB6E66F4E7148B268B18924F024FD6D
:10E2A800029B93F800E0BEF1140F01F0EB84D4F860
:10E2B80014510135C4F814514EE6DFF8B89199F8B5
:10E2C80000108F0801F00386654E07F101084FEA38
:10E2D800481806EB080C06F12002A6F1700012EDB2
:10E2E800076A52ED056A12ED037A52ED017A52ED92
:10E2F800025A12ED084A52ED064A12ED045A26EE69
:10E30800066A66EEA66A27EE077A67EEA77AA4EE93
:10E31800046A20329445E4EEA46A00F11000A5EEE8
:10E32800057AE5EEA57AF1EEC65AB1EEE66AF1EEA7
:10E33800C76AB1EEE77A40ED085A00ED076A40ED8A
:10E34800066A00ED057ACAD1A8F12002324404EB2E
:10E35800071711F0030018BF08320FD052ED017AE9
:10E3680012ED027A67EEA77A0138E7EE077A02F132
:10E378000802B1EEE77AA7EC017AEFD1BEF1140FEB
:10E3880001F06D840135C4F81451FEF7D1BCD4F8FE
:10E39800185134493448354BEA00114415448A88E9
:10E3A800196800EE102A643AC82AA8BFC822782A39
:10E3B800B8BF782207EE902AB8EEC07AF8EEE77A6E
:10E3C80000EB850577EE670A77EE876A67EE877A4E
:10E3D80020EEA67AB8EE400AC7EE870A2846D5F896
:10E3E8001490D5F81880EF692E6A19F043F9029B4A
:10E3F800C5F8149093F800E0C5F81880BEF1140F22
:10E40800EF612E6201F01E84D4F81821184BD4F85D
:10E418001451013283FB0213A3EBE27303EB4303B2
:10E42800D31A0135C4F81831C4F81451F7E5F7F7D1
:10E43800D9F8029B039093F800E0BEF1140F05BFD2
:10E44800DFF83480D4F81451D4F81451A8F80050E7
:10E45800FDF75FB8B0400020F0240020E024002041
:10E4680060250020A0430020A4560020105700205B
:10E4780056555555AA400020EC640020306E99BCD2
:10E488002716983DA40DC93F843459BEDB0F494077
:10E49800D06D393A00000000F0EEE76AB7EE005A96
:10E4A80035EE665A1FED0B4A5FED0B5A1FED0A6AEF
:10E4B8001FED0C7A94ED6B0AF1EEC54AE6EE845A2C
:10E4C800F5EEC07AA6EEA56AF1EE10FAA6EE867A07
:10E4D80048BF5FED127A27EE247A48BF37EEC77A35
:10E4E80027EE000A25F0DCFDB0F5617F00F3A28677
:10E4F80007EE900AF8EEE76A5FED1B7A66EEA76A08
:10E5080007EE906ABDEEE67AF8EEE77A17EE103A73
:10E518002033402B41F295841FED220A25F0C0FDDF
:10E5280000B207EE900AB8EEE77AFFF7C0BAC14A20
:10E5380002F1500503E00432954200F0C5821378D9
:10E54800262BF8D19678D3789E42F4D2FFF7F1BA09
:10E55800B94810F02FF9FEF7F1BCB84810F02AF9C5
:10E56800FEF7E6BCB64810F025F9FEF7EDBCB54D50
:10E57800B54F95ED004A95ED057AD5ED014A95ED33
:10E58800066AD5ED046A95ED035AD5ED025A67EE91
:10E59800897A07EB8602A4EE277AA4EEA76A66EECC
:10E5A800C76AA5EE476AE5EEA76A20EE070A85ED79
:10E5B800056AC5ED066A82ED007A29EE088A25F01B
:10E5C8006FFD69EE288AD5ED0E5AD5ED176A95EDDF
:10E5D800091AD5ED121A95ED0F5A95ED187A95EDA1
:10E5E8000A2AD5ED132A95ED0D6AD5ED167A95ED23
:10E5F8000C3AD5ED0B3A95ED154AD5ED144AE1EEF6
:10E60800085A002207EB8601E8EEA16A00B2C4F8B6
:10E618000021A2EE085AC4F80421C4F80821A8EE83
:10E62800A27A26EE656A67EEE67AA3EE655AA3EE4D
:10E63800886AA6EEC47AE8EEA47A85ED0E5AC1ED92
:10E64800205A85ED0F6AC1ED406A85ED177AC5ED50
:10E65800187AFEF727BBD4F89C51049B5D1BFEF784
:10E6680027BABBF93820CBF8201007EE902A0121F1
:10E67800F8EEE77ACBF86020CBF87C100022012F67
:10E68800CBED1C7ACBED1B7ACBF8742001F06B82B2
:10E69800AF427CF4A2AFBBF93A20CBF8642007EE76
:10E6A800902A00210122F8EEE77ACBF82410CBF863
:10E6B80090200022012FCBED217ACBED207ACBF8E8
:10E6C800882001F05482AF427CF4BBAFBBF93C20F8
:10E6D800CBF8682007EE902A00210122F8EEE77AAD
:10E6E800CBF82810CBF8A4200022012FCBED267AF6
:10E6F800CBED257ACBF89C207CF4D7AF9FED538ADD
:10E70800032E49D04CB107EE904AF8EEE77AF4EEC2
:10E71800C87AF1EE10FA01F1DF834D4A4D4C1168C9
:10E72800DBF86820A8F8060094F8200102EB5502EF
:10E7380092FBF5F50022CBF828508A620A63CA6278
:10E7480028B1454A126832F480637CF4B1AF434A79
:10E75800126812F4003241F0FE8141481146835C90
:10E76800012B02F10C0200F0928301311829F6D135
:10E77800FCF79EBF3B494B69002B3DF47EA83A4805
:10E788003A4B008893FBF0F00B684FF0010E1860CD
:10E7980081F811E0FDF771B8B0EE480A25F080FC69
:10E7A80000B2AFE723690622652BA27034D922781C
:10E7B800032A14BF6FF0FF026FF07F02A3F1650315
:10E7C80003EA020303F1010314BF4FF480728022AD
:10E7D8009A42236120D23A68E768023203EB0708BD
:10E7E800904581F04984224A6760D16FC4F8088057
:10E7F800490203FB01F30521176042F81C3C42F86B
:10E80800183CA170A2681B49012023F0B1FE012821
:10E8180041F028840623A3700021174823F0C8FA82
:10E82800012841F01F84A3780133DBB2A370FFF7FE
:10E8380062B900BFB0720020188500202C86002025
:10E848005C85002034430020C84000200000000000
:10E8580074330020E02400207C680020F031002080
:10E86800AC58030890620020A862002020A107008D
:10E878000886002078740020E48500202278237D13
:10E88800AF4FDFF8FC92032A14BF4FF480784FF0A3
:10E898008008002B42D0012BFBD1AA4B6268196873
:10E8A800386800234FEA412E4FF0FF31B1FBFEF1EB
:10E8B80012EB010B43F1000C0021614500F102004D
:10E8C80008BF584538BF83465A469F49022010F072
:10E8D800DDFE032801F26B8101A353F820F000BF8D
:10E8E8009FC80008F9E800089FC80008F9E8000870
:10E8F8006268A3682669991AB14284BFE2602161FF
:10E9080003283FF44FAF0133B3FBF8F208FB123290
:10E918000AB143449B1A0022636022753A6849464B
:10E928000232002010F0B2FE032801F2408101A358
:10E9380053F820F09FC80008EDE900089FC80008B8
:10E94800ADE7000841F27013E35C002B3DF4A3AF80
:10E958007E480FF02FFFFDF79EBF7D4B00930320ED
:10E96800A070302305227B49784823F0D5FFFDF7B6
:10E9780092BF03236370FDF78EBF00230AAE3146B2
:10E988001846092210F042FD01287DF484AF0A9B45
:10E9980093F8FE21552A01F0128141F2B4120221A6
:10E9A8000123A1546370FDF776BF0AAE41F2FC174C
:10E9B8003146E0590023092210F028FD01287DF492
:10E9C8006AAF00230A9A2370B2F80B30B3F5007FC0
:10E9D80001F0E38241F2B41203210123A1546370D0
:10E9E800FDF759BF636884F814A00133A36054E7A6
:10E9F800594A5A4DD2ED006A594A95ED006A127883
:10EA0800C4ED646A84ED656A002A00F0238276EE1C
:10EA1800665A94F99821C4ED615A0132C4ED626ACC
:10EA280000F08A85049BC4F89C31002537EE677A8C
:10EA3800FCEEE77A4B4E84ED687A17EE902AA4F83C
:10EA48008C21FF2296ED005A84F89821FEF740B8F1
:10EA5800DFED457A454B94ED687AC3ED007AC3ED56
:10EA6800017AC3ED027A424BF0EE674AF0EE673A5C
:10EA78001968FDF7FDB83F4B1D7805F0010CFDF74F
:10EA880094BC3D49DFED3D7A0968C4ED4C7A11F03C
:10EA9800805840F0C383DAF8001011F4800800F0C1
:10EAA800EC814FF00008B6EE007A67EE877AF4EE54
:10EAB800E57AF1EE10FAC8BFF0EE675A40F3AE837C
:10EAC800C4ED685AFDF71DBB234A244DD2ED007AE8
:10EAD800234A95ED007A1278C4ED647A84ED657A5C
:10EAE800002A00F0318377EE676A94F99821C4ED23
:10EAF800616A0132C4ED627A00F05A86049BC4F858
:10EB08009C3100259FED187A164E84ED687AFF2215
:10EB180096ED005A84F89821FDF7DABF73EEE77A8C
:10EB2800B7EE007AF4EEC77AF1EE10FAC4ED4C7A3B
:10EB380041F3278084EEA77A8DED0A7AFDF7D7BADC
:10EB48007C860020848600207C740020E4850020D8
:10EB5800111B0308AC7C0308F8440020744900200A
:10EB6800445900208849002000000000C8430020C4
:10EB780084680020097100205C46002000000080A5
:10EB880078740020002F00F0CD8625EE866ACC48E8
:10EB9800A5EE076AB0EE675AA6EE265ABDEEC56A1C
:10EBA80016EE10CA16EE107AF445A8BF77466145EE
:10EBB800C8BF0F4606EE107AB8EEC66A012A80ED85
:10EBC800006A3DF4F6AB95ED046A9DED0B5A25EE0F
:10EBD800866AA5EE076AB0EE675AA6EE265ABDEE1B
:10EBE800C56A16EE10CA16EE107AF445A8BF774625
:10EBF8006145C8BF0F4606EE107AB8EEC66A022A0B
:10EC080080ED016A3DF4D5AB95ED086A9DED0C5A8F
:10EC180025EE866AA5EE076AB0EE675AA6EE265A72
:10EC2800BDEEC56A16EE10CA16EE107AF445A8BFF6
:10EC380077466145C8BF0F4606EE107AB8EEC66A39
:10EC4800032A80ED026A3DF4B4AB95ED0C6A9DEDA4
:10EC58000D5A25EE866AA5EE076AB0EE675AA6EE4B
:10EC6800265ABDEEC56A16EE10CA16EE107AF4459D
:10EC7800A8BF77466145C8BF0F4606EE107AB8EEC2
:10EC8800C66A042A80ED036A3DF493AB95ED106AD9
:10EC98009DED0E5A25EE866AA5EE076AB0EE675A14
:10ECA800A6EE265ABDEEC56A16EE10CA16EE107A02
:10ECB800F445A8BF77466145C8BF0F4606EE107AEF
:10ECC800B8EEC66A052A80ED046A3DF472AB95ED8C
:10ECD800146A9DED0F5A25EE866AA5EE076AB0EE16
:10ECE800675AA6EE265ABDEEC56A16EE10CA16EE8B
:10ECF800107AF445A8BF77466145C8BF0F4606EEAF
:10ED0800107AB8EEC66A062A80ED056A3DF451AB62
:10ED180095ED186A9DED105A25EE866AA5EE076AEC
:10ED2800B0EE675AA6EE265ABDEEC56A16EE10CAB0
:10ED380016EE107AF445A8BF77466145C8BF0F465E
:10ED480006EE107AB8EEC66A072A80ED066A3DF428
:10ED580030AB95ED1C6A9DED115A65EE865AE5EECD
:10ED6800075AE6EEA57AFDEEE77A17EE902A964561
:10ED7800A8BF96468A42A8BF714607EE901AF8EED9
:10ED8800E77AC0ED077AFDF714BBBEF1010F7FF7F4
:10ED9800B5AC07EE103AB8EEC77AC7EE876AB1EE9F
:10EDA800E68AADE4BEF1010F40F3E18607EE103AC2
:10EDB800B8EEC77AC7EE876AB1EEE68A032E13D09B
:10EDC8004CB107EE904AF8EEE77AF4EEC87AF1EE25
:10EDD80010FA01F18180DBF8642002EB550292FB06
:10EDE800F5F2CBF824206EE4B0EE480A25F058F985
:10EDF80000B2E5E7BEF1010F40F3B58607EE103A21
:10EE0800B8EEC77AC7EE876AB1EEE68A032E13D04A
:10EE18004CB107EE904AF8EEE77AF4EEC87AF1EED4
:10EE280010FA01F15980DBF8602002EB550292FBE1
:10EE3800F5F2CBF820202BE4B0EE480A25F030F9A3
:10EE480000B2E5E7F7EE006AFDF7FCBCF7EE006AF2
:10EE5800FDF77EBC76EEC65AF0EE466AD9E5822208
:10EE6800FDF7E4BFDFED177AFDF7ACBF164BD3F81B
:10EE780000E0BEF93270FEF792BAB6EE007AF4EE10
:10EE8800C75AF1EE10FA3FF70EAEFDF73AB9D4F8CB
:10EE980024614A003EB1551800EB850576786D78F7
:10EEA800B542BCF405AC0A4400EB82000022C4F869
:10EEB8002401A4F80C22C4F81022FCF7F9BB00BF07
:10EEC8001C440020000002438468002095ED006A7D
:10EED8009DED0A4AE44825EE866AFDEEE43AA4EE82
:10EEE800076AB0EE674AA6EE264A13EE901AB4EE09
:10EEF800C45AF1EE10FAB0EE446A88BFB0EE646A04
:10EF0800BDEEC66A16EE108A16EE107AF045A8BF56
:10EF180077464145C8BF0F4606EE107AB8EEC66A76
:10EF2800012A80ED006A3DF440AA95ED046A9DED42
:10EF38000B4A25EE866AA4EE076AB0EE674AA6EE8B
:10EF4800264AB4EEC45AF1EE10FAB0EE446A88BF0D
:10EF5800B0EE646ABDEEC66A16EE108A16EE107A36
:10EF6800F045A8BF77468845B8BF0F4606EE107A29
:10EF7800B8EEC66A022A80ED016A3DF416AA95ED3C
:10EF8800086A9DED0C4A25EE866AA4EE076AB0EE83
:10EF9800674AA6EE264AB4EEC45AF1EE10FAB0EE6D
:10EFA800446A88BFB0EE646ABDEEC66A16EE108A7F
:10EFB80016EE107AF045A8BF77468845B8BF0F46C9
:10EFC80006EE107AB8EEC66A032A80ED026A3DF4AE
:10EFD800ECA995ED0C6A9DED0D4A25EE866AA4EE26
:10EFE800076AB0EE674AA6EE264AB4EEC45AF1EEB6
:10EFF80010FAB0EE446A88BFB0EE646ABDEEC66A25
:10F0080016EE108A16EE107AF045A8BF77468845A6
:10F01800B8BF0F4606EE107AB8EEC66A042A80ED2D
:10F02800036A3DF4C2A995ED106A9DED0E4A25EEDE
:10F03800866AA4EE076AB0EE674AA6EE264AB4EEE0
:10F04800C45AF1EE10FAB0EE446A88BFB0EE646AB2
:10F05800BDEEC66A16EE108A16EE107AF045A8BF05
:10F0680077468845B8BF0F4606EE107AB8EEC66AEE
:10F07800052A80ED046A3DF498A995ED146A9DED82
:10F088000F4A25EE866AA4EE076AB0EE674AA6EE36
:10F09800264AB4EEC45AF1EE10FAB0EE446A88BFBC
:10F0A800B0EE646ABDEEC66A16EE108A16EE107AE5
:10F0B800F045A8BF77468845B8BF0F4606EE107AD8
:10F0C800B8EEC66A062A80ED056A3DF46EA995ED8C
:10F0D800186A9DED104A25EE866AA4EE076AB0EE1E
:10F0E800674AA6EE264AB4EEC45AF1EE10FAB0EE1C
:10F0F800446A88BFB0EE646ABDEEC66A16EE108A2E
:10F1080016EE107AF045A8BF77468845B8BF0F4677
:10F1180006EE107AB8EEC66A072A80ED066A3DF454
:10F1280044A995ED1C6A9DED114A65EE865AE7EEF5
:10F13800045AE6EEA57AB4EEE75AF1EE10FAC8BF23
:10F14800F0EE647AFDF721B977EEC76AF0EE477AF8
:10F15800CBE4BEF834309FED457A07EE903AF8EEEE
:10F16800E77A434B67EE877AC3ED007AFDF76FB90C
:10F17800404A4FEA89065FEA9C0900EB060802EB61
:10F18800C313264400F0FE8609F101094FEA091964
:10F1980003EB090703F1100208F1100006F1100152
:10F1A80012ED024A12ED035A12ED016A12ED047AC9
:10F1B80050ED024A50ED035A50ED016A50ED047AC1
:10F1C80064EE244A65EE255A66EE266A67EE277ACB
:10F1D8001032974241ED024A41ED035A41ED016A6E
:10F1E80041ED047A00F1100001F11001D8D1A9F124
:10F1F80010094B4408EB09004E441CF0030C3EF484
:10F2080064AFB3EC017AF0EC017A67EE277ABCF1CF
:10F21800010CE6EC017AF4D1FEF757BFB7EE007A9D
:10F2280077EE677AF4EEE75AF1EE10FA88BFF0EE5F
:10F23800675A45E407EE906ADFED0F6AF8EEE77A61
:10F2480066EEA65A9FED0D5A9FED0D6A9FED0D7A59
:10F25800A5EE856A26EEA55AA5EE867AE5EE076A3A
:10F2680026EEA70AFFF75AB91C4400206F12833A0A
:10F2780018000020C840002084F9223F92E741B9D5
:10F288009730083C15A82ABE95ED006A9DED0A4AFC
:10F29800AE4825EE866AFDEEE43AA4EE076AB0EEC3
:10F2A800674AA6EE264A13EE907AB4EEC45AF1EEF7
:10F2B80010FAB0EE446A88BFB0EE646ABDEEC66A62
:10F2C80016EE10CA16EE101AF445A8BF7146674527
:10F2D800C8BF394606EE101AB8EEC66A012A80ED94
:10F2E800006A3DF49FAF95ED046A9DED0B4A25EE4B
:10F2F800866AA4EE076AB0EE674AA6EE264AB4EE1E
:10F30800C45AF1EE10FAB0EE446A88BFB0EE646AEF
:10F31800BDEEC66A16EE10CA16EE101AF445A8BF5E
:10F328007146BC45B8BF394606EE101AB8EEC66A33
:10F33800022A80ED016A3DF475AF95ED086A9DEDEE
:10F348000C4A25EE866AA4EE076AB0EE674AA6EE76
:10F35800264AB4EEC45AF1EE10FAB0EE446A88BFF9
:10F36800B0EE646ABDEEC66A16EE10CA16EE101A42
:10F37800F445A8BF7146BC45B8BF394606EE101A19
:10F38800B8EEC66A032A80ED026A3DF44BAF95EDEC
:10F398000C6A9DED0D4A25EE866AA4EE076AB0EE6A
:10F3A800674AA6EE264AB4EEC45AF1EE10FAB0EE59
:10F3B800446A88BFB0EE646ABDEEC66A16EE10CA2B
:10F3C80016EE101AF445A8BF7146BC45B8BF3946B9
:10F3D80006EE101AB8EEC66A042A80ED036A3DF4F8
:10F3E80021AF95ED106A9DED0E4A25EE866AA4EED2
:10F3F800076AB0EE674AA6EE264AB4EEC45AF1EEA2
:10F4080010FAB0EE446A88BFB0EE646ABDEEC66A10
:10F4180016EE10CA16EE101AF445A8BF7146BC4580
:10F42800B8BF394606EE101AB8EEC66A052A80ED4E
:10F43800046A3DF4F7AE95ED146A9DED0F4A25EE8A
:10F44800866AA4EE076AB0EE674AA6EE264AB4EECC
:10F45800C45AF1EE10FAB0EE446A88BFB0EE646A9E
:10F46800BDEEC66A16EE10CA16EE101AF445A8BF0D
:10F478007146BC45B8BF394606EE101AB8EEC66AE2
:10F48800062A80ED056A3DF4CDAE95ED186A9DED2E
:10F49800104A25EE866AA4EE076AB0EE674AA6EE21
:10F4A800264AB4EEC45AF1EE10FAB0EE446A88BFA8
:10F4B800B0EE646ABDEEC66A16EE10CA16EE101AF1
:10F4C800F445A8BF7146BC45B8BF394606EE101AC8
:10F4D800B8EEC66A072A80ED066A3DF4A3AE95ED3C
:10F4E8001C6A9DED114A65EE865AE7EE045AE6EE6F
:10F4F800A57AB4EEE75AF1EE10FAC8BFF0EE647AD6
:10F50800FDEEE77A17EE901A8E45A8BF8E468F4219
:10F51800D8BF774607EE907AF8EEE77AC0ED077A1B
:10F52800FDF77DBE0A494A69002A3CF48FAA0A6899
:10F5380013604B74FCF78ABAD4F89C51049B5D1B8A
:10F54800FFF774BA034EFCF7F9BF00BF1C44002054
:10F5580090620020A84B0020002F00F0AC83E04D03
:10F568009DED0A4A95ED006A25EE866AA4EE076AC3
:10F57800B0EE674AA6EE264AB0EE446A33B1B4EE5E
:10F58800445AF1EE10FAC8BFB0EE646AFDEEE44AE0
:10F59800BDEEC66A14EE907A16EE101A8F4214EE7B
:10F5A80090CA00F3F2847145A8BF714606EE101A9E
:10F5B800CC48B8EEC66A012A80ED006A3CF4F9AE80
:10F5C80095ED046ADDED0B4A25EE866AA4EE876A9E
:10F5D800F0EE674AE6EE264AB0EE646A002B00F0C9
:10F5E800BB84B4EEE45AF1EE10FA40F3B584394620
:10F5F8007145A8BF714606EE101AB8EEC66A022A0F
:10F6080080ED016A3CF4D5AE95ED086ADDED0C4A53
:10F6180025EE866AA4EE876AF0EE674AE6EE264A89
:10F62800B0EE646A002B00F08D84B4EEE45AF1EE7B
:10F6380010FA40F3878439467145A8BF714606EE33
:10F64800101AB8EEC66A032A80ED026A3CF4B1AE1D
:10F6580095ED0C6ADDED0D4A25EE866AA4EE876A03
:10F66800F0EE674AE6EE264AB0EE646A002B00F038
:10F678005F84B4EEE45AF1EE10FA40F35984394647
:10F688007145A8BF714606EE101AB8EEC66A042A7C
:10F6980080ED036A3CF48DAE95ED106ADDED0E4AFF
:10F6A80025EE866AA4EE876AF0EE674AE6EE264AF9
:10F6B800B0EE646A002B00F03184B4EEE45AF1EE47
:10F6C80010FA40F32B8439467145A8BF714606EEFF
:10F6D800101AB8EEC66A052A80ED046A3CF469AED1
:10F6E80095ED146ADDED0F4A25EE866AA4EE876A69
:10F6F800F0EE674AE6EE264AB0EE646A002B00F0A8
:10F708000384B4EEE45AF1EE10FA40F3FD8339466F
:10F718007145A8BF714606EE101AB8EEC66A062AE9
:10F7280080ED056A3CF445AE95ED186ADDED104AAA
:10F7380025EE866AA4EE876AF0EE674AE6EE264A68
:10F74800B0EE646A002B00F0D683B4EEE45AF1EE12
:10F7580010FA40F3D08339467145A8BF714606EECA
:10F76800101AB8EEC66A072A80ED066A3CF421AE84
:10F7780095ED1C6ADDED114A65EE865AE4EE875A6E
:10F78800E5EEA67A002B00F0AE83F4EEC57AF1EE32
:10F7980010FA40F1A8833A467245A8BF72469446CB
:10F7A80007EE90CAF8EEE77AC0ED077AFCF701BEDB
:10F7B800D4F89C51049B5D1BFFF7A4B996ED000A91
:10F7C8000593039224F06CFC4749DFF850E1D1F827
:10F7D800EC10DFF84CC1039AACF800008EFB013E38
:10F7E800C917C1EBAE1107EE901AF8EEE77A059B40
:10F7F800FDEEE77A17EE901AACF80210FCF7A3BEFC
:10F8080007EE906ADFED396A9FED397A84F8046271
:10F81800F8EEE77A67EEA67A77EE876ABDEEE66AD3
:10F8280016EE103A2033402B40F2B582DFED316AF4
:10F83800314BBDEEE77AC3ED016A17EE103A20337B
:10F84800402B00F2EF829FED2D7AF4EEC77AF1EEAD
:10F8580010FA40F32384DFED2A5A9FED2A6A01E06B
:10F86800F0EE477AF4EEC67AF1EE10FA37EEE57A62
:10F87800F6DCDFED257AB4EEE77AF1EE10FA40F126
:10F888000A84DFED1F5A9FED216A01E0B0EE677A26
:10F89800B4EEC67AF1EE10FA77EE257AF6D49FED3B
:10F8A800147AF4EEC77AF1EE10FA40F3BE829FEDB7
:10F8B800137A77EE677A67EEA75A9FED155A9FED90
:10F8C800156A9FED157AA5EE856A27EEA55AA5EE6D
:10F8D800867AE5EE077AC4ED827AFDF7C1BD00BFEE
:10F8E800F04800201C4400206800002035FA8E3CB7
:10F8F800DB0FC93F0000000018000020DB0F494063
:10F90800DB0FC940E4CB1641DB0F49C0E4CB16C17D
:10F9180092E741B99730083C15A82ABED34D62102A
:10F92800EC64002025EE866AA5EE076AB0EE675AF9
:10F93800A6EE265ABDEEC56A16EE100A814200F3FD
:10F94800B0817045A8BF704606EE100AB8EEC66AC8
:10F95800B8F1000F00F0CF83DE48012A80ED006A7D
:10F968003CF427AD95ED046A9DED0B5A25EE866AA9
:10F97800A5EE076AB0EE675AA6EE265ABDEEC56A2E
:10F9880016EE107AB94200F38A817745A8BF774608
:10F9980006EE107AB8EEC66AB8F1000F00F0E183FF
:10F9A800022A80ED016A3CF404AD95ED086A9DEDEC
:10F9B8000C5A25EE866AA5EE076AB0EE675AA6EEDF
:10F9C800265ABDEEC56A16EE107AB94200F3718167
:10F9D8007745A8BF774606EE107AB8EEC66AB8F142
:10F9E800000F00F0DF83032A80ED026A3CF4E1ACEB
:10F9F80095ED0C6A9DED0D5A25EE866AA5EE076A0F
:10FA0800B0EE675AA6EE265ABDEEC56A16EE107A13
:10FA1800B94200F34C817745A8BF774606EE107AC5
:10FA2800B8EEC66AB8F1000F00F0B183042A80ED81
:10FA3800036A3CF4BEAC95ED106A9DED0E5A25EEB6
:10FA4800866AA5EE076AB0EE675AA6EE265ABDEE9C
:10FA5800C56A16EE107AB94200F327817745A8BF28
:10FA6800774606EE107AB8EEC66AB8F1000F00F0D5
:10FA78008383052A80ED046A3CF49BAC95ED146AF7
:10FA88009DED0F5A25EE866AA5EE076AB0EE675A15
:10FA9800A6EE265ABDEEC56A16EE107AB94200F3F4
:10FAA80002817745A8BF774606EE107AB8EEC66A97
:10FAB800B8F1000F00F01483062A80ED056A3CF4C3
:10FAC80078AC95ED186A9DED105A25EE866AA5EE7C
:10FAD800076AB0EE675AA6EE265ABDEEC56A16EE5C
:10FAE800107AB94200F3CC807745A8BF774606EE76
:10FAF800107AB8EEC66AB8F1000F00F00783072A3B
:10FB080080ED066A3CF455AC95ED1C6A9DED115AE2
:10FB180065EE865AE7EE055AE5EEA67AFDEEE77A37
:10FB280017EE902A914203DC7245A8BF724611462F
:10FB380007EE901AF8EEE77AB8F1000F7FF434AECA
:10FB4800089B002B7FF430AE059B079A9342B8BF01
:10FB5800F0EE647A28E6604A1278032A00F01982E7
:10FB68000022FEF7FABD9FED668AFFF74FB99FEDB9
:10FB7800648AFFF723B9D4F89C51049B5D1BFDF7F9
:10FB8800F5BF5649096811F080587EF48CAFFEF72E
:10FB980082BF9FED530ADFF8588125EE800A24F0D2
:10FBA8007FFAD4F81451A8F80600FDF752B9237D5E
:10FBB800FEF76FBE4B484C498046FEF775BA93F87E
:10FBC800FF21AA2A7EF4E9AED3F8C61149B193F809
:10FBD800C221A2F10B0001282DD902F0F702062A52
:10FBE80029D0D3F8D61149B193F8D221A2F10B004C
:10FBF800012820D902F0F702062A1CD0D3F8E61112
:10FC080049B193F8E221A2F10B00012813D902F0BF
:10FC1800F702062A0FD0D3F8F61100293EF4BDAE3C
:10FC280093F8F231A3F10B02012A04D903F0F70388
:10FC3800062B7EF4B2AE41F2FC120123A150A37050
:10FC4800FEF7B4BEF5F7CEFC029BDFF8A48093F86C
:10FC580000E0039BC01AA8F80200FEF7D5BBF5F731
:10FC6800C1FC029BDFF8888093F800E0039B99F8B9
:10FC78000010D4F81451C01AA8F80400FEF782BB8B
:10FC88000F4634E7F5F7AEFC029BDFF8648093F883
:10FC980000E0039BC01AA8F80200FEF708BB0F4655
:10FCA80076E6084650E60F46FEE60F46D9E60F46CA
:10FCB800B4E60F468FE60AA9BDEEE46A01EB8202BC
:10FCC80094460A48034D09941A4616EE107A43469C
:10FCD8002CE000BF1C4400207C3800205C4600203B
:10FCE8000000C84248420020E0240020F0480020DC
:10FCF800EC64002092E741B99730083C15A82ABE69
:10FD080000000000E4CB1641DB0FC940E4CB16C16C
:10FD1800DB0FC93FDB0F4940DB0FC9BFDB0F49C011
:10FD28006145A5EC016A00F1100031D090ED006A40
:10FD3800B1EC014A25EE866AA7EE046AB0EE674A7E
:10FD4800A6EE864AB0EE446A32B1B4EE445AF1EEF9
:10FD580010FAC8BFB0EE646ABDEEC66A16EE108A25
:10FD6800474506EE107A04DCF045A8BFF04606EEDB
:10FD7800108AB8EEC66A002BD2D1089C002CCFD1CD
:10FD8800059CA046079CA045B8BFB0EE646AC7E7CB
:10FD9800099CFCF70EBBF4EEC77AF1EE10FA40F3BB
:10FDA80081815FED275A1FED296A01E0F0EE476A6D
:10FDB800F4EEC66AF1EE10FA36EEE57AF6DC5FED9F
:10FDC800296AB4EEE67AF1EE10FA40F161815FED4E
:10FDD800325A1FED326A01E0B0EE667AB4EEC67AA6
:10FDE800F1EE10FA77EE256AF6D41FED377AF4EEC5
:10FDF800C76AF1EE10FA40F3B9801FED3A7A77EE50
:10FE0800666A66EEA65A1FED455A1FED456A1FED54
:10FE1800457AA5EE856A26EEA55AA5EE867AE5EE20
:10FE2800076A05E55FED4A7A55E51FED457AF4EE78
:10FE3800C77AF1EE10FA44BF1FED487A77EE677A79
:10FE480039E51FED4C7AF4EEC76AF1EE10FA40F38B
:10FE580012825FED535A1FED556A01E0F0EE476AD2
:10FE6800F4EEC66AF1EE10FA36EEE57AF6DC5FEDEE
:10FE7800556AB4EEE67AF1EE10FA40F16C815FED66
:10FE88005E5A1FED5E6A01E0B0EE667AB4EEC67A9D
:10FE9800F1EE10FA77EE256AF6D41FED637AF4EEE8
:10FEA800C76AF1EE10FA05DD1FED667A77EE666A2D
:10FEB800FFF7C6B91FED687AF4EEC76AF1EE10FADB
:10FEC80044BF1FED6A7A77EE666AFFF7B9B9BD4F8E
:10FED80007F18002FEF73DBAA8F80600ABF8A85073
:10FEE800B84CFBF7ECBBFDEEE77A17EE902ABA4266
:10FEF800FFF656AC50E4BDEEC66A16EE101AB942CB
:10FF0800BFF62AAC39462AE4BDEEC66A16EE101AC8
:10FF1800B942BFF6FDAB3946FFF7FDBBBDEEC66A79
:10FF280016EE101AB942BFF6CFAB3946FFF7CFBB72
:10FF3800BDEEC66A16EE101AB942BFF6A1AB394635
:10FF4800FFF7A1BBBDEEC66A16EE101AB942BFF69E
:10FF580073AB3946FFF773BBBDEEC66A16EE101ACF
:10FF6800B942BFF645AB3946FFF745BB9FED967AD8
:10FF7800F4EEC76AF1EE10FA44BF9FED947A77EE7B
:10FF8800666A3EE74046FFF738B914EE901AFFF765
:10FF98000DBB1EF02BFAFBF78BBB137C022B7EF4F8
:10FFA80019AD92F8FE31552B7EF414AD92F8FF315D
:10FFB800AA2B7EF40FADD689E759854B37441F60CD
:10FFC80092F80DE041F210210EF1FF337F2B44F837
:10FFD80001E03EF6FFACCEF100033EEA03037EF4F7
:10FFE800F9AC4FEA4E2341F21821013B6350D08A05
:08FFF80000B9506A774941F29B
:020000040801F1
:100000000423E050B2F811305B0103F2FF135B12DE
:100010000B60B2F8131001B9116A40001E44064487
:10002000891B41F2082C40F6F476B1FBFEF1B14297
:1000300044F80C1040F21F814FF6F476B14240F2C2
:10004000C08003212170D26A65493B44184441F2C3
:100050000C2641F21C230978A051E25009B923F083
:100060008BFDA3780133A370FCF719BC02287CF444
:1000700016AC41F2B4120123A3546370FCF70FBC19
:1000800021F064FD2369FEF7B2BB94F87831002BB0
:100090007BF4AEADFBF799BDF0EE476AA9E6F0EE52
:1000A000477A00E4B0EE677AFFF7E7BBB0EE667A16
:1000B00089E6132B05D1B0EE480A23F0F5FF069B25
:1000C0001880B0EE480ADBF8083246489847029B91
:1000D0001B78132BB0EE408A7DF4EDA823F0E4FFEB
:1000E000069B5880FDF7E7B8089B002B7FF4E8AC2F
:1000F000059B079FBB42B8BFB0EE646AE0E4089B73
:10010000002B7FF42DAC059B07988342B8BFB0EE5F
:10011000646A25E4089B002B7FF4F5AC059B079FE0
:10012000BB42B8BFB0EE646AEDE42F4BD3ED007A6A
:10013000B1EE677AF4EEC7DAF1EE10FA12D4F4EE0B
:10014000E7DAF1EE10FA88BFF0EE67DA274B87EDB9
:1001500000CA1B689342BBF6A3ABFBF707BCF0EEEB
:10016000476A9EE6F0EE47DAF0E7089B002B7FF443
:100170001BAC059B079FBB42B8BFB0EE646A13E49B
:10018000089B002B7FF479AC059B079FBB42B8BF4F
:10019000B0EE646A71E4089B002B7FF44BAC059BC6
:1001A000079FBB42B8BFB0EE646A43E4089B002BD4
:1001B0007FF41DAC059B079FBB42B8BFB0EE646ADD
:1001C00015E40222227000223EE700BFE024002056
:1001D000DB0FC9BFDB0F49C0748600209486002066
:1001E00054860020A4560020E4480020C84800207F
:1001F000244A254B10681B689847244BD7ED006AAA
:1002000093ED007A224BD3ED007A224B83ED020A64
:10021000214B67EE277A2B4427EEAC7AD3ED007A98
:100220001E4B67EE277AF0EE665AEDEEA75A93ED75
:10023000006AB1EE467AB4EEE57AF1EE10FA08DC27
:10024000F4EEC65AF1EE10FA8CBFB0EE467AB0EE7C
:10025000657A134B1B78012B02D0192B7BF432AC3F
:10026000DFED107AF4EEE7DAF1EE10FACCBF0123FD
:100270000023FBF732BC01232370FEF7AFBBB0EEC7
:10028000667AF8E55C48002070480020B0470020FE
:1002900018000020BC43002080480020E8480020CF
:1002A000F44A0020000096420C4B1B78DB0700D577
:1002B00070470B490B68002BFAD04FF47A7202FB9F
:1002C00003F39842F4D3074B1B781BB9064B9A688B
:1002D0001B69136000230B60704700BF0971002089
:1002E000283000201C3000200830002008B511F014
:1002F000C5FA024B024ADA60FEE700BF00ED00E0FB
:100300000400FA05024A034B1278197809F08AB8FA
:10031000B8240020B92400209F4B1B7803B17047FC
:100320002DE9F0439D4D2B688BB013B90BB0BDE8A0
:10033000F0839B4E9B4A3378044601A8D75C1AF0A1
:100340004AFF736803F5C333A0339C4205D9032FDA
:1003500068D8DFE807F0485C3F10934B1B78DB0759
:10036000E4D42B68002BE1D01B681B68002BDDD088
:1003700020469847DAE704AF38461AF02CFF97E892
:10038000070007AB03C39DF810101A80002974D131
:1003900008A814F03FFE0DF11E0014F053FE38467D
:1003A0000A2207A924F014FE7F4B1A78071C18BFF5
:1003B000012702F001027D49337808787460013327
:1003C00093FBF0F100FB11333370002AC9D0002FEA
:1003D000C7D1ABE7DFF8D08198F8002012F0010216
:1003E00051D00027E7E79DF80430DFF8BC8143B324
:1003F00098F80030D9075CD56C4A3378117874606E
:10040000013393FBF1F201FB123333708EE704A842
:1004100014F018FE0746002840D1634B1A7802F00A
:100420000102C8E7604A614933780978107874603E
:100430000133C00793FBF1F201FB1233337090D507
:1004400074E798F80030DA07D6D404A814F0E2FD77
:10045000002840F0848055493378087898F80020C7
:100460007460013302F0010293FBF0F100FB1133E1
:100470003370002A3FF475AF58E70DF11D0107A84E
:1004800014F0ECFD87E707A814F0D0FD00284AD14E
:1004900098F80020002702F001028CE707A81AF064
:1004A0009AFE9DF81E009DF8103083422ED1002741
:1004B000B3E704A90DF1030014F0D0FD0028CAD061
:1004C00007A81AF088FE9DF81C009DF803309DF8DF
:1004D0001D10834203D19DF810308B42BBD02B6896
:1004E0004BB11A79824206D35A798A4203D31B68E8
:1004F000DB6803B198472D4A337811787460013373
:1005000093FBF1F201FB123333702AE72B68002BC7
:1005100083D09A79824280D31B681B69002B3FF4F9
:100520007CAF984779E7272011F03AFF074600286B
:10053000AED01F4BDB88002BAAD1272011F0D4FEB0
:100540009DF81C308146E8B1002BA1D1012014F0A8
:1005500073FE98F800204F4602F001022BE707A82F
:100560001AF039FEBDF82000BDF8103083423FF488
:1005700072AF2B68002BBED01B689B69002BBAD0D2
:100580009847B8E7002B83D014F056FE98F8002067
:1005900002F001020FE700BF1C4E00200C7100208A
:1005A000F8260020B02F002009710020B42F002071
:1005B000107100202DE9F04F2DED028BA0F10A0300
:1005C00089B00C46ED2B00F26F86DFE813F02201B4
:1005D0006D066D066D066D066D066D066D066D0683
:1005E0006D066D066D066D066D066D066D066D0673
:1005F0006D066D066D066D066D066D066D062F02A5
:100600006D066D066D0625066D066D066D06990173
:100610006D0656016D063E016D0633016D0628021A
:100620006D0603026D06EF016D066D066D06EA01AB
:10063000E4016D06D2016D066D06CC016D06A501C3
:100640006D066D066D0689046D066D066D066D06F8
:100650006B046D0602016D0634063B056D066D06E2
:100660006D066D066D066D066D06FB046D06CE0407
:100670006D069B046D065E056D0659066D066D06DA
:100680006D066D060703EA05E305B205EE006D068B
:100690006D062A03A6026D066F02EB026D066D065B
:1006A0006D066D06E0026D066D06BF026D066D06F5
:1006B0006D06B102F203DF037C036D066D066D0665
:1006C0006E036D066D064E036D066D066D066D06B6
:1006D0006D066D066D066D066D066D066D066D0682
:1006E0006D066D066D0607036D066D066D066D06DB
:1006F0006D066D066D066D066D066D066D066D0662
:100700006D066D066D066D066D066D066D066D0651
:100710006D066D066D066D066D066D066D066D0641
:100720006D066D066D066D066D066D066D066D0631
:1007300040036D066D066D066D066D066D066D0651
:100740006D066D066D066D066D066D066D066D0611
:100750006D066D066D066D066D066D066D066D0601
:100760006D066D066D066D066D066D066D066D06F1
:100770006D066D066D066D066D066D066D066D06E1
:100780006D066D066D066D066D066D066D066D06D1
:100790006D066D066D066D066D06610437046D0607
:1007A0006D066D066D066D060804AF4E337853B1C5
:1007B000AE4F002537F8021F2046F0F74DFE337884
:1007C0000135AB42F6DC012009B0BDEC028BBDE87F
:1007D000F08FA54E3378002BF5D0A54F0025B846F5
:1007E000236817F81520591C21601A7098F8011019
:1007F00001EB810101EB810101F2EE2189B220467A
:10080000F0F72AFE33780135AB4208F10208E7DC45
:10081000D9E7984D284622F0D5FA0028D3DD2B469B
:100820000544226813F8011B501C9D422060117082
:10083000F7D1C8E7904D05F1800655F8041F204612
:10084000F0F7F3FDAE42F8D1BDE78C4D05F140065F
:10085000B5F880102046F0F7FFFD236895F8822058
:10086000591C21601A70236895F883200435591C9F
:10087000AE4221601A70EBD1A5E7814D0B682A7A50
:10088000591C21601A70A98B2046F0F7E5FD298BD1
:100890002046F0F7E1FD698B2046F0F7DDFD236887
:1008A000EA7C591C21601A70A98C2046F0F7D4FD0F
:1008B000E98C2046F0F7D0FD2368AA7F591C2160FF
:1008C0001A70236895F82020591C21601A70698CD1
:1008D0002046F0F7C1FD2368EA7A591C21601A709E
:1008E000E9682046F0F7A1FD23682A7C591C2160A5
:1008F0001A70236895F82120591C21601A7062E74C
:100900000B68604A581C117820601970236852786F
:10091000591C21601A7056E70B685A4A5A4D1178D3
:100920005A4A581C2060197011682046F0F77DFD66
:100930002368534A591C127A21601A70298820466C
:10094000F0F78AFDA9882046F0F786FD2989204620
:10095000F0F782FD20460021F0F77EFD20460021C1
:10096000F0F77AFD2FE7084608224549F0F746FDE3
:1009700029E70B68464A474990785D1C2560187046
:1009800023685278581C20601A7023680A79591C11
:1009900021601A7017E70B680122991821601A70FC
:1009A00011E708460021F0F740FD0CE73A4D3B4EB9
:1009B00005F1300795F90210394B93F906208A4268
:1009C00003F1080300F073849E42F6D10835BD425E
:1009D000F0D1F8E6334B03F15A0522685979501CDF
:1009E0002060117022681978501C206011702268F4
:1009F0005978501C2060117022689978501C206032
:100A000011702268D978501C206011702268197901
:100A10000633501C9D4220601170DED1D3E60B6876
:100A2000174A591C527D21601A70CCE61E4D05F103
:100A3000500628781DF0E6FE2368027A591C2160D2
:100A40001A7023686A78591C21601A702368AA7882
:100A5000591C21601A702368EA780435591CAE428B
:100A600021601A70E5D1AEE6786A00202A3E0020A7
:100A7000BC7300201A3E0020683900206C39002029
:100A80003074002054440020902F0020C0360020F5
:100A9000B0460020BC2400202C5E0020A05C00207A
:100AA000705C0020FC310020B0720020A64D0B6865
:100AB0002A68591C127821601A702B68226899786C
:100AC000531C2360002311702A6821681A440133E3
:100AD0005279481C032B20600A70F5D123682A68DC
:100AE000591C127A21601A7023682A68591CD2781E
:100AF00021601A7023682A68591C127921601A70C3
:100B00002B6820465989F0F7A7FC2A682368527A97
:100B1000591C21601A702A68F8E68C4B084619683F
:100B2000F0F783FC8A4B20461988F0F795FC4AE6DB
:100B3000884D08462988F0F78FFC69882046F0F731
:100B40008BFCA9882046F0F787FC3CE6824D05F136
:100B50006006A9882046F0F77FFCE9882046F0F778
:100B60007BFC29892046F0F777FC2368AA7A591C78
:100B700021601A702368EA7A591C21601A7055F8AE
:100B80000C1B2046F0F751FCAE42E2D11BE6734944
:100B900052232268501C2060137011F8013F002B73
:100BA000F7D110E66E4800232268056803EB430185
:100BB000561C6D5C26601570026825680A446E1C20
:100BC000527826602A70026825680A4401339278B8
:100BD000691C0A2B21602A70E6D1F4E500258146C4
:100BE000DFF89C81DFF89CB1049503950595069587
:100BF00001214FF6FF7A05E001350B2D00F07583DA
:100C000018F9011F4F1C4AFA05F3F5D0DE07F3D59A
:100C1000BBF800302B41D807EED505A8F0F774FFDC
:100C2000EAE7504D08462988F0F716FC6988204607
:100C3000F0F712FCB5F904304B4AD91782FB0323B5
:100C4000C1EBA301204689B2F0F706FCBBE50B68B7
:100C5000464A591C1278216005A81A70F0F7F4FA78
:100C600023685A1C22601870ADE50B68404F591C70
:100C70003A7821601A703B78002B3FF4A4AD002530
:100C8000EEB230461AF032FB23684278591C2160DC
:100C900030461A701AF02AFB01892046F0F7DCFB77
:100CA0003B780135AB42EBDC8DE5324D0846298AB5
:100CB000F0F7D2FB698A2046F0F7CEFBA98A2046DE
:100CC000F0F7CAFB7FE5DFF8C0E00027FEB271460F
:100CD00000232268501C206016702268501C20607F
:100CE0001370226811F8010F0133551C062B256083
:100CF0001070EED10137062F0EF1060EE6D11E4917
:100D000000232268501C206017702268501C20604D
:100D10001370226811F8010F0133551C0B2B25604D
:100D20001070EED12368154A581C072120601970F5
:100D300023680021581C20601970236892F8F02065
:100D4000591C21601A703EE5886800202868002040
:100D50002C680020784900204430002018530308F4
:100D6000846800203068002067666666EE6A0020AE
:100D7000C9640020205900204F3A00206C3900201F
:100D800048530308806800202B3A00200B68A34AD0
:100D9000A3491078A34A5D1C2560187023688978E0
:100DA000581C2060197023689278591C21601A70B1
:100DB00009E50A689C4B9D491878551C2560107000
:100DC00022685878551C2560107022689B78501C4A
:100DD000206013702046C988F0F73EFBF3E405A8B5
:100DE000F0F732FA00283FF4EEACBDF814102046BC
:100DF000F0F732FB23689DF81620591C21601A7009
:100E000023689DF81720591C21601A7023689DF8EB
:100E10001820591C21601A7023689DF81920591C4C
:100E200021601A7023689DF81A20591C21601A70DD
:100E30002046BDF81C10F0F70FFBC4E47C4B03F117
:100E4000700522681978501C20601170226859784A
:100E5000501C2060117022689978501C206011701D
:100E60002268D978501C2060117022681979501CB2
:100E70002060117022685979501C2060117022681E
:100E800099790733501CAB4220601170D9D19AE494
:100E9000634D0846E989F0F7DFFAA9892046F0F7A3
:100EA000DBFA90E40B68634D591C2A7921601A70B3
:100EB00023686A79591C21601A7029882046F0F746
:100EC000CBFA2368AA79591C21601A7069882046D8
:100ED000F0F7C2FA2368EA79591C21601A7072E4AB
:100EE0000B6800255A1C0A60204629461D70F0F741
:100EF0009CFA29462046F0F798FA29462046F0F752
:100F000094FA60E4454E0B6872794B4D591C216090
:100F10001A702B682046198CF0F79EFA2B68204631
:100F2000D98BF0F799FA71892046F0F795FAB189D3
:100F30002046F0F791FA2B682046598CF0F78CFA8E
:100F40002B682046998CF0F787FAF1892046F0F754
:100F500083FA318A2046F0F77FFA2A68236892F8EC
:100F60002620591C21601A702DE42C4EF378002B9A
:100F700000F095820B680822591C21601A702368C2
:100F80000122991821601A7023682C4D591C2A7966
:100F900021601A702368AA78591C21601A70298868
:100FA0002046F0F759FAE9892046F0F755FA236808
:100FB000F279591C21601A702368EA78591C216063
:100FC0001A7000E414F042F9FF28054600F07E8212
:100FD00008A8002300F80C3D14F028F82268184BEC
:100FE000511C2160157022681978501C2060117006
:100FF00022685978501C2060117022689978501C22
:101000002060117022689DF81410501C206011702F
:1010100020469988F0F720FAFFF7D5BB84540020CA
:1010200090460020A04600208846002078490020F5
:1010300004310020944900208468002020590020B9
:10104000107100200B68BB4D591C012221601A70E1
:101050002368AA78591C21601A700BF0CBFF236813
:10106000B54AB6495E1C26601870B1F90010B2F995
:101070000000F0F715FC23685A1C226018702988BC
:101080002046F0F7E9F9FFF79EBB20460021F0F774
:10109000E3F920460021F0F7DFF920460021F0F7C0
:1010A000DBF92368A64D00265A1C22601E702368B7
:1010B0002A68591C92F82C2021601A7023682A682B
:1010C000591C92F8362021601A7023682A68591C2E
:1010D00092F8372021601A7023685A1C22601E7013
:1010E00023685A1C22601E7023685A1C22601E70DE
:1010F0002B682046598FF0F7AFF92B682046198FDF
:10110000F0F7AAF923682A68591C92F82E2021606A
:101110001A7023685A1C22601E702B682046598E54
:10112000F0F79AF92B682046998EF0F795F9FFF7BA
:101130004ABB844D844E9FED858ADFF85082DFEDF7
:10114000848A05F120070EE0FCEEE77ACDED017A06
:10115000BDF8041020460435F0F77EF9BD4206F1D3
:1011600018063FF430AB717C0029F3D0794BD5EDF4
:10117000007A1B78012BE7D1774B1B68DB0440F129
:101180008481F5EE407AF1EE10FA40F0B28140F23F
:10119000DC51DFE7084610227049F0F72FF9FFF71E
:1011A00012BB6F4B9B8AB3F5006F00F27681B3F5EB
:1011B000806F00F29C81B3F5007F34BF01270227C6
:1011C000684D05F10C0655F8041B91FBF7F120461C
:1011D00089B2F0F741F9AE42F5D1634D634F05F1A5
:1011E0000C06B5EC010AD7ED077A80EE270A22F04B
:1011F0005BFF81B22046F0F72FF9AE42F1D15C4D92
:1012000005F10C0655F8041B204689B2F0F724F9C5
:10121000AE42F7D1FFF7D7BA564D08462988F0F706
:101220001BF9A9882046F0F717F929892046F0F71D
:1012300013F9FFF7C8BA0B684F4D01269A190A60D7
:101240001E700EF055FE002840F035814B4B226891
:10125000511C21601070226841F2B410511C185CBE
:10126000216041F27811107059582046890AF0F730
:10127000DCF8A96A20464908F0F7D7F8FFF7A3BAC7
:101280000B683F4A3F49D0783F4A5D1C2560187083
:1012900023684979581C206019702368D278591C3A
:1012A00021601A70FFF78FBA0020FFF78DBA23680C
:1012B0005A1C2260197029882046F0F7CDF823685F
:1012C000EA78591C21601A7023682A79591C216018
:1012D0001A702368AA79591C21601A7023686A79E8
:1012E000591C21601A70FFF771BBDFF8A4A000251C
:1012F0004FF0A8080135C5F1200208FA02F2A5F165
:1013000020032AFA05F6164328FA03F31E43282D74
:1013100006F001024FF000033CD01343EAD0E8B2DC
:1013200011F03EF80028E5D0294605A8F0F7ECFBBF
:10133000E0E700BF6A3E00206C4600206E460020B9
:10134000846800201C4400206058002000004042B7
:1013500000E0824444590020205700200C44002023
:101360003868002068680020145700209854002036
:10137000C4490020902F0020645E00207474002077
:101380009046002020400020A0460020DB9B914199
:1013900090E33FF47B4B1B78DA0700F19280002545
:1013A000794E2F4602E00135282D0DD029463046D2
:1013B000F0F7B9FB0028F6D0294605A8F0F7B3FBF3
:1013C00000285DD10137EEE7704B714DB3F8501036
:1013D0002046F0F741F86F4B1988204689B2F0F7A4
:1013E0003BF86D4B19684B0103F02002C1F3400339
:1013F0001343C1F3800243EA4203C1F3C00243EA4C
:101400008203C1F3401243EAC20301F01001194301
:101410002046F0F721F803A904222046EFF7EEFF5B
:10142000236829785D4A581C206019701188642946
:10143000A8BF64212046F0F70FF8B9F1960F4BD002
:1014400000212046F0F708F82168B7F1190348BFDA
:10145000A7F11203A3F3C4034A1C226020461A46D4
:101460000B7004A9EFF7CAFF23684D4A581C1121DD
:101470002060197020461168EFF7D7FFFFF7A3B976
:10148000394603A8F0F740FB9CE7F4EEC87AF1EE8A
:1014900010FA52DA4FF47A715CE6082790E60B688E
:1014A000B178404A581C2060197023681278591C82
:1014B00021601A7068E595F824203B4BAABB3046A2
:1014C000C5E6059B43F00103059368E723685A1CB2
:1014D00022601870FFF777B923680322591C216036
:1014E0001A7023686A78591C21601A70ACE70427C7
:1014F00066E6F4EEC87AF1EE10FA3FF548AEF4EE87
:10150000E87AFDEEE77AF1EE10FA17EE901A2BD892
:101510006FF4F973303903FB01F140F2E73391FBCB
:10152000F3F101F2DB5189B214E65978022916D0A1
:1015300003290CBF0420304689E6FDEEE77A40F22D
:10154000E73217EE903A303B02FB03F388FB0312BD
:10155000D917C1EB622101F2E93189B2FAE5042A17
:1015600034BF0220032072E640F2F313A1F5836139
:1015700003FB01F140F2E73391FBF3F101F2DD519E
:1015800089B2E7E509710020B870002068000020EA
:101590001C620020385D00202468002026330020D3
:1015A0007C680020844600207474002038B5094D02
:1015B0002B8823EA0000834228800AD0064B14219E
:1015C000FF220E2002241C7059709A701CF02EFF0E
:1015D000288838BD806800203033002038B5094D98
:1015E0002B881843834228800AD0074B1421FF22FE
:1015F0000E2002241C7059709A701CF017FF288866
:1016000038BD00BF8068002030330020024A1368D4
:1016100018431060704700BF7C680020664B674825
:1016200070B55822012500211D7023F0FAFC644A90
:101630006449654C654800230B60136000F01EFD93
:101640002946052000F06AFD6579291C4FF0070046
:1016500018BF012100F062FDA679311C4FF008008F
:1016600018BF012100F05AFDA37A002B7BD0584C03
:10167000002D40F08380311C18BF0121092000F0AB
:101680004DFD2168534DC1F340510F2000F046FD40
:101690002968CA0700F182804C4E11F002016FD117
:1016A000003118BF0121032000F038FD4A4A4B4B9E
:1016B000128E93FBF2F3642BB8BF64230121042044
:1016C000C6F8143100F02AFD454B0620197800F0C9
:1016D00025FD01210A2000F021FD29680B20C1F31E
:1016E000800100F01BFD2B6813F0140F14BF0121C3
:1016F00000210C2000F012FD21680D20C1F3802193
:1017000000F00CFD21684B0508D5364B1B7A083BD1
:10171000012B9CBF4FF4FA63C6F8B432C1F3004109
:101720000E2000F0FBFC21680F20C1F3405100F0B7
:10173000F5FC21681020C1F3804100F0EFFC216826
:101740001120C1F3C06100F0E9FC0121122000F07A
:10175000E5FC0121132000F0E1FC01211420BDE88B
:10176000704000F0DBBCE37A194C002B80D121687B
:1017700011F4802182D0002D3FF47DAF01217DE75F
:101780000121022000F0CAFC174B2968DB6A642B98
:10179000B8BF6423B36701F0020181E7134B0B4E1E
:1017A0001B68642B4FF00101B8BF642308467364C3
:1017B00000F0B4FC296870E728280020D02700201A
:1017C0002C280020CC27002014680020680000206E
:1017D00020570020246800202C5E002040420F008B
:1017E000007300203074002038680020105700205B
:1017F00030B4034600F12405064C07CC0C3343F803
:101800000C0C43F8081C43F8042CAB42F4D130BC58
:10181000704700BF54530308034B33F80C2F02806A
:101820009B788370704700BF54530308084B1968B6
:1018300061B130B45D68074C642202FB05F2B2FB73
:10184000F1F2228030BC002018605860704700BF61
:1018500000270020263300200B4A136803605368DA
:10186000436030B59368094C83601421002301FB69
:1018700003429579AD0602D51379C37230BD0133A9
:10188000082BF4D130BD00BF63530308FC73030879
:10189000704700BF6F4B1B78002B3AD02DE9F04109
:1018A0006D4B6E4D9B79AC68A860013B82B0041B08
:1018B000032B00F29C80DFE803F04A02312910F08C
:1018C00075FD002800F09B80654B66491B78B5F8D4
:1018D0004220D1ED037AEA64DB0700F1AA8002FB23
:1018E00004F007EE900ADFED606A604BB8EEE77A2D
:1018F000D5ED127A5A60E7EE267A1A60BDEEE77AE5
:10190000C5ED127A85ED117A83ED027A02B0BDE859
:10191000F081564A1360536093607047544B1B68C4
:101920001801F3D5FF2019F0E1FC03780A2B88BFDA
:1019300000214E4B9CBFB0F90420B0F90610296578
:1019400088BF0A466A655A601A609960DEE7494AAC
:10195000494BD279DFF8308133F81220B8F90230E0
:101960004648B8F9001092B207EE902A40F6E447D4
:1019700007FB02F6C3EB1633B8EE670A4FF47A762C
:1019800006FB03F393FBF1F3AB61EEF797FDD5F89C
:1019900018E0D5ED047ADFED346AB8F90220334B54
:1019A000B8F900C0C3F804E00EFB04F007EE100A1B
:1019B000B8EEC77ABCEEC06AE7EE267A8DED016A12
:1019C000BDF80410C5ED047ABDEEE77A07FB01F718
:1019D000C2EB173706FB07F683ED027A96FBFCF69F
:1019E00085ED037A6E611E6002B0BDE8F0811F4B89
:1019F00000221A605A609A6002B0BDE8F0811C4B68
:101A00001B68DE067FF560AF154BB5F842201B78EA
:101A1000EA64D9077FF563AFB5F94010184B00FBB6
:101A200001F083FB0013C017C0EBA3100244EA646B
:101A300055E7FDEEE77A134E17EE900AA0F57A719E
:101A400001FB01F386FB0306D817C0EB2610084400
:101A5000E2E700BF12680020146800200027002081
:101A600009710020A84B00202FE33E31F0650020D3
:101A70002057002028620020486200201C270020F8
:101A8000D34D62101F85EB5180460020F0B53E4BD0
:101A90005B79012B83B03DD0022B0FD03B4B002252
:101AA0001A805A803A4B1B78022B05D1374A394BA2
:101AB0005188128819805A8003B0F0BD364B1B68DC
:101AC0001B01EFD5FF2019F011FC03780A2B56D823
:101AD000B0F902203149D31781FB0212C3EBA203F4
:101AE0009BB207EE903AB8EE670A2D4C04F15C0009
:101AF000A4F85A30EEF7E2FCFCEEC07A234AB4F8C0
:101B00005A30CDED017A5380BDF80430A4F8583036
:101B10001380C7E7234A244B9278214D33F81240B3
:101B2000A4B207EE904A05F18400B8EE670AEEF71A
:101B3000C5FC1E4A1549107896785378FCEEC07A99
:101B400000EB4010CDED017ABDF8042044F6FB77A0
:101B5000C3EB033300FB027200FB0474B2FBF3F22D
:101B6000B4FBF3F3B2FBF6F2B3FBF6F392B29BB223
:101B7000A5F88020A5F882300A804B8092E79FED7F
:101B80000C0A0023B1E700BF14680020046600209F
:101B9000E8640020EC640020205700206766666639
:101BA0000027002028620020486200200F35002016
:101BB00000000000F8B52D4D2D4968792D4C2E4BB5
:101BC0002E4E042264270A7001284FF0000184F889
:101BD000A82084F8B170A4F8AA10A4F8AC1084F876
:101BE000B010C4F8B41031701980598021D0022887
:101BF00010D0A979224A00230129136084F8B83053
